:100000000C94A6170C94DF170C94DF170C94DF17D1
:100010000C948B430C948B430C948B430C948B4328
:100020000C94DF170C94DF170C94DF170C94DF1778
:100030000C94DF170C94452B0C94DF170C94DF17EE
:100040000C94DF170C94AC270C948DD00C94DF1714
:100050000C94F58D0C94EB8D0C94DF170C94DF173A
:100060000C94DF170C94DF170C94DF170C94DF1738
:100070000C94DF170C94DF170C94DF170C94DF1728
:100080000C945E820C94DF170C94DF174E414E499E
:100090004E495459494E46CDCCCC3D0AD7233C1746
:1000A000B7D13877CC2B329595E6241FB14F0A0093
:1000B0000020410000C84200401C4620BCBE4CCA83
:1000C0001B0E5AAEC59D7400407A10F35A00A07200
:1000D0004E18090010A5D4E80000E8764817000083
:1000E000E40B54020000CA9A3B000000E1F5050051
:1000F0000080969800000040420F000000A086019A
:10010000000000102700000000E803000000006469
:1001100000000000000A00000000000100000000D4
:10012000002C76D888DC674F0823DFC1DFAE59E1A9
:10013000B1B796E5E3E453C63AE651997696E8E618
:10014000C28426EB898C9B62ED407C6FFCEFBC9CEB
:100150009F40F2BAA56FA5F490055A2AF75C936BFD
:100160006CF9676DC11BFCE0E40D47FEF520E6B5B8
:1001700000D0ED902E0300943577050080841E0892
:100180000000204E0A000000C80C333333330F98B0
:100190006E12831141EF8D2114893BE65516CFFE77
:1001A000E6DB18D1844B381BF77C1D901DA4BBE403
:1001B00024203284725E228100C9F124ECA1E53D45
:1001C000275045544700504C41005072696E7420CE
:1001D00041626F72746564004D3235005061757311
:1001E000696E672E2E2E004D323400454550524F19
:1001F0004D2056657273696F6E204572726F720082
:10020000454550524F4D20496E64657820457272C5
:100210006F7200454550524F4D2043524320457266
:10022000726F72003F0049676E6F726500526573AE
:10023000657400496E697469616C697A6520454529
:1002400050524F4D0000FE0003FF8007C7C007015A
:10025000E00000E00000F00000700400700E00708C
:100260001F00703F80F00E00E00F01E007C7C003E1
:10027000FF8000FE0000FE0003FF8007C7C00F01E3
:10028000E00E00E03F80F01F00700E007004007070
:100290000000700000F00000E00701E007C7C003A5
:1002A000FF8000FE000E000E000E000E000E000E7D
:1002B000000E000E007FC03F801F000E00040004EF
:1002C000000E001F003F807FC00E000E000E000ECB
:1002D000000E000E000E000E00FFFFFF7F80FFC02B
:1002E000FFC0FFC07F807F80FFC0FFC0FFC03F0016
:1002F0001E000C0050726F6265205A204F666673B4
:1003000065740020082046616374002008204D6158
:1003100078002008204D696E004F6666004F6E0021
:100320004175746F74656D700045207374657073EA
:100330002F6D6D005A2053746570732F6D6D0059C9
:100340002053746570732F6D6D0058205374657061
:10035000732F6D6D00416476616E63656420536533
:100360007474696E67730054656D7065726174753D
:1003700072650053746570732F6D6D00436F6E6608
:10038000696775726174696F6E003F004E657874BD
:1003900020436F726E657200446F6E65004E657823
:1003A0007400486F6D696E672058595A0053746F16
:1003B00072652053657474696E6773004C6F616475
:1003C0002053657474696E677300426564205472CB
:1003D000616D6D696E670050726F6265205A204FC3
:1003E0006666736574004661646520486569676880
:1003F00074004F6666004F6E00426564204C65765F
:10040000656C696E67004C6576656C2042656400BA
:100410004732394E00473239004175746F20486FBA
:100420006D65004D6F74696F6E0053572D4D6F648D
:10043000650053746F77004465706C6F7900536585
:100440006C662D5465737400526573657400436F58
:100450006E66696775726174696F6E005265737458
:100460006F72652044656661756C7473004C6F61D2
:10047000642053657474696E67730053746F72659A
:100480002053657474696E677300424C546F7563D2
:10049000680050726F6265205A204F6666736574FB
:1004A00000416476616E6365642053657474696E9F
:1004B0006773004D61696E003F004261636B0053DA
:1004C000746F70004D323200417474616368204D66
:1004D00065646961004D3231005072696E74206646
:1004E000726F6D204D656469610052656C65617362
:1004F00065204D6564696100436F6E66696775725A
:100500006174696F6E0054656D70657261747572A7
:1005100065004D6F74696F6E00526573756D65206F
:100520005072696E740054756E650053746F70205C
:100530005072696E74005061757365205072696EF7
:100540007400496E666F2053637265656E000A4DD4
:100550003234004D3233202573003F0053746172F2
:1005600074205072696E740043616E63656C005054
:1005700072696E740043616E6E6F7420656E74658F
:1005800072207375626469723A200002202E2E0078
:100590000152656672657368004D61696E002100E5
:1005A000486F74656E6420746F6F20636F6C6400B5
:1005B0004261636B0050726F63656564004D6F74D8
:1005C000696F6E0044697361626C65205374657075
:1005D00070657273004D383400426564204C657656
:1005E000656C696E67004175746F20486F6D6500BA
:1005F000473238004D61696E0050726568656174FC
:10060000202420426564005072656865617420246E
:1006100020456E640054656D706572617475726515
:1006200000C601C101436F6F6C646F776E0050723A
:10063000656865617420240046616E2053706565AD
:100640006400426564004E6F7A7A6C65004D6169A2
:100650006E0050726F6265205A204F666673657433
:1006600000466C6F770046616E20537065656400CC
:10067000426564004E6F7A7A6C65005370656564FC
:10068000004D61696E00486F6D696E672046616953
:100690006C6564006F70656E00545249474745525F
:1006A0004544003A20007A5F6D696E00795F6D699C
:1006B0006E00785F6D696E005265706F7274696E5E
:1006C0006720656E6473746F7020737461747573E2
:1006D0000A0020746F6F206C6F6E672065787472EB
:1006E0007573696F6E2070726576656E7465640AE5
:1006F0000020636F6C6420657874727573696F6E27
:100700002070726576656E7465640A00486F6D6569
:100710002025732573257320466972737400576111
:10072000726E696E673A20486F6D696E6720427518
:100730006D702044697669736F72203C20310A0025
:100740000202040000E0C0000000C0000000000041
:100750000068430000634300007A430000A04000AB
:1007600000A04000000040FFFDFCFAF8F6F4F2F0B3
:10077000EEECEAE9E7E5E3E1E0DEDCDAD9D7D5D46F
:10078000D2D0CFCDCBCAC8C7C5C3C2C0BFBDBCBA0B
:10079000B9B7B6B4B3B2B0AFADACAAA9A8A6A5A478
:1007A000A2A1A09E9D9C9A99989795949392908FC0
:1007B0008E8D8B8A8988878684838281807F7E7DE7
:1007C0007B7A797877767574737271706F6E6D6CF1
:1007D0006B6A696867666564636261605F5E5D5CE1
:1007E0005B5A5958585756555453525150504F4EC2
:1007F0004D4C4B4A4A49484746464544434242418C
:10080000403F3E3E3D3C3B3B3A3938383736353544
:10081000343332323130302F2E2E2D2C2B2B2A29EF
:100820002928272726252524232322212120201F8C
:100830001E1E1D1C1C1B1B1A19191818171616151D
:100840001514131312121111100F0F0E0E0D0D0CA3
:100850000C0B0A0A0909080807070606050504041F
:10086000030302020100000000000100000001007B
:10087000008000555555000000400033333300AA76
:10088000AA2A004992240000002000C7711C009988
:10089000991900D1451700555515003BB113002497
:1008A00049120011111100000010000F0F0F00E39A
:1008B000380E0043790D00CCCC0C00C3300C00E89E
:1008C000A20B0064210B00AAAA0A00703D0A009D39
:1008D000D80900427B090092240900DCD308008873
:1008E0008808001042080000000800F0C1070087D7
:1008F00087070075500700711C07003EEB0600A13A
:10090000BC06006990060066660600703E0600613F
:1009100018060017F4050074D105005BB00500B29D
:10092000900500627205005555050078390500B83C
:100930001E0500050505004EEC040087D40400A147
:10094000BD040090A7040049920400C17D0400EE9C
:10095000690400C7560400444404005C32040008E3
:1009600021040041100400000004003FF00300F8DF
:10097000E0030026D20300C3C30300CCB503003A52
:10098000A803000A9B0300388E0300C08103009F68
:10099000750300D0690300505E03001D530300344B
:1009A000480300913D030033330300162903003848
:1009B0001F030097150300300C0300030303000B13
:1009C000FA020049F10200BAE802005CE002002DE0
:1009D000D802002DD0020059C80200B0C002003178
:1009E000B90200DAB10200AAAA0200A0A30200BC68
:1009F0009C0200FA9502005C8F0200DF88020082F0
:100A0000820200457C020027760200277002004324
:100A10006A02007C640200D05E02003F590200C8F6
:100A2000530200000061430000614300007A43006C
:100A300000E0C0000000C00000000053657474694D
:100A40006E67732053746F726564000000FA430090
:100A500000FA430000A0400000C8410000A042008E
:100A600000A0420000C8430080C043F4010000F42D
:100A7000010000640000008813000024F4D430500A
:100A8000C38E20C2A24017828B7011127A910D8101
:100A90006CD90AA861E108C7586607615143061E70
:100AA0004B5D05C145A7041A411104093D98037126
:100AB0003931034036DB0265339102D43054028071
:100AC0002E1D02632CEE01752AC501B028A001106D
:100AD0002781018F2564012B244B01E0223401ACD6
:100AE000211F018D200D01801FFC00841EED009749
:100AF0001DDF00B81CD200E61BC600201BBC006432
:100B00001AB200B219A8000A19A0006A189900D1F7
:100B100017910040178B00B516840031167E00B384
:100B20001579003A157300C7146F0058146A00EE67
:100B30001366008813630025135E00C7125B006C08
:100B400012570015125400C111510070114F0021AD
:100B5000114B00D61049008D10470046104400028A
:100B6000104200C00F4000800F3E00420F3C0006C4
:100B70000F3B00CB0E3800930E37005C0E3500277C
:100B80000E3400F30D3200C10D3100900D300060C5
:100B90000D2E00320D2D00050D2C00D90C2B00AEB2
:100BA0000C2900850C29005C0C2700350C27000E51
:100BB0000C2600E80B2400C40B2400A00B23007DAE
:100BC0000B23005A0B2100390B2100180B2000F8D1
:100BD0000A1F00D90A1E00BB0A1E009D0A1D0080C4
:100BE0000A1D00630A1C00470A1B002C0A1B001187
:100BF0000A1A00F7091A00DD091900C4091900AB27
:100C0000091900920917007B091800630917004CA5
:100C100009160036091600200916000A091500F504
:100C2000081500E0081400CC081400B8081400A44B
:100C3000081400900813007D0812006B0813005878
:100C4000081200460812003408110023081100128F
:100C500008110001081100F0071000E0071000D093
:100C6000071000C0071000B0070F00A10710009187
:100C7000070E0083070F0074070F0065070E00576B
:100C8000070E0049070E003B070D002E070E00203F
:100C9000070D0013070D0006070D00F9060C00ED07
:100CA000060D00E0060C00D4060C00C8060C00BCC3
:100CB000060C00B0060C00A4060B0099060C008D73
:100CC000060B0082060B0077060B006C060B00611A
:100CD000060A0057060B004C060A0042060A0038B6
:100CE000060A002E060A0024060A001A060A001048
:100CF00006090007060A00FD050900F4050900EBD6
:100D0000050900E2050900D9050900D0050900C759
:100D1000050900BE050900B5050800AD050800A5D8
:100D20000509009C050800940508008C050800844E
:100D30000508007C050800740508006C05070065BF
:100D40000508005D050700560508004E0507004729
:100D50000507004005080038050700310507002A8F
:100D6000050700230507001C050600160507000FF0
:100D70000507000805060002050700FB040600F54C
:100D8000040700EE040600E8040600E2040700DBA6
:100D9000040600D5040600CF040600C9040600C3FB
:100DA000040600BD040600B7040600B1040500AC4B
:100DB000040600A6040600A00405009B0406009596
:100DC000040500900406008A0405008504050080DF
:100DD0000406007A04050075040500700405006B24
:100DE00004050066040500610405005C0405005765
:100DF000040500520405004D0405004804050043A5
:100E00000405003E0404003A0405003504050030E2
:100E10000404002C04050027040400230405001E1C
:100E20000404001A04040016040500110404000D53
:100E3000040400090405000404040000040400FC88
:100E4000030400F8030400F4030400F0030400ECBE
:100E5000030400E8030400E4030400E0030400DCEE
:100E6000030400D8030400D4030400D0030400CC1E
:100E7000030400C8030300C503030024F404D920BD
:100E80001BC40C5C0E9804C4095F0265077101F471
:100E900005F900FB04B30048048700C1036900584A
:100EA00003550003034500BE023A0084023100539B
:100EB000022A002902250004022000E4011C00C8C7
:100EC000011900AF0117009801140084011300718B
:100ED0000110006101100051010E0043010D0036A8
:100EE000010B002B010B0020010B00150109000C68
:100EF00001090003010800FB000800F3000800EBF3
:100F0000000700E4000600DE000600D8000600D25C
:100F1000000600CC000500C7000500C2000500BDAA
:100F2000000400B9000400B5000400B1000400ADE5
:100F3000000400A9000400A5000300A20003009F14
:100F40000004009B0003009800030095000200933A
:100F5000000300900003008D0002008B0003008856
:100F60000002008600020084000300810002007F6E
:100F70000002007D0002007B000200790002007781
:100F8000000100760002007400020072000100718E
:100F90000002006F0002006D0001006C0002006A98
:100FA00000010069000200670001006600010065A1
:100FB00000010064000200620001006100010060A5
:100FC0000001005F0002005D0001005C0001005BA9
:100FD0000001005A000100590001005800010057AB
:100FE00000010056000100550001005400010053AB
:100FF00000000053000100520001005100010050A8
:101000000001004F0001004E0000004E0001004DA5
:101010000001004C0001004B0000004B0001004AA1
:10102000000100490001004800000048000100479D
:101030000001004600000046000100450000004598
:101040000001004400010043000000430001004291
:10105000000000420001004100000041000100408A
:101060000001003F0000003F0001003E0000003E84
:101070000001003D0000003D0001003C0000003C7C
:101080000000003C0001003B0000003B0001003A72
:101090000000003A0001003900000039000100386A
:1010A0000000003800000038000100370000003761
:1010B0000001003600000036000000360001003557
:1010C000000000350000003500010034000000344D
:1010D0000000003400010033000000330000003342
:1010E0000001003200000032000000320001003137
:1010F000000000310000003100010030000000302D
:10110000000000300001002F0000002F0000002F21
:101110000000002F0001002E0000002E0000002E15
:101120000001002D0000002D0000002D0000002D0A
:101130000001002C0000002C0000002C0000002CFE
:101140000001002B0000002B0000002B0000002BF2
:101150000001002A0000002A0000002A0000002AE6
:1011600000010029000000290000002900000029DA
:1011700000000029000100280000002800000028CD
:1011800000000028000000280001002700000027C0
:1011900000000027000000270000002700010026B3
:1011A00000000026000000260000002600000026A7
:1011B000000100250000002500000025000000259A
:1011C000000000250000002500010024000000248C
:1011D000000000240000002400000024000100237F
:1011E0000000002300000023000000230000002373
:1011F0000000002300000023000100220000002264
:101200000000002200000022000000220000002256
:101210000001002100000021000000210000002149
:10122000000000210000002100000021000100203A
:10123000000000200000002000000020000000202E
:101240000000002000000020000000200001001F1E
:101250000000001F0000001F0000001F0000001F12
:101260000000001F0000001F0001001E0000001E03
:101270000000001E0000001E000000393000003396
:1012800025000087190000B00F0000DB080000BD3A
:10129000040000740200003F01000020436F756EDF
:1012A0007420583A0042656400453100450062658B
:1012B00064002C2073797374656D2073746F707083
:1012C000656421204865617465725F49443A200075
:1012D0004572723A204D415854454D50004D415889
:1012E00054454D50207472696767657265640048A3
:1012F000656174696E67204661696C656400486564
:101300006174696E67206661696C6564004572721C
:101310003A204D494E54454D50004D494E54454D8F
:10132000502074726967676572656400544845525D
:101330004D414C2052554E415741590054686572F9
:101340006D616C2052756E6177617900202F0020ED
:1013500042403A0020403A007C3C3E5E2B3D3F2F0D
:101360005B5D3B2C2A225C00434F4D4D554E49435B
:101370004154494F4E0044525952554E0045525225
:101380004F525300494E464F004543484F00535477
:101390004F505045442E20005072696E7465722083
:1013A00073746F707065642064756520746F206558
:1013B00072726F72732E204669782074686520659A
:1013C00072726F7220616E6420757365204D3939B9
:1013D0003920746F20726573746172742E202854E2
:1013E000656D7065726174757265206973207265D0
:1013F0007365742E2053657420697420616674656A
:10140000722072657374617274696E67290A004E86
:101410006F20436865636B73756D2077697468200E
:101420006C696E65206E756D6265722C204C6173FF
:1014300074204C696E653A20004E6F2043686563E6
:101440006B73756D2077697468206C696E65206EAA
:10145000756D6265722C204C617374204C696E65E9
:101460003A2000636865636B73756D206D69736DF9
:10147000617463682C204C617374204C696E653A0A
:1014800020004C696E65204E756D6265722069732F
:10149000206E6F74204C617374204C696E65204E11
:1014A000756D6265722B312C204C617374204C6910
:1014B0006E653A20004D3131300053657269616CC0
:1014C00020737461747573206D69736D61746368E2
:1014D0000A0053442072656164206572726F720A5B
:1014E000002121204B494C4C2063617573656420B9
:1014F000627920746F6F206D75636820696E616317
:10150000746976652074696D65202D20637572722B
:10151000656E7420636F6D6D616E643A20004D6579
:1015200064696120496E73657274656400627573E5
:10153000793A2070617573656420666F7220696EF8
:101540007075740A00627573793A207061757365FD
:101550006420666F7220757365720A006275737914
:101560003A2070726F63657373696E670A00506C1E
:1015700065617365205265736574005052494E541D
:1015800045522048414C5445440025533A202553A8
:10159000004B494C4C45442E20005072696E7465D6
:1015A000722068616C7465642E206B696C6C2829EC
:1015B0002063616C6C6564210A0053544F505045A0
:1015C000442E20005072696E7465722073746F70BF
:1015D0007065642064756520746F206572726F7227
:1015E000732E2046697820746865206572726F7268
:1015F00020616E6420757365204D39393920746F10
:1016000020726573746172742E202854656D706544
:101610007261747572652069732072657365742ECA
:101620002053657420697420616674657220726548
:101630007374617274696E67290A006563686F3A32
:10164000004572726F723A004F4646004F4E00429C
:10165000696C696E656172204C6576656C696E6750
:1016600020477269643A0A0021212053544F5020C8
:1016700063616C6C65642062656361757365206F7E
:101680006620424C546F756368206572726F7220D9
:101690002D20726573746172742077697468204DAF
:1016A0003939390A0021212053544F502063616C8D
:1016B0006C65642062656361757365206F662042A6
:1016C0004C546F756368206572726F72202D2072A2
:1016D0006573746172742077697468204D39393983
:1016E0000A004F46460A00466164652048656967FE
:1016F00068742000426564204C6576656C696E678D
:1017000020004661696C656420746F20656E6162BB
:101710006C6520426564204C6576656C696E670A6D
:1017200000496E76616C6964206D6573682E0A00ED
:1017300050726F62696E6720506F696E7400255336
:101740002025692F2569002E0A002F0050726F6234
:10175000696E67206D65736820706F696E74200014
:10176000202844525952554E29004732392041759C
:10177000746F20426564204C6576656C696E670005
:101780003F20284C2C522C462C4229206F75742067
:101790006F6620626F756E64732E0A003F285629AB
:1017A0006572626F7365206C6576656C20696D701B
:1017B0006C61757369626C652028302D34292E0A9E
:1017C00000426164205A2076616C75650A004E6F94
:1017D0002062696C696E65617220677269640A00D3
:1017E0004732384C300020204D3230312058004DE7
:1017F000617820416363656C65726174696F6E2006
:1018000028756E6974732F7332290020204D323091
:10181000332058004D617820666565647261746597
:10182000732028756E6974732F732900205200206D
:10183000204D323034205000416363656C65726125
:1018400074696F6E2028756E6974732F7332292046
:1018500028503C7072696E742D616363656C3E2024
:10186000523C726574726163742D616363656C3E92
:1018700020543C74726176656C2D616363656C3EC7
:101880002900204A0020540020530020204D3230EF
:1018900035204200416476616E6365642028423CD5
:1018A0006D696E5F7365676D656E745F74696D6594
:1018B0005F75733E20533C6D696E5F66656564724B
:1018C0006174653E20543C6D696E5F74726176652B
:1018D0006C5F66656564726174653E204A3C6A753A
:1018E0006E635F6465763E29002044002049002035
:1018F000204D333031205000486F74656E642050A5
:1019000049440020440020490020204D3330342039
:10191000500042656420504944002E0A00206E6F3A
:10192000742064697361626C65642E20536861720F
:101930006564207769746800203B204C6576656C8F
:10194000696E67200020204D3432302053004175ED
:10195000746F20426564204C6576656C696E670023
:1019600020460020420020480020204D3134352000
:1019700053004D6174657269616C206865617475AE
:101980007020706172616D657465727300204A0029
:101990002020473239205720490020204D3134394A
:1019A0002043203B20556E69747320696E20436587
:1019B0006C736975730A0054656D70657261747536
:1019C000726520556E697473002020473231203BC8
:1019D000004C696E65617220556E69747300204910
:1019E0006E76616C696420657874727564657220C6
:1019F00000536C6565702E2E2E005A2050726F6257
:101A0000652050617374204265640A005A20507248
:101A10006F626520506173742042656400205A3AF9
:101A2000200020593A200042656420583A20004D99
:101A300065736820706F696E74206F7574206F66AF
:101A40002072616E67650A00436C69636B20746F76
:101A500020526573756D652E2E2E00616C736F209C
:101A6000656E61626C6564290A004E6F204D6F7669
:101A7000652E004E6F206D656469610A00456E64D5
:101A80002066696C65206C6973740A004265676939
:101A90006E2066696C65206C6973740A00286E6F2D
:101AA0002066696C6529004E6F7420534420707263
:101AB000696E74696E670A005344207072696E74AF
:101AC000696E672062797465200043757272656E75
:101AD000742066696C653A20002E0A0044656C65C6
:101AE00074696F6E206661696C65642C2046696C50
:101AF000653A200046696C652064656C65746564B0
:101B00003A002569730025696D20256973002569F0
:101B1000682025696D202569730025696420256981
:101B2000682025696D20256973002569792025695C
:101B300064202569682025696D202569730050722D
:101B4000696E742074696D653A20006F6B006F6672
:101B50006600891384137D13761368134445425538
:101B6000473A004D3131322053687574646F776E97
:101B7000004D3131332053004D656761205A657245
:101B80006F20322E30204F46462E00434F4E46499E
:101B9000475F4558504F5254004D454154504143C2
:101BA0004B00434F4F4C45525F54454D50455241B9
:101BB00054555245004348414D4245525F54454DAE
:101BC00050455241545552450042414259535445A3
:101BD0005050494E470041524353004D4F54494FD6
:101BE0004E5F4D4F44455300544845524D414C5F64
:101BF00050524F54454354494F4E00455854454E5A
:101C00004445445F4D3230004C4F4E475F46494C8F
:101C1000454E414D45004155544F5245504F525449
:101C20005F53445F5354415455530053445F5752DC
:101C30004954450052455045415400534443415294
:101C4000440050524F4D50545F535550504F5254D2
:101C500000484F53545F414354494F4E5F434F4DEB
:101C60004D414E445300454D455247454E43595F03
:101C700050415253455200434153455F4C494748F8
:101C8000545F4252494748544E45535300544F47BE
:101C9000474C455F4C494748545300534F465457AF
:101CA0004152455F504F574552004255494C445FA1
:101CB00050455243454E54004C4556454C494E47BD
:101CC0005F44415441005A5F50524F4245005255C3
:101CD0004E4F5554004155544F4C4556454C0050BD
:101CE00052494E545F4A4F420050524F475245535B
:101CF00053004155544F5245504F52545F54454D37
:101D000050004155544F5245504F52545F504F531D
:101D100000564F4C554D455452494300454550528D
:101D20004F4D0042494E4152595F46494C455F5420
:101D300052414E534645520053455249414C5F581B
:101D40004F4E5F584F4646004649524D5741524507
:101D50005F4E414D453A4D61726C696E20322E30B6
:101D60002E392E332D6B6164312028446563203277
:101D70003720323032312031333A34343A3130295D
:101D800020534F555243455F434F44455F55524C96
:101D90003A6769746875622E636F6D2F6B61642F8B
:101DA0004D61726C696E2050524F544F434F4C5FDF
:101DB00056455253494F4E3A312E30204D414348FB
:101DC000494E455F545950453A4D656761205A6503
:101DD000726F20322E302045585452554445525F80
:101DE000434F554E543A3120555549443A64626642
:101DF00063636435352D656262612D343631352D6E
:101E0000616264372D31393661613433386633307D
:101E1000340A002F2F004D31343520533C696E6455
:101E200065783E206F7574206F662072616E6765FD
:101E30002028302D31290A003F4A206F7574206F09
:101E4000662072616E67652028302E303120746FF5
:101E500020302E33290A0020580020204D61783A86
:101E60002000200020204D696E3A2000203B2000F9
:101E700020204D32313120530046523A0020466C2A
:101E80006F773A2000206F7574206F662072616E44
:101E900067650A00536572766F20003A2000205370
:101EA0006572766F200050726F6265204F666673B0
:101EB0006574205A0050726F6265204F66667365C4
:101EC00074205A0064697300656E0043290A00613A
:101ED000626C656420286D696E2074656D702000E9
:101EE000436F6C64206578747275646573206172E9
:101EF0006520004D34323120696E636F7272656304
:101F00007420706172616D657465722075736167AC
:101F1000650A004D65736820706F696E74206F7577
:101F200074206F662072616E67650A0045455052E5
:101F30004F4D204F4B0A00290A0020746F20003FAC
:101F40005A206F7574206F662072616E6765202855
:101F500000290A0020746F20003F59206F757420FB
:101F60006F662072616E676520282D00290A0020A7
:101F7000746F20003F58206F7574206F6620726167
:101F80006E676520282D004D383400446F6E652043
:101F90007072696E74696E672066696C650A004DBF
:101FA0003737004D333100496E76616C69642065C6
:101FB000787472756465720A004361703A00202873
:101FC0006D6D2900203B0020204D38353120580010
:101FD0005A2D50726F6265204F66667365740043B8
:101FE0006F6F6C696E672E2E2E0048656174696E86
:101FF000672E2E2E0045312025530020573A002011
:10200000573A0042656420436F6F6C696E672E2EED
:102010002E004265642048656174696E672E2E2E1D
:102020000023646566696E652044454641554C54FD
:102030005F00626564004B6420004B6920004B70B8
:102040002000504944204175746F74756E65206698
:10205000696E6973686564212050757420746865C1
:10206000206C617374204B702C204B6920616E646E
:10207000204B6420636F6E7374616E74732066729C
:102080006F6D2062656C6F7720696E746F20436F8F
:102090006E66696775726174696F6E2E680A0050AA
:1020A0004944204175746F74756E65206661696C72
:1020B0006564212074696D656F75740A0050494428
:1020C000204175746F74756E65206661696C656416
:1020D000212054656D706572617475726520746F2E
:1020E0006F20686967680A00504944204379636C2F
:1020F00065730025532025692F256900204B643A1C
:102100002000204B693A2000204B703A20002043E9
:102110006C617373696320504944200A00204E6F3C
:10212000206F76657273686F6F740A002054753A79
:102130002000204B753A2000206D61783A20002065
:102140006D696E3A200020643A2000206269617354
:102150003A20005761697420666F72206865617467
:102160002075702E2E2E00504944204175746F74D6
:10217000756E652073746172740A00504944204181
:1021800075746F74756E65206661696C6564212075
:1021900054656D706572617475726520746F6F201F
:1021A000686967680A00504944204175746F747506
:1021B0006E6500504944204175746F74756E6520DA
:1021C0006661696C656421204261642068656174A0
:1021D00065722069640A004572723A207574663827
:1021E00020666F6E74206E6F7420696E6974696109
:1021F0006C697A65642E004572723A20757466388F
:1022000020666F6E74206E6F7420696E69746961E8
:102210006C697A65642E004572723A20757466386E
:1022200020666F6E74206E6F7420696E69746961C8
:102230006C697A65642E0042656400456E636C6F5C
:1022400073757265002568753A253032687500250A
:10225000303268753A25303268750025303268753D
:1022600027253032687500202020202020200020E3
:1022700020202000657272001FE020102010201026
:10228000102010202010201030300840048003005F
:102290001FE03FF03FF03FF01FE01FE03FF03FF056
:1022A0003FF00FC0078003003FFFF038007030FCA4
:1022B0003020FC102078102030102C00D02E31D08F
:1022C0002F7BD02F7BD02E31D02C00D0203010206F
:1022D000781020FC1030FC303800703FFFF03FFFDA
:1022E000F03800703186302387102787902F87D0F1
:1022F0002F03D02030102078102078102030102F9D
:1023000003D02F87D027879023871031863038005D
:10231000703FFFF01FFFF81FFFF804104002082075
:1023200002082004104008208010410010410008DD
:1023300020800410400000001FFFF81FFFF8001D60
:10234000C43F0000000C86198000000D0E198000AB
:10235000000F0B198000000D9F198000000DD3990C
:102360008000001CFBFF00000000000000000000D7
:1023700000000000F380001F80007700001980003B
:102380005B1CF6131DAE5B35AB0635FB5B3DA70C46
:10239000BD9B4B30EB19B19BE39D8E9F9D8E000141
:1023A000E00000000001200000000001E00000004B
:1023B000000C0F00FE07022503BB017FFE08FE088C
:1023C000FE05080806000040F0C8888898781005C7
:1023D0000808060000C0F88888888888F805050580
:1023E0000600012030F830200508080600002070A3
:1023F000F820202020E00509090600FF2070A8A889
:10240000B888887020070505070001D86C366CD89D
:102410000509090600FFF8A88888888888A8F805B3
:102420000A0A0600FE205050505088A8A888700361
:10243000030306000340A040FFFFFFFFFFFFFFFF75
:10244000FFFFFFFFFFFFFFFFFFFFFFFFFFFF00009A
:10245000000605FF010707060200808080808000DB
:1024600080030303060105A0A0A0050606060000E0
:1024700050F85050F8500509090600FF2070A8A038
:102480007028A87020050707060000C8C810204063
:10249000989805070706000040A0A040A890680192
:1024A00003030602058080800309090601FF20401E
:1024B000408080804040200309090601FF804040A1
:1024C00020202040408005070706000020A870203B
:1024D00070A8200505050600012020F82020020331
:1024E000030601FFC04080050101060003F8020257
:1024F00002060100C0C005070706000008101020F2
:10250000404080050707060000708898A8C88870BA
:1025100003070706010040C040404040E0050707B0
:10252000060000708808102040F805070706000024
:10253000F8081030088870050707060000103050B2
:1025400090F81010050707060000F880F0080888CA
:1025500070050707060000304080F0888870050786
:1025600007060000F80810102020200507070600C5
:1025700000708888708888700507070600007088DA
:102580008878081060020505060100C0C000C0C0C0
:102590000206060601FFC0C000C040800305050614
:1025A00001012040804020050303060002F800F8E6
:1025B000030505060101804020408005070706004D
:1025C0000070881020200020050707060000708892
:1025D000B8A8B88070050707060000708888F888DA
:1025E0008888050707060000F04848704848F0054D
:1025F000070706000070888080808870050707063E
:102600000000F04848484848F0050707060000F871
:102610008080F08080F8050707060000F88080F0D1
:102620008080800507070600007088808098887089
:10263000050707060000888888F888888803070748
:10264000060100E04040404040E00507070600006A
:10265000381010101090600507070600008890A041
:10266000C0A09088050707060000808080808080D9
:10267000F805070706000088D8A888888888050715
:10268000070600008888C8A89888880507070600FC
:102690000070888888888870050707060000F08821
:1026A00088F080808005070706000070888888A869
:1026B0009068050707060000F08888F0A09088055C
:1026C00007070600007088807008887005070706F5
:1026D0000000F820202020202005070706000088A1
:1026E0008888888888700507070600008888888899
:1026F00050502005070706000088888888A8A85041
:1027000005070706000088885020508888050707BD
:1027100006000088885020202020050707060000BA
:10272000F80810204080F80309090601FFE08080C6
:102730008080808080E00507070600008040402000
:102740001010080309090601FFE0202020202020A6
:1027500020E005030306000520508805010106005E
:10276000FEF8030303060105804020050505060069
:102770000070087888780507070600008080F088D8
:102780008888F005050506000070808088700507C0
:10279000070600000808788888887805050506007F
:1027A000007088F08070050707060000304840E0A0
:1027B0004040400507070600FE708888887808704A
:1027C0000507070600008080F088888888030707CF
:1027D0000601004000C0404040E00409090601FE37
:1027E00010003010101010906005070706000080E0
:1027F000808890E09088030707060100C0404040B1
:102800004040E0050505060000D0A8A8A8A80505D9
:1028100005060000B0C88888880505050600007018
:10282000888888700507070600FEF0888888F08091
:10283000800507070600FE7888888878080805055F
:1028400005060000B0C880808005050506000078F8
:10285000807008F00507070600002020F8202020DF
:10286000180505050600008888889868050505068E
:10287000000088888850200505050600008888A883
:10288000A850050505060000885020508805070758
:102890000600FE8888885020408005050506000057
:1028A000F8102040F80309090601FF20404040804D
:1028B000404040200109090602FF8080808080801E
:1028C0008080800309090601FF804040402040408D
:1028D000408005030306000248A890FF43616E6E26
:1028E0006F74206F70656E2073756264697220006A
:1028F00053442063617264206F6B0A006F70656ED1
:10290000526F6F74206661696C65640A00766F6C43
:10291000756D652E696E6974206661696C65640AFF
:10292000004E6F20534420636172640A002E0A0037
:102930006F70656E206661696C65642C2046696CF9
:10294000653A200046696C652073656C6563746543
:10295000640A002053697A653A200046696C652054
:102960006F70656E65643A2000454E4420535542B1
:10297000524F5554494E450A002220706F73002271
:1029800020706172656E743A2200535542524F5561
:1029900054494E452043414C4C2074617267657424
:1029A0003A220053756263616C6C204F76657266E3
:1029B0006C6F77004578636565646564206D617848
:1029C00020535542524F5554494E4520646570740A
:1029D000683A00667265736800646F696E6700200C
:1029E00066696C653A20004E6F77200057726974F3
:1029F000696E6720746F2066696C653A20006D61AE
:102A0000726C696E66772E6F726700322E302E39C7
:102A10002E332D6B616431001FFFFFFFFFFFFF604E
:102A20000000000001FF400000000000FF800000E7
:102A30000000007F83CF00000C303F87FF80000C38
:102A4000301F867980000C000F8C30C7838C30E7F4
:102A50008C30CFC7CC31F38C30DCECEC33B98C301C
:102A6000D86C6C33198C30D06C0C33198C30D86C1A
:102A70000C33198C30DC6C0E3B198C30CF7C079FEB
:102A8000198C30C77C038F194000000000000260E1
:102A90000000000000061FFFFFFFFFFFF870012C81
:102AA0000190012701B0012201C0011D01F00118B0
:102AB000011002130130020E0160020901900204AC
:102AC00001C002FF000003FA004003F5008003F09C
:102AD00000D003EB002004E6007004E100E004DC19
:102AE000004005D700C005D2004006CD00D006C882
:102AF000008007C3003008BE00F008B900C009B468
:102B000000B00AAF00B00BAA00D00CA500000EA0C8
:102B100000500F9B00C01096005012910000148CC2
:102B200000C0158700B0178200B0197D00D01B7857
:102B300000001E730040206E0090226900F02464A3
:102B40000040275F0090295A00E02B5500102E50BE
:102B50000020304B0010324600E033410090353CFD
:102B6000001037370070383200A0392D00B03A28F5
:102B700000A03B2300603C1E00103D1900903D1456
:102B800000103E0F00703E0A00C03E0500003F00EE
:102B900000403FFBFF803FF6FFC03FF1FF20205089
:102BA0006C616E6E657242756666657242797465B7
:102BB000733A20002046726565204D656D6F72790D
:102BC0003A200020436F6D70696C65643A2044655B
:102BD0006320323720323032310A00204C61737466
:102BE00020557064617465643A20323032312D3082
:102BF000392D3033207C20417574686F723A20285B
:102C00006B61642C20416E796375626963204D6548
:102C10006761205A65726F20322E302041424C206D
:102C2000323456290A004D61726C696E20322E30A2
:102C30002E392E332D6B6164310A0020536F667478
:102C4000776172652052657365740A00205761745C
:102C50006368646F672052657365740A002042726E
:102C60006F776E206F75742052657365740A00204B
:102C700045787465726E616C2052657365740A00E4
:102C8000506F77657255700A0073746172740A0030
:102C90004732385859004D31303031006572726F0B
:102CA000722077726974696E6720746F2066696C30
:102CB000650A00446F6E6520736176696E672066F1
:102CC000696C652E0A004D323900456E6473746F6D
:102CD000707300255320256320256320256320255C
:102CE0006300205A3A0020593A0020583A00656E95
:102CF0006473746F7073206869743A200000000078
:102D0000010200090A000000000403080700000097
:102D100000000000000000000000000000004D6FF7
:102D200076652025736D6D004D6F766520302E31F0
:102D30006D6D004D6F766520316D6D004D6F766560
:102D40002031306D6D004D6F7665204178697300DC
:102D50004D6F7665204578747275646572004D6FAD
:102D60007665205A004D6F76652059004D6F766567
:102D70002058005072696E742066726F6D204D6528
:102D800064696100FFFFFF205A3A200020593A2071
:102D90000042656420583A20004D656761205A65FD
:102DA000726F20322E302052656164792E0050728D
:102DB000696E74696E672E2E2E005072696E7420D3
:102DC00050617573656400204500205A0020590049
:102DD00020204D393220580053746570732070657F
:102DE0007220756E6974003B2000220A00556E6BDC
:102DF0006E6F776E20636F6D6D616E643A20220096
:102E00006F6B00DB0FC93F45BCDA3F8FB30240FC5C
:102E1000F0274056946140FE4B9B4084A5D840E08B
:102E2000231841346A5641E859974164DBD5416E15
:102E3000271742B4B75542CE1A9742C8AED542B50D
:102E4000885A43D40684BFA65FA7BF7443E0BF106F
:102E5000B11AC01C2C58C0E8F697C0B849D6C04E6D
:102E60004E17C124D355C1802497C1A0B5D5C11236
:102E70001A17C244AE55C2781797C26CACD5C26758
:102E8000885AC320746F6F206C6F6E6720657874EA
:102E9000727573696F6E2070726576656E746564A5
:102EA0000A0020636F6C6420657874727573696FB3
:102EB0006E2070726576656E7465640A006F6B0AC9
:102EC00000526573656E643A200020453A00205A2E
:102ED0003A0020593A00583A000000220025002804
:102EE000002B0000002100240027002A000202021B
:102EF000020202020204040404040404040303039F
:102F000003030303030101010101010101010204A3
:102F100008102040800102040810204080010204B3
:102F20000810204080804020100804020145727281
:102F30006F722077726974696E6720746F204545DF
:102F400050524F4D210A000081DD89E411241FBE3B
:102F5000CFEFD0E4DEBFCDBF84B780937A1514BE27
:102F60000FB6F894A8958091600088618093600006
:102F7000109260000FBE12E0A0E0B1E0E0E4F5EED8
:102F800001E00BBF02C007900D92A239B107D9F73B
:102F900025E1A2E9B2E001C01D92AA37B207E1F72C
:102FA00017E1C5EAD7E104C02197FE010E94EEEFC8
:102FB000C43AD107C9F70E9447DE0C9494F20C94EE
:102FC0000000A0E1B0E0E7EEF7E10C9417F08C010F
:102FD000DC01ED91FC910280F381E02DBE016F5F79
:102FE0007F4F0995882309F45DC08981807C91F524
:102FF0006F81637070E0762F6627770F770F888573
:10300000B4E08B9FC0011124682B792B89858295B0
:10301000869586958370682B6F5F7F4F90E080E088
:103020002A852370220F3B8537FB332730F9232B6A
:103030003E813F70230F3327331F2750310904C0CF
:10304000660F771F881F991F2A95D2F76096E4E0D4
:103050000C9433F0803419F568856695669570E0B8
:1030600090E080E0CB01772766272A85622B0985CF
:1030700010E0102F0027012E000C220B330B602BC9
:10308000712B822B932B6F5F7F4F8F4F9F4F4AE0A7
:10309000660F771F881F991F4A95D1F7D7CF8BE00E
:1030A000F801848360E070E0CB01D0CF0895FC018B
:1030B000828108954F925F926F927F928F929F923A
:1030C000AF92BF92CF92DF92EF92FF92CF93DF93B6
:1030D000CDB7DEB728970FB6F894DEBF0FBECDBFD1
:1030E00060913407709135076115710511F1809178
:1030F000300790913107A0913207B091330789834F
:103100009A83AB83BC83072E000C880B990B0E941B
:1031100029E929813A814B815C810E9440F04B0171
:103120005C0120E030E040E251EC0E9423E987FF9F
:1031300007C081E080933401C12CD12C760113C0EB
:1031400020E030E040E251E4C501B4010E94A4F166
:10315000181604F581E080933401C12CD12C9FE72F
:10316000E92E93E4F92EC701B60128960FB6F8941C
:10317000DEBF0FBECDBFDF91CF91FF90EF90DF900C
:10318000CF90BF90AF909F908F907F906F905F9007
:103190004F90089580913B0790913C07A0913D0787
:1031A000B0913E078D839E83AF83B88780913401B1
:1031B000882391F01092A6041092A7041092A804FC
:1031C0001092A9041092A2041092A3041092A404D5
:1031D0001092A504109234012091A6043091A70406
:1031E0004091A8045091A904C501B4010E9441F086
:1031F0002B013C0120E030E0A9010E94A4F1C12C88
:10320000D12C760187FD14C02D813E814F815885D8
:1032100060E070E08FE793E40E94B8F06B017C01FE
:10322000A30192010E9423E9181614F473016201AC
:10323000C092A604D092A704E092A804F092A90438
:1032400020913707309138074091390750913A075C
:10325000C501B4010E9488E94B015C0180929A0487
:1032600090929B04A0929C04B0929D04A7019601A9
:103270006D817E818F8198850E9488E96B017C0138
:10328000C0929E04D0929F04E092A004F092A10408
:103290004090A2045090A3046090A4047090A504F0
:1032A00029813A814B815C816091960470919704E9
:1032B00080919804909199040E9440F020913F07DA
:1032C0003091400740914107509142070E9488E9A0
:1032D000A30192010E9440F020ED3CEC4CE45DE340
:1032E0000E9488E9A30192010E9441F09B01AC0178
:1032F0002093A2043093A3044093A4045093A50404
:1033000089819A81AB81BC818093960490939704C4
:10331000A0939804B0939904C501B4010E9441F0B0
:10332000A70196010E9441F06B017C0120E030E092
:103330004FE753E40E9423E9181634F4C12CD12C32
:103340008FE7E82E83E4F82E20E030E0A901C701E2
:10335000B6010E94A4F187FF06CFEECE6091300740
:103360007091310780913207909133070895FC01E5
:1033700090E1A5E8B4E001900D929A95E1F70895E7
:10338000EF92FF920F931F93E0928B03F0928C03C6
:1033900000938D0310938E03B62F172F022FF32E59
:1033A000242F582FB0938F031093900350939103C1
:1033B0006FEFFF27B01B1F09520B30F4509510958B
:1033C000B195160B560B66276093BB04A6E0BA9F17
:1033D0000092AF04712DEE271A9F700DE11D5A9FC8
:1033E000E00D7093B004E093B104AFE0BA9F009297
:1033F000B304712DEE271A9F700DE11D5A9FE00D49
:103400007093B404E093B504AAE0BA9F0092B704A5
:10341000712DEE271A9F700DE11D5A9FE00D7093DC
:10342000B804E093B9041F910F91FF90EF900895B5
:10343000A5E0B0E0EEE1FAE10C9410F06F36710512
:103440008105910578F4FB01EE0FFF1FEE0FFF1FC2
:10345000E959F74F65917591859194912596EBE027
:103460000C942CF0F62EE72E282FE7E6F7E0002745
:10347000BB275F2D8E2D922F992341F4982F852FF6
:10348000B85F992319F4982F8827B85F903138F4E2
:1034900082959295582F5F70807F952BBC5F9034FA
:1034A00028F4880F991F880F991FBE5F903818F471
:1034B000880F991FB395880F991FE90FF01F54913A
:1034C00081E09927B85079F1C0F0B0FF02C0550FE4
:1034D000881FB1FF04C0550F881F550F881FB2FF0A
:1034E00006C082955295152F1F70507F812BB3FF18
:1034F0001AC0982F852F552716C0B195B0FF02C06E
:1035000085955795B1FF04C0859557958595579535
:10351000B2FF05C08295507F5295582B8F70B3FF34
:1035200002C0582F8827BB247727AA27B2E0F59E30
:10353000B0187109A00BB00BE59E7019A109B00B72
:10354000259FA019B109F89E7019A109B00BE89E3A
:10355000A019B109289FB019F99EA019B109E99ED7
:10356000B0195B9DA12C99244427662733278B9D96
:10357000A00C911C401F601F301F9B9D900C411D93
:10358000601F301F579FA00C911C401F601F301FF1
:10359000879F900C411D601F301F979F400D611D3C
:1035A000301F5A9F900C411D601F301F8A9F400D95
:1035B000611D301F9A9F600D311D5B9F400D611D85
:1035C000301F8B9F600D311D9B9F300DB1E0AA27EE
:1035D0007727BB24F49EB0187109A00BB00BE49EB2
:1035E0007019A109B00B249FA019B109F69E70199A
:1035F000A109B00BE69EA019B109269FB019F39E50
:10360000A019B109E39EB019BF187E09A20B20F0E2
:10361000B1E04B0F601F301F1124762F642F90E014
:10362000832F1CCFFC017081472F50E0062E02C073
:10363000559547950A94E2F740FF14C040911D0448
:1036400050E0062E02C0559547950A94E2F740FFD8
:1036500009C021E030E001C0220F6A95EAF7209509
:103660002723208308958F929F92AF92BF92CF928B
:10367000DF92EF92FF92FC01C080D180E280F38064
:1036800020E030E048EC52E4C701B6010E9488E92E
:103690004B015C0120E030E0A901C701B6010E94A6
:1036A00023E920E030E040EA50E487FF04C020E056
:1036B00030E040EA50ECC501B4010E9441F02DEC2D
:1036C0003CEC4CEC5DE30E9488E90E9420F19B01F8
:1036D0008BE237FF05C022273327261B370B8DE2ED
:1036E00080939902C90168EE73E00E94DBEFCB0181
:1036F000EAE0F0E0BF010E94DBEF805D80939A0278
:10370000C90164E670E00E94DBEFCB01BF010E94BB
:10371000DBEF805D80939B02C901BF010E94DBEF5C
:103720009C01CB01BF010E94DBEF805D80939C0276
:103730008EE280939D02205D20939E0289E992E0B3
:10374000FF90EF90DF90CF90BF90AF909F908F90C1
:1037500008954F925F926F927F928F929F92AF9255
:10376000BF92CF92DF92EF92FF92FC01C080D18096
:10377000E280F38020E030E04AE754E4C701B6017C
:103780000E9488E94B015C0120E030E040E251EC0E
:10379000C701B6010E9423E9181654F420E030E076
:1037A00048EC52E4C701B6010E94A4F187FD8AC02B
:1037B00020E030E0A901C701B6010E9423E987FF9C
:1037C00072C060E070E080EA90ECA50194010E9474
:1037D00041F02DEC3CEC4CEC5DE30E9488E90E944A
:1037E00020F16B017C01F7FC63C020E137E240E08F
:1037F00050E00E9473EFCA01B9012AE030E040E0D6
:1038000050E00E9473EF605D60939902C701B601BA
:1038100028EE33E040E050E00E9473EF9AE0892EFA
:10382000912CA12CB12CCA01B901A50194010E94CF
:1038300073EF605D60939A02C701B60124E630E041
:1038400040E050E00E9473EFCA01B901A501940164
:103850000E9473EF605D60939B028EE280939C02F6
:10386000C701B601A50194010E9473EF6B01CA0163
:10387000B901A50194010E9473EF605D60939D0200
:10388000F0E3CF0EC0929E0289E992E0FF90EF90A4
:10389000DF90CF90BF90AF909F908F907F906F9070
:1038A0005F904F90089560E070E080EA90E48DCFE3
:1038B000F094E094D094C094C11CD11CE11CF11C84
:1038C0006DE2A2CF20E030E0A901C701B6010E945D
:1038D00023E987FF6BC060E070E080EA90ECA5010F
:1038E00094010E9441F02DEC3CEC4CEC5DE30E9415
:1038F00088E90E9420F14B015C0120E030E0A90141
:10390000C701B6010E9423E987FD0BC020E030E02B
:1039100040E251E4C701B6010E94A4F160E287FDD4
:1039200013C0B7FC48C0C501B40128EE33E040E045
:1039300050E00E9473EFCA01B9012AE030E040E094
:1039400050E00E9473EF605D60939A02C501B4017C
:1039500024E630E040E050E00E9473EF8AE0482E19
:10396000512C612C712CCA01B901A30192010E9452
:1039700073EF605D60939B028EE280939C02C501B1
:10398000B401A30192010E9473EF6B01CA01B90156
:10399000A30192010E9473EF605D60939D0280E33A
:1039A000C80EC0929E028AE992E070CF60E070E09B
:1039B00080EA90E494CFB094A09490948094811C79
:1039C000911CA11CB11C6DE2BFCF282F81E32436CE
:1039D00009F080E280939B0290E22A3040F03AE0C6
:1039E000822F632F0E94AEEF0E94AEEF905D909306
:1039F0009C02822F6AE00E94AEEF905D90939D0240
:103A000085E280939E028BE992E0089560912E01F9
:103A100070912F01072E000C880B990B0E9429E949
:103A20002AE037ED43E25CE30E9488E960936F018E
:103A30007093700180937101909372010895CF93F8
:103A4000DF93EC01CB01BA010E9429E923E333E3C0
:103A500043E250E40E9488E920E030E040E05FE388
:103A60000E9441F00E9425F16883DF91CF91089573
:103A70000E9429E923E333E343E250E40E9488E90A
:103A800020E030E040E05FE30E9441F00E9425F139
:103A900024E6629FC001112481589F4F6FEF70E0B0
:103AA0000E94DBEF862F91CF80917407811104C0B3
:103AB000809128078093A70708958091BF148823D9
:103AC000C1F081508093BF14E9EFF2E1882351F0F7
:103AD0008150990B2BE1289FF001299FF00D1124B3
:103AE000EF54FC4E8BE1AEEDB2E101900D928A9560
:103AF000E1F72091BF14211105C08091C9148064A1
:103B00008093C91481E090E0A0E0B0E0211103C0EF
:103B100080E090E0DC0180936A0790936B07A093AC
:103B20006C07B0936D071092650781E0809367077B
:103B300083E080936A010895CF93DF93EC01CB017A
:103B4000BA010E9429E9688379838A839B83DF9184
:103B5000CF910895CF93DF93EC01CB01BA010E947E
:103B600029E92DEC3CEC4CEC5DE30E9488E968838C
:103B700079838A839B83DF91CF910895CF93DF93DD
:103B8000EC01CB01BA010E9429E92AE037ED43E2BA
:103B90005CE30E9488E9688379838A839B83DF9151
:103BA000CF910895CF92DF92EF92FF92CF93DF9360
:103BB00000D000D0CDB7DEB70E9429E92AE037ED6A
:103BC00043E25CE30E9488E96B017C0120E030E085
:103BD000A9010E9423E92DEB37E346E055E387FF77
:103BE00004C02DEB37E346E055EBC701B6010E9458
:103BF00041F069837A838B839C83CE010196A9DD92
:103C00000F900F900F900F90DF91CF91FF90EF905A
:103C1000DF90CF900895CF93DF93EC01CB01BA01F1
:103C20000E9429E90E9420F179836883DF91CF9176
:103C300008958F929F92AF92BF92CF92DF92EF92B0
:103C4000FF92FC01C080D180E280F38020E030E070
:103C5000A901C701B6010E9423E987FD99C06DEB58
:103C600077E386E095E3A70196010E9441F09F77F4
:103C700020E030E048EC52E40E9488E920E030E0A7
:103C800040EA50E40E9441F02DEC3CEC4CEC5DE34A
:103C90000E9488E90E9420F16B017C0180E2809300
:103CA000980260E2F0E1CF16F7E2DF06E104F104EA
:103CB0008CF0C701B60120E137E240E050E00E94FD
:103CC00073EFCA01B9012AE030E040E050E00E9401
:103CD00073EF605D6093990260E288EEC81683E03E
:103CE000D806E104F1048CF0C701B60128EE33E0F8
:103CF00040E050E00E9473EFCA01B9012AE030E0D1
:103D000040E050E00E9473EF605D60939A0260E2D1
:103D1000E4E6CE16D104E104F1048CF0C701B6014B
:103D200024E630E040E050E00E9473EFCA01B901A0
:103D30002AE030E040E050E00E9473EF605D609365
:103D40009B028AE0882E912CA12CB12CC701B601D0
:103D5000A50194010E9473EF6B01CA01B901A5018D
:103D600094010E9473EF605D60939C028EE28093E9
:103D70009D02F0E3CF0EC0929E0288E992E0FF9090
:103D8000EF90DF90CF90BF90AF909F908F9008956D
:103D90006DEB77E386E095EB66CFA4E0B0E0E3ED72
:103DA000FEE10C9419F00E9429E92DEC3CEC4CEC5E
:103DB0005DE30E9488E969837A838B839C83CE01CB
:103DC000019637DF2496E2E00C9435F0CF92DF9233
:103DD000EF92FF92CF93C82F0E94D9CF6B017C0145
:103DE00024EA30E74DE75FE360910A0170910B012F
:103DF00080910C0190910D010E9423E987FD18C06C
:103E00008AEF90E0A0E0B0E08C0D9D1DAE1DBF1DBF
:103E100080939B0390939C03A0939D03B0939E0378
:103E2000C0930001CF91FF90EF90DF90CF90089565
:103E300080E090E0DC01E8CFCF93DF93EC018D814F
:103E40000E942B8E60E08B810E94F4CEDF91CF9197
:103E50000895CF92DF92EF92FF920F931F93CF932B
:103E60008C01C62F69017A01E7DF0E946DD08C2F8B
:103E700080640E941F8E8F2D0E941F8E8E2D0E94A7
:103E80001F8E8D2D0E941F8E8C2D0E941F8E87E805
:103E9000C11101C085E90E941F8ECC3011F40E942F
:103EA000248EC0E00E94248EF801868387FF04C020
:103EB000CF3F11F0CF5FF6CFCF911F910F91FF90C1
:103EC000EF90DF90CF90089561E0FC0183810E9424
:103ED000F4CE8FEF0C941F8E0F931F93CF938C0112
:103EE000ABDF0E946DD0C82F882369F08DEF0E9450
:103EF0001F8E0E946DD0C82FC801E6DF8C2FCF9196
:103F00001F910F91089582E1F8018483F5CFB0E00D
:103F1000A0E0EDE8FFE10C940FF0EC016A017B01F9
:103F20004801590120E030E0A90167E392DFA501D3
:103F3000980167E1CE018DDF81111DC08F81833033
:103F400039F089E0CC0CDD1CEE1CFF1C8A95D1F702
:103F5000A701960169E1CE017CDF11E0882319F009
:103F600010E087E08C83CE01AFDF812FCDB7DEB7C5
:103F7000ECE00C942BF089E08C8310E0F4CFCF932D
:103F8000DF93EC016EBDFA01CA019E5F0DB407FE1E
:103F9000FDCF20812EBD0DB407FEFDCF21812EBDAA
:103FA0003296E817F90791F70DB407FEFDCF8FEFB2
:103FB0000E941F8E8FEF0E941F8E0E94248E8E8380
:103FC0008F71853041F083E18C83CE017DDF80E00D
:103FD000DF91CF91089581E0FBCF0F931F93CF9393
:103FE000DF93EC018B0128DF0E946DD081110BC0A3
:103FF00085E18C8310E0CE0167DF812FDF91CF91C7
:104000001F910F910895A8016CEFCE01B8DF182F12
:10401000882371F3F0CF0F931F93CF93DF93EC01BD
:1040200089018F81833039F089E0440F551F661F65
:10403000771F8A95D1F79A01AB0168E1CE0109DFBC
:10404000811127C0A8016EEFCE0199DF182F8823B8
:10405000A9F00E946DD0182F8823C1F020E030E035
:10406000A9016DE0CE01F5DE882321F086E18C8385
:1040700010E004C00E94248E8111F8CFCE0124DF0D
:10408000812FDF91CF911F910F91089587E18C834C
:10409000F5CF86E0ECCF1F93CF93DF93EC01CCDE1E
:1040A00020E030E0A9016CE0CE01D3DE11E08823EE
:1040B00019F010E083E08C83CE0106DF812FDF91C1
:1040C000CF911F9108951F93CF93DF93EC018F81C0
:1040D000833039F089E0440F551F661F771F8A959A
:1040E000D1F79A01AB0162E1CE01B3DE11E0882382
:1040F00019F010E085E08C83CE01E6DE812FDF91A0
:10410000CF911F9108958F929F92AF92BF92EF929D
:10411000FF920F931F93CF93DF938C01EB017A01F2
:104120000E94D9CF4B015C012CE2820E21E0921E4D
:10413000A11CB11C0E94248EF80186838F3F69F474
:104140000E94D9CF681979098A099B0997FDF2CF96
:1041500081E1F8018483C0E021C08E3F69F5F1E080
:10416000EF1AF1088FEF8EBDFE012FEF0DB407FEA1
:10417000FDCF8EB581932EBDCF018C1B9D0B8E156F
:104180009F05A0F30DB407FEFDCF8EB5CE0DDF1D4C
:1041900088830E94248E0E94248EC1E0C80194DE90
:1041A0008C2FDF91CF911F910F91FF90EF90BF90D7
:1041B000AF909F908F9008958FE0CBCF0F931F9378
:1041C000CF93DF93EC018B0137DE40E052E0B80182
:1041D000CE0199DFDF91CF911F910F9108950F9339
:1041E0001F93CF93DF93EC0189018F81833039F0E6
:1041F00089E0440F551F661F771F8A95D1F79A01F2
:10420000AB0161E1CE0125DE882351F084E08C838F
:10421000CE015ADE80E0DF91CF911F910F9108957A
:1042200040E052E0B801CE016EDFF5CFB0E0A0E093
:10423000ECE1F1E20C940FF0EC01162F1F821C82CE
:104240004B830E94D9CF6B017C0120EDC20E27E089
:10425000D21EE11CF11CA89561E08B810E94F4CE76
:104260008B810E94C2B4249A2C9A279A2698259A68
:1042700081E00E942B8E85E08D830E942B8E0AE0C8
:104280008FEF0E941F8E0150D9F7A89520E030E0F3
:10429000A90160E0CE01DDDD8E83813079F00E94DE
:1042A000D9CF6C197D098E099F0997FDEFCF81E069
:1042B0008C83CE0109DE1A8280E065C0A8952AEAC7
:1042C00031E040E050E068E0CE01C3DD853031F5FB
:1042D00081E08F83A8958F81812C912C54018230AD
:1042E00029F4812C912CA12C80E4B82E20E030E020
:1042F000A90167E3CE01ADDDA501940169E2CE011C
:10430000A8DD8E838823F1F00E94D9CF6C197D0936
:104310008E099F0997FDEACF8AE0CACF04E00E9488
:10432000248E8E830150D9F78A3A11F482E0D1CFDE
:104330000E94D9CF6C197D098E099F0997FDBFCFC7
:1043400082E0B6CF8F818230B9F420E030E0A9015D
:104350006AE3CE017EDD882311F088E0A9CF0E94B8
:10436000248E807C803C11F483E08F830E94248E15
:104370000E94248E0E94248ECE01A6DD81E08A83D5
:10438000173030F41D83CDB7DEB7ECE00C942BF082
:1043900088E18C8391CF0F931F93CF93DF93EC0130
:1043A0008B0120E030E0A90169E053DD882351F062
:1043B00080E18C83CE0188DD80E0DF91CF911F9179
:1043C0000F91089540E150E0B801CE019CDEF5CF99
:1043D000CF93C82FCB010E943E8383EA96E00E94D0
:1043E0003E8384E996E0CC2311F089E996E00E94AF
:1043F0003E838AE00E941D83CF910895EF92FF9241
:104400000F931F93CF937B018A01C2E48F3F09F082
:10441000C4E580E20E941D838C2F0E941D838AE3E5
:104420000E941D83F701608171818281938142E046
:104430000E94E1B48CE493E10E943E83F801608124
:1044400071818281938142E00E94E1B462E070E078
:1044500080E090E00E9450CFCF911F910F91FF908C
:10446000EF9008950C94E5CF4091890321E0422715
:104470006CE070E00C9496B44091890321E04227EF
:1044800064E070E00C9496B44091890321E04227E7
:1044900061E070E00C9496B44091890321E04227DA
:1044A00061E070E00C9496B44091890321E04227CA
:1044B00068E070E00C9496B44091890321E04227B3
:1044C0006CE070E00C9496B441E061E070E00C9414
:1044D00096B44091890321E042270C9496B46CE095
:1044E00070E00C9483CF61E070E00C9483CF61E0C6
:1044F00070E00C9483CF6CE070E00C9483CF64E0A8
:1045000070E00C9483CF9091B00281E089270C94E5
:10451000B67861E088E297E00C94427920E030E0E0
:10452000A901BC0185E791E00C94B0C580E090E062
:10453000A0E8B0E480937D0190937E01A0937F0179
:10454000B09380018AE292E0E9DF80E090E0A0EFA2
:10455000B1E48093750190937601A0937701B093B5
:1045600078018093790190937A01A0937B01B093B5
:104570007C01E091F803EE0FFF0BE65FFD4F8081B9
:1045800091818330910539F184309105C9F1029709
:1045900061F480E090E0A3E4B3E48093750190932C
:1045A0007601A0937701B093780182E192E0B6DFC3
:1045B00010927D0110927E0110927F011092800175
:1045C0008AE292E0ABDF8091F8038F5F8430ECF4F5
:1045D0008093F803089580E090E0A3E4B3E480932F
:1045E000750190937601A0937701B0937801809341
:1045F000790190937A01A0937B01B0937C01D5CF90
:1046000080E090E0A3E4B3E4F2CF1092F8030895C1
:10461000A4E0B0E0EEE0F3E20C9419F084EF91E056
:10462000A0E0B0E089839A83AB83BC83BE016F5F57
:104630007F4F88E70E94E5812496E2E00C9435F0F4
:10464000B0E0A0E0E6E2F3E20C9419F020E24F8142
:1046500058856E818D810E94A7CAE2E00C9435F0E6
:1046600080912807909129070C941AD0609128070F
:104670008FEF0C9424D080912807682F0C9424D0BD
:104680006FEF809128070C9424D06CE472E582E0EF
:104690000C94B5CC60E572E581E00C94B5CC64E592
:1046A00072E580E00C94B5CC68E572E583E00C948B
:1046B000B5CC109265070C94DEDC4FE350E064EC5F
:1046C00074E086EE96E00C947AF280915F139091FC
:1046D0006013891B8F7011F40C94967A81E0089511
:1046E00080916A01882341F06091F0037091F10399
:1046F00041E081E00C9447CA0895CF93DF93EC0129
:104700000E9463D71B82DF91CF910895CF93DF93EF
:10471000EC01462F41706C857D858E859F850E94BA
:1047200074D4882351F0888920E2829FC00111242B
:104730008B569F4EDF91CF91089590E080E0FACFA5
:10474000CF93DF93EB01FC012381211104C080E0B2
:10475000DF91CF9108952250223028F48FE2888390
:10476000198281E0F5CF60E0D1DF009781F3DC01B1
:1047700060E080E09EE22D91203299F0883031F4A3
:104780009E01260F311DF90190836F5F9E01260F58
:10479000311DAD0141505109FA014081F9014083B9
:1047A0006F5F8F5F8B3039F7FE01E60FF11D1082CE
:1047B000D8CFACE0B0E0EFEDF3E20C940AF05C018E
:1047C000DC0159968D909C90F40181859285A3859A
:1047D000B4859C01AD012F5F3F4F4F4F5F4F29873D
:1047E0003A874B875C87D50114964D905D906D900C
:1047F0007C901797411451046104710409F459C065
:10480000BFEF4B1A5B0A6B0A7B0A312C7301620102
:104810001D821E821F821886F40181859285A385E0
:10482000B4852D813E814F815885281739074A0765
:104830005B0708F056C089859A85AB85BC858C15C9
:104840009D05AE05BF0550F482E0C82ED12CE12CA9
:10485000F12C92E0492E512C612C712C9E012F5F7E
:104860003F4FB701A601C4010E947ED68823C9F13B
:1048700089819A81AB81BC81892B8A2B8B2B01F199
:10488000260137019FEF491A590A690A790A2D81D1
:104890003E814F8158852F5F3F4F4F4F5F4F2D8394
:1048A0003E834F8358873FEFC31AD30AE30AF30AC4
:1048B000B3CF408051806280738033243394A6CF7D
:1048C000C414D504E604F70411F70FEF1FEF2FEF20
:1048D0003FE0B701A601C4010E9404D6782E8111E1
:1048E00006C0712C872D2C96E1E10C9426F0F50181
:1048F00044815581668177814115510561057105B6
:1049000039F097018601C4010E9404D6882349F337
:10491000D5011496CD92DD92ED92FC92179733203B
:1049200051F0D701C6010196A11DB11DF40180838C
:104930009183A283B383F50185899689A789B08D78
:10494000892B8A2B8B2B71F6C58AD68AE78AF08E43
:10495000818180688183C6CF40E050E0BA010C9429
:10496000ACD74F925F926F927F92AF92BF92CF92ED
:10497000DF92EF92FF920F931F93CF93DF931F92DB
:10498000CDB7DEB78C017B015A01C22EDB015996EF
:104990008D919C91F801928F818FCB01DDDF712C7D
:1049A000F70180859185A285B38541895289638904
:1049B000748984179507A607B70708F052C055E019
:1049C000B695A795979587955A95D1F7F82FFF70CB
:1049D000DF2ED70113968C91823010F480E0DAC07C
:1049E00041E050E0BE016F5F7F4FC7010E94A7D832
:1049F0000197A1F7F70180859185A285B3854F9630
:104A0000A11DB11D80879187A287B387F0E2DF9E49
:104A1000B00111246B567F4E61157105F9F2DB016F
:104A20008C91882341F0853E09F04BC0772029F016
:104A300077247394B5CF71100EC080919512909128
:104A40009612A0919712B0919812F80184879587D9
:104A5000A687B787D08ADB018C918111E9CF7724B3
:104A600073948C2D8274823409F0B8CF772009F4C6
:104A7000A1C0F801D08861E0C80148DE009709F4C0
:104A8000ADCF20E2DC011D922A95E9F72BE0F5017C
:104A9000DC0101900D922A95E1F721E238E2FC0158
:104AA000318B208B40E058E057874687338B228B31
:104AB000318F208F578B468B0E942BD4811109C0D8
:104AC0008DCF4BE050E0C5010E942AF2892B09F0FE
:104AD00067CFF0E2DF9ED00111249D012B563F4E9F
:104AE000F9018385817121F08C2D827109F000C15B
:104AF000F801818D928D409195125091961260919E
:104B00009712709198124487558766877787D08A65
:104B1000FD01EB56FF4E44885588712C612C320103
:104B200055244424D80155964D925D926D927C9205
:104B30005897428D538D70E060E0442955296629CD
:104B4000772955964D935D936D937C935897D90132
:104B50001B962C91287109F0BDC0848D958DA68D72
:104B6000B78DF801818B928BA38BB48B81E083830B
:104B70008C2D8F70F8018183148215821682178222
:104B8000108611861286138681E0C4FE03C0C80118
:104B90000E9431D80F90DF91CF911F910F91FF901C
:104BA000EF90DF90CF90BF90AF907F906F905F902D
:104BB0004F900895D70113968C911397823009F482
:104BC0000DCF51968D919D910D90BC91A02D803E61
:104BD0009F4FAF41B10508F001CFC701EADD88233F
:104BE00009F4FCCE0E942BD4882309F4F7CED70118
:104BF0005996ED91FC915A9714964D905D906D9059
:104C00007C901797B2E04B1A5108610871088585AE
:104C100004C0440C551C661C771C8A95D2F7868507
:104C20009785A089B189480E591E6A1E7B1E81E0B6
:104C30008093991240929512509296126092971218
:104C400070929812E5E9F0E180E092E0DF019C01CA
:104C50001D9221503040E1F7DD24D394D7015996BD
:104C6000ED91FC918481D816C0F480919A129091B4
:104C70009B12DC01ED91FC910288F389E02D25E97E
:104C800030E1B301A2014D0D511D611D711D09954A
:104C9000882309F4A3CED394E1CF258580E092E068
:104CA000A0E0B0E004C0880F991FAA1FBB1F2A957F
:104CB000D2F7F7014189528963897489840F951F5E
:104CC000A61FB71F818B928BA38BB48B85E990E1D4
:104CD000D12CD7CE203161F498012F5E3F4F0E9436
:104CE000FAD6882329F084E0D80113968C9340CF1C
:104CF000D80113961C9272CEFC0123812111FDCCA8
:104D00000895A1E4B0E0E7E8F6E20C9409F04C0164
:104D10005B017A01222E19821C821C8E1F8E611566
:104D2000710569F410E0CE014C96E6DFCE010196E4
:104D3000E3DF812FCF5BDF4FE2E10C9425F0FC0134
:104D400083818111EFCFFA0180818F3251F18B0184
:104D5000CE0101966C012C0180E2382E360122969C
:104D60003FAE229721963FAE21973FAE3EAE3DAE7D
:104D70003CAE3BAE3AAE39AE38AE3FAA970190E0BA
:104D800047E0D9018D91882309F447C08F3209F497
:104D900044C08E3209F54A3029F298E04AE09D017C
:104DA000F0CFFB01838182508230A0F0618D728D43
:104DB000CE014C960E948FDC882309F4B3CF8E017C
:104DC000045E1F4FC7017C010196F70120812F323D
:104DD000D1F3BECF8B01F6CFE8E5F3E12491222396
:104DE00021F031968213FACF9DCF491708F49ACF5C
:104DF000813208F497CF8F3709F494CF3FE9380F09
:104E00003A3108F420EEE7E3F0E0EC0FFD1FE90F84
:104E1000F11D820F80839F5FC2CF8FA9803209F47A
:104E200081CF7901F90180812F5F3F4F8F32C9F324
:104E30008823C1F021E0AE01495C5F4FB801C60193
:104E400090DD882309F46ECF0A151B0511F0C80107
:104E500054DCCE014C964C145D0409F0C30186016C
:104E60006C017DCF222DAE01495C5F4FB801C401BA
:104E700078DD182F58CFEF92FF921F93CF93DF93D7
:104E8000CDB7DEB728970FB6F894DEBF0FBECDBF03
:104E9000182F8AEAE82E82E1F82EF70160857185E5
:104EA000072E000C880B990B0E9429E96D837E83E5
:104EB0008F839887F70184819581A681B781898343
:104EC0009A83AB83BC83AE014B5F5F4FBE016F5FC4
:104ED0007F4F80E093DA9CE2E92E97E0F92EF7010C
:104EE00060857185072E000C880B990B0E9429E9BB
:104EF0006D837E838F839887F70184819581A68156
:104F0000B78189839A83AB83BC83AE014B5F5F4FCC
:104F1000BE016F5F7F4F8FEF71DA87E11802F001FA
:104F20001124E655FD4E628570E084E593E10E9410
:104F30009B8CF701628570E08FE493E10E949B8C6B
:104F400028960FB6F894DEBF0FBECDBFDF91CF918C
:104F50001F91FF90EF9008950F930FB70F9300915B
:104F60006E000B7F00936E0078940F930BB70F9336
:104F70000CB70F921F922F933F934F935F936F93B2
:104F80007F938F939F93AF93BF93EF93FF931124DE
:104F90000E942165FF91EF91BF91AF919F918F91F9
:104FA0007F916F915F914F913F912F911F900F9043
:104FB0000CBF0F910BBF0F910460F89400936E002B
:104FC0000F910FBF0F911895CF93DF931092990314
:104FD000CAEAD2E1198618860E94E5CF1A865D9842
:104FE000CCE2D7E0198618860E94ED6B1A865C9891
:104FF000DF91CF910895B0E0A0E0E1E0F8E20C94F9
:105000000FF0B0E4A0E06A2F70E0AB014B0F511D30
:1050100055954795411111C0EFE9FAE265917491F8
:10502000072E000C880B990B0E9429E9CDB7DEB73B
:10503000ECE00C942BF0B42FE8CFA41711F0B413CC
:1050400003C0EBE9FBE2EACF9A0121503109220FBC
:10505000331F220F331FF901E356F54DE590F4900D
:10506000F901EF55F54DC591D4918E159F051CF3AF
:10507000A42FC817D9070CF4C6CFF901E156F54D96
:1050800005911491F901ED55F54DC590D490BC01F1
:105090006E197F09072E000C880B990B0E9429E9D5
:1050A0004B015C01B601601B710B072E000C880BD5
:1050B000990B0E9429E99B01AC01C501B4010E9432
:1050C00088E94B015C01BE016E197F09072E000CB7
:1050D000880B990B0E9429E99B01AC01C501B40121
:1050E0000E94B8F06B017C01B801012E000C880B06
:1050F000990B0E9429E99B01AC01C701B6010E94EE
:1051000041F094CFEF92FF920F931F93CF93C82F4C
:105110007B018A0180912707833090F00E94AB8940
:10512000C7010E943E8382EB92E10E943E83CF3F03
:10513000F1F48EEA92E10E943E838AE00E941D8390
:1051400043DFA89580919504811123C081E080936D
:10515000950482E08093270737DF65EA72E1CF3F4D
:1051600011F069EA72E140E0C8010E944D8DC7FD6F
:10517000E4CF8CEA92E10E943E836C2F0C2E000C4F
:10518000770B880B990B0E9497B28AE00E941D83CF
:10519000D4CFCF911F910F91FF90EF900895B0E081
:1051A000A0E0E5EDF8E20C940BF0EC016B014A0194
:1051B000B22EFA014080518062807380A301920177
:1051C0006D817E818F8198850E9423E98823A1F0DB
:1051D0004D825E826F827886AA24A39420E030E01C
:1051E000A901F40160817181828193810E94A4F1FF
:1051F00018160CF0A12CAC828C818230A1F0833087
:1052000009F44FC08130D1F52D813E814F81588501
:10521000F60160817181828193810E9423E987FD7B
:105220002DC082E08C83B7010F2C000C880B990BEA
:105230000E9429E99B01AC016D817E818F81988557
:105240000E9440F09B01AC01F60160817181828176
:1052500093810E94A4F187FD16C00E94D9CF6B01F3
:105260007C019801A8EEB3E00E949FEFC60ED71E06
:10527000E81EF91EC882D982EA82FB82CDB7DEB76A
:10528000E0E10C9427F00E94D9CF088119812A818E
:105290003B81601B710B820B930B97FDEFCF83E07B
:1052A0008C834CE253E16CE373E18B2D2BDFE6CF73
:1052B00040ED52E16DED72E125CFCF93DF93A895DC
:1052C0008091AC129091AD120E940FB46093AE1217
:1052D0007093AF128093B0129093B11280912E0709
:1052E00090912F0788DE6093300770933107809389
:1052F000320790933307C091AC12D091AD128091D8
:10530000630190916401C817D90714F480E0D0DFDD
:105310008091B2129091B312181619066CF4809114
:105320006101909162018C179D0734F44DE053E1C7
:105330006AE173E180E0E6DE20912E0730912F07CD
:105340008091DD069091DE062817390714F48FEF5F
:10535000AFDF8091340790913507181619068CF449
:1053600020912E0730912F0780915F01909160016D
:105370008217930734F44DE053E16AE173E18FEF54
:10538000C1DEDF91CF910895A4E0B0E0EAECF9E24C
:105390000C940FF080912707811106C0A8952496E0
:1053A000ECE00C942BF028C18091AA048111F7CF76
:1053B00081E08093AA0480919A03811107C0109222
:1053C000AA042496ECE00C942BF016C176DF109220
:1053D0009A030E94D9CF4B015C010E94B2B26B01CB
:1053E0007C016091670170916801072E000C880BA9
:1053F000990B0E9429E99B01AC01C701B6010E94EB
:10540000A4F118160CF4E7C06091B2127091B312B7
:10541000072E000C880B990B0E9429E969837A8377
:105420008B839C8334E0E32EF12C08E210E020E033
:10543000AE014F5F5F4F6EEA72E184E193E1AFDE50
:10544000C090AE12D090AF12E090B012F090B112B6
:105450006091650170916601072E000C880B990B15
:105460000E9429E99B01AC01C701B6010E94A4F189
:105470001816CCF46091670170916801072E000C3A
:10548000880B990B0E9429E99B01AC01C701B60169
:105490000E9423E987FF07C00E94BBB20E9420F14F
:1054A0007595679501C060E06093B4128091A61273
:1054B0009091A712A091A812B091A9120097A105EE
:1054C000B105C1F0A5019401281B390B4A0B5B0BF8
:1054D000DA01C901B7FD0EC00E94B2B20E9420F1EC
:1054E0002091A4123091A512621773070CF47DC0AD
:1054F0000E94E5CF0E94AE1920E030E04AEF52E46E
:105500000E94A4F118160CF463C080919503909149
:105510009603A0919703B09198030097A105B10558
:10552000A1F0881A990AAA0ABB0AB7FC0EC00E9409
:10553000AE190E9420F120919303309194036217D9
:1055400073070CF44BC00E94ED6B609134077091AF
:105550003507072E000C880B990B0E9429E96983F7
:105560007A838B839C8392E0E92EF12C04E110E096
:105570002FEFAE014F5F5F4F60E377E08DE193E186
:105580000EDE8090300790903107A0903207B090E7
:10559000330720E030E040EA50E4C501B4010E9446
:1055A000A4F187FD11C020E030E04AEF52E4C501CC
:1055B000B4010E9423E918163CF00E945A180E9478
:1055C00020F17595679501C060E060933607F7CECE
:1055D0008FEF6EDE9ACF80E06BDE16CF4FEE52E19A
:1055E0006EEF72E18FEF8EDDB0CF4FEE52E16EEFD6
:1055F00072E180E087DD7ECFCF92DF92EF92FF9263
:10560000CF93DF93EC01C880D980EA80FB808BE9DF
:1056100092E10E943E83C701B6010E940375CC80CF
:10562000DD80EE80FF8082ED9EE20E943E83C70116
:10563000B6010E940375C884D984EA84FB848EEC89
:105640009EE20E943E83C701B6010E9403758AE074
:105650000E941D83DF91CF91FF90EF90DF90CF905C
:105660000895BC012091760430917704409176042E
:10567000509177042417350731F481E02617370756
:1056800009F080E008959A01F1CF0F930FB70F93BF
:1056900000916E000F930B7F00936E0000916F00DE
:1056A0000D7F00936F000F930BB70F930CB70F9202
:1056B0001F922F933F934F935F936F937F938F939B
:1056C0009F93AF93BF93EF93FF931124E1D4FF9186
:1056D000EF91BF91AF919F918F917F916F915F916A
:1056E0004F913F912F911F900F900CBF0F910BBFC7
:1056F0000F910260F89400936F000F9100936E0079
:105700000F910FBF0F91189500C000C08091E10666
:1057100080FF1FC0459A8FEF80932F048091E10690
:1057200081FF1AC0479A8FEF809330048091E10681
:1057300082FF15C02A988FEF809331048091E10693
:1057400083FF10C028988FEF8093320400C000C000
:105750000895459881E0E0CF479881E0E5CF2A9A07
:1057600081E0EACF289A81E0EFCF80918A03982FD9
:10577000977F90938A03982F937081E011F080E0D7
:1057800008955E9A08955E9880918A038860809358
:105790008A030895E82FF0E021E030E0082E02C0EF
:1057A000220F331F0A94E2F72095309590918A03D7
:1057B000922390938A03EA50FE4F2081922321E0A6
:1057C00019F020E0822F0895813079F038F082308E
:1057D000C9F7159A909177079B7F04C05E9A9091C4
:1057E00077079E7F90937707EDCF5E9A909177072A
:1057F0009D7FF8CF80E0CEDF81E0CCDF82E0CADFA2
:10580000B4CF813079F070F0823071F021E030E077
:1058100001C0220F8A95EAF780918A03822B809338
:105820008A0308955E98F2CF1598F0CFB0E0A0E01B
:10583000ECE1FCE20C9411F0C9E6DDE00FE817E0C2
:1058400089E7A82E8DE0B82EC12CD12C7601C39407
:1058500069917991899199910E9427E928893989DB
:105860004A895B890E9488E90E9425F1F8016193C9
:105870007193819391938F01C616D706E806F906B6
:1058800010F46B017C01AC16BD0611F76FEF7FEFD2
:10589000CB01A70196010E9451EF20939F073093FF
:1058A000A0074093A1075093A207CDB7DEB7EAE067
:1058B0000C942DF00F931F93CF93DF930DE71DE012
:1058C000C8EAD7E0F80121913191419151918F01BE
:1058D00060E070E080E89FE30E94B8F069937993FC
:1058E00089939993F7E0C83BDF0761F70E94D3C51E
:1058F0009DDFDF91CF911F910F910895DBCFDACF1C
:10590000D9CFD8CF90915F1380916013981306C0C0
:105910008091B10D9091B20D892B21F080E00E9411
:105920003C8EF0CF089590915F138091601398138F
:1059300007C08091B10D9091B20D892B09F45ACF17
:1059400080E00E943C8EEFCFCF92DF92EF92FF92E9
:10595000CF93DF932091B002222319F1EC01089636
:105960000E9467766B017C0120E030E0A9010E9473
:1059700023E920E030E0A901882349F0CE010E940C
:10598000DF76A70196010E9488E99B01AC0168853A
:1059900079858A859B850E9440F0688779878A8708
:1059A0009B87DF91CF91FF90EF90DF90CF9008958C
:1059B000CF92DF92EF92FF92CF93DF932091B002CC
:1059C000222319F1EC0108960E9467766B017C0195
:1059D00020E030E0A9010E9423E920E030E0A901A5
:1059E000882349F0CE010E94DF76A70196010E942C
:1059F00088E99B01AC01688579858A859B850E9431
:105A000041F0688779878A879B87DF91CF91FF90E4
:105A1000EF90DF90CF900895AEE1B0E0E2E1FDE2DB
:105A20000C940BF09E8F8D8F5B018A01FC01EA5B69
:105A3000FF4F2081318142815381298B3A8B4B8BDF
:105A40005C8BCA01B9010E9427E96B017C01D50179
:105A50002D913D914D915C910E9488E90E94A5F0A5
:105A60002B013C01F8012081318142815381C70122
:105A7000B6010E9488E90E94A5F04B015C01C301B8
:105A8000B2010E9425F16D8B7E8B8F8B988F6837CA
:105A900071058105910540F428E730E040E050E0D1
:105AA0002D8B3E8B4F8B588FC501B4010E9425F181
:105AB000698F7A8F8B8F9C8F68377105810591056F
:105AC00040F488E790E0A0E0B0E0898F9A8FAB8F38
:105AD000BC8FED8DFE8DEE5AFF4F208131814281CA
:105AE000538129873A874B875C87CA01B9010E9495
:105AF00029E92B013C016D897E898F89988D0E944F
:105B000027E96D837E838F83988720E030E0A901A9
:105B1000C301B2010E9423E9882309F4BBC1A70194
:105B20009601C701B6010E9488E94B015C012D81F5
:105B30003E814F815885CA01B9010E9488E99B01C5
:105B4000AC01C501B4010E9440F04B015C01A3010E
:105B50009201C301B2010E9441F09B01AC01C50159
:105B6000B4010E94B8F00E94A5F00E9425F169835B
:105B70007A838B839C8369857A858B859C859095B8
:105B80008095709561957F4F8F4F9F4F0E9429E9B7
:105B90004B015C01698D7A8D8B8D9C8D0E9427E96C
:105BA00069877A878B879C8720E030E0A901C5014F
:105BB000B4010E9423E9882309F470C129853A853C
:105BC0004B855C85CA01B9010E9488E96D877E8793
:105BD0008F87988BA7019601C701B6010E9488E9BB
:105BE0009B01AC016D857E858F8598890E9440F070
:105BF0006B017C01A5019401C501B4010E9441F033
:105C00009B01AC01C701B6010E94B8F00E9451F19E
:105C1000AD8DBE8D95962D913D914D915C9198974E
:105C20002D873E874F87588B69017A0129813A81F8
:105C30004B815C81C21AD30AE40AF50A0E9425F15D
:105C4000C61AD70AE80AF90AF7FE8CC02D813E81F0
:105C50004F815885CA01B9010E9488E96B017C0116
:105C600020E030E0A901C301B2010E9423E98823AA
:105C700009F418C16D857E858F8598890E9427E972
:105C80009B01AC010E9441F0A30192010E9488E9AE
:105C90004B015C0129853A854B855C85CA01B901B8
:105CA0000E9488E99B01AC01C501B4010E9441F04A
:105CB000A70196010E9440F04B015C0120E030E01A
:105CC00040E850E4C301B2010E9488E99B01AC01A5
:105CD000C501B4010E94B8F00E94A5F04B015C011F
:105CE00020E030E0A9010E94A4F187FF03C0812CCD
:105CF000912C5401C501B4010E9425F169837A8376
:105D00008B839C832D853E854F85588926173707C1
:105D10004807590720F429833A834B835C836981C0
:105D20007A818B819C810E9427E94B015C01A30150
:105D30009201C301B2010E9441F09B01AC01C50177
:105D4000B4010E9488E9A70196010E9441F00E94D7
:105D5000DDF10E9425F1698B7A8B8B8B9C8BC12C9A
:105D6000D12C760169897A898B899C892D893E8914
:105D70004F89588D621B730B840B950B0E9427E98A
:105D8000A30192010E94B8F020E034E244EF59E40C
:105D90000E9488E90E9425F14B015C0169897A899A
:105DA0008B899C89298D3A8D4B8D5C8D621B730B81
:105DB000840B950B0E9427E9A30192010E94B8F081
:105DC00020E034E244EF59E40E9488E90E9425F182
:105DD0006D837E838F839887C501B4010E94181A52
:105DE0002B013C016D817E818F8198850E94181A5C
:105DF00029813A814B815C81AD8DBE8D99962D9321
:105E00003D934D935C939C9789019A010C0D1D1D48
:105E10002E1D3F1DFD0105A716A727A730ABE65B8A
:105E2000FF4F2D893E894F89588D208331834283CE
:105E30005383D5968D929D92AD92BC92D8972D8129
:105E40003E814F815885D9962D933D934D935C9318
:105E5000DC973D97408251826282738234966083E0
:105E600071838283938329893A894B895C89D1968E
:105E70002D933D934D935C93D4973D96298D3A8D08
:105E80004B8D5C8D20833183428353836E96E0E19A
:105E90000C9427F060E070E0CB0165CE60E070E02C
:105EA000CB01B4CE60E070E0CB0116CF90916F00D3
:105EB00081E091FD02C080E0089590916F009D7F88
:105EC00090936F000895EFE6F0E080818260808318
:105ED0000895CF93C82FEADF94E0C99F9001112461
:105EE000F901E758FB4F2B573B4FD9014D915D917D
:105EF0006D917C91408351836283738391E0909391
:105F000078048111E0DFCF910895CF93DF938091E2
:105F1000E006811105C08091E206882309F44EC095
:105F200080910A04329B4DC0816080930A04809165
:105F30000A04339B48C0826080930A0480910A045B
:105F4000349B43C0846080930A04C0916904C0FFFD
:105F50000FC08091E10680FF0BC080910A0480FF92
:105F600007C08091260781608093260780E0B1DF1B
:105F7000C1FF0FC08091E10681FF0BC080910A0430
:105F800081FF07C08091260782608093260781E009
:105F9000A0DFC2FF13C08091E10682FF0FC0809195
:105FA000E206882359F080910A0482FF07C080919D
:105FB000260784608093260782E08BDFDF91CF91F4
:105FC00008958E7FB2CF8D7FB7CF8B7FBCCF6EDF32
:105FD0001092A3071092A4071092A5071092A6078B
:105FE000811171CF08950F931F9380915F1390914A
:105FF0006013891B8F7009F449C090915C13992339
:1060000061F0833040F48FEF890F29F080935C13A7
:1060100090E080E038C010925C13809160132BE513
:10602000829FC00111248854984FFC01208120FDDB
:10603000EFCF4091A3075091A4076091A5077091FD
:10604000A607E95AFF4F0081118122813381401B4D
:10605000510B620B730B4093A3075093A4076093FB
:10606000A5077093A607209160132F5F2F702093D0
:106070005D133091601320915E13321304C02091A0
:106080005D1320935E131F910F910895A0DFC0CF81
:10609000A3E1B0E0EEE4F0E30C9409F08FEF9FEFA2
:1060A00090938900809388002AE02983312C212C49
:1060B00078948091720490917304A0917404B091CB
:1060C0007504892B8A2B8B2B09F0C2C1809178042F
:1060D0008823D1F08091760490917704109278040F
:1060E000892B91F010927704109276041092690433
:1060F00090915F1380916013981731F08091601335
:106100008F5F8F70809360138091760490917704F5
:10611000892B09F49DC140916E0450916F046091E8
:1061200070047091710480916A0490916B04A09145
:106130006C04B0916D040091600410E030E020E048
:10614000841B950BA60BB70B081719072A073B07EB
:1061500010F4D901C8018A8B840F951FA61FB71FA1
:1061600080936E0490936F04A0937004B0937104B5
:10617000E1E0C0903704D0903804E0903904F0900A
:106180003A048091470490914804A0914904B09149
:106190004A04C80ED91EEA1EFB1EC0924704D092C4
:1061A0004804E0924904F0924A04F7FC33C040915D
:1061B0002F04042E000C550B660B770B8091850481
:1061C00090918604A0918704B0918804840F951F54
:1061D000A61FB71F8093850490938604A09387041D
:1061E000B09388048091330490913404A0913504D5
:1061F000B0913604B701A601481B590B6A0B7B0B03
:10620000DB01CA018093470490934804A09349049A
:10621000B0934A0400913B0410913C0420913D044A
:1062200030913E0480914B0490914C04A0914D0418
:10623000B0914E04080F191F2A1F3B1F00934B04F7
:1062400010934C0420934D0430934E0437FD33C01B
:1062500040913004042E000C550B660B770B809197
:10626000890490918A04A0918B04B0918C04840FCE
:10627000951FA61FB71F8093890490938A04A0934B
:106280008B04B0938C048091330490913404A091DA
:106290003504B091360428013901481A590A6A0AAE
:1062A0007B0AD301C20180934B0490934C04A093CA
:1062B0004D04B0934E0440913F04509140046091CE
:1062C00041047091420480914F0490915004A09138
:1062D0005104B0915204480F591F6A1F7B1F40930D
:1062E0004F0450935004609351047093520477FD0F
:1062F00033C080903104082C000C9908AA08BB0810
:1063000080918D0490918E04A0918F04B09190049F
:10631000880D991DAA1DBB1D80938D0490938E043A
:10632000A0938F04B093900480913304909134042F
:10633000A0913504B09136043A014B01681A790AEC
:106340008A0A9B0AD401C30180934F04909350049E
:10635000A0935104B093520480904304909044045D
:10636000A0904504B0904604809153049091540449
:10637000A0915504B0915604880D991DAA1DBB1D0E
:106380008093530490935404A0935504B0935604FF
:10639000B7FD33C040903204042C000C5508660849
:1063A00077088090910490909204A0909304B0900C
:1063B0009404840C951CA61CB71C809291049092A6
:1063C0009204A0929304B09294048090330490902D
:1063D0003404A0903504B09036042C013D014818D7
:1063E00059086A087B085301420180925304909235
:1063F0005404A0925504B0925604E11104C0E091F7
:106400008400F0918500F7FE5F9A37FF469A77FF88
:106410002B9AB7FF299AE0918400F0918500E091D2
:106420008400F0918500F7FE5F9837FF469877FF6C
:106430002B98B7FF29985A88552021F08091840025
:10644000909185002A8921502A8BE0E0211191CE7C
:106450008091720490917304A0917404B0917504BA
:10646000892B8A2B8B2B09F0B0C640907604509074
:1064700077045B8A4A8A4114510409F402C7809167
:106480006E0490916F04A0917004B09171044091DA
:106490006A0450916B0460916C0470916D048417D0
:1064A0009507A607B70708F449C010927704109221
:1064B00076041092690490915F138091601398178D
:1064C00009F4DFC6809160138F5F8F708093601333
:1064D000A0EDCA2EA7E0DA2EE12CF12C80917604F3
:1064E00090917704892B09F068C67DDD909377043D
:1064F00080937604892B09F460C64090760450900E
:1065000077045B8A4A8AD2018C9183FF08C5C20155
:1065100045960E94B7191092770410927604109253
:10652000690490915F13809160139817F1F2809144
:1065300060138F5F8F7080936013D7CF4091650495
:106540005091660460916704709168044817590778
:106550006A077B0708F40FC24091610450916204FE
:106560006091630470916404EA89FB8985A996A906
:10657000A7A9B0AD481759076A077B0708F0D0C133
:10658000411551056105710509F066C080908F03C2
:1065900090909003A0909103B09092038BE792E1CA
:1065A000A1E0FC010591159125913491081519057B
:1065B0002A053B0558F4B694A79497948794AA0F9C
:1065C0000496E7E9F2E1E817F90759F7A0936004A8
:1065D000F0E28F169104A104B10428F4E0E28E2EBB
:1065E000912CA12CB12C20E2821A9108A108B108AB
:1065F000811438E09306A104B10408F49AC1A4E020
:106600009A9EC00111248558914FFC013296259124
:106610003491B82DEE27B39F8001B29F010D1E1F4C
:1066200006940E1F1E1F112430E020E0FC01C590CF
:10663000D490F12CE12CC01AD10AE20AF30A4C0DD5
:106640005D1D6E1D7F1D4093610450936204609335
:1066500063047093640442CF10E00A81942F852E66
:10666000862FBC81AD81FE81EF81388529854B80E5
:10667000E0918B03E99FA12DFF2730918C03399F77
:10668000A00DF11D10908D03199EF00DE89DA00D39
:10669000F11D389DF00DE89FF00D4A2EBF2F4A9E48
:1066A000E12D332722274F9EE00D311D211FBA9F78
:1066B000E00D311D211FBF9F300D211D432EB22F34
:1066C0004A9E012D332722274F9E000D311D211F89
:1066D000BA9F000D311D211FBF9F300D211D432E7C
:1066E000B22FEE2790918F038090900380919103B9
:1066F0000090BB04012A09F483C03091B704349D93
:10670000E119910B810A810B2091B804249DE019B5
:106710009109810A810B0091B904049D90198108A7
:10672000810B3B9FE0199109810A810B2B9F9019E6
:106730008108810B0B9F801881094A9E012D332708
:1067400022274F9E000D311D211FBA9F000D311DC4
:10675000211FBF9F300D211D432EB22F3091B30456
:10676000349DE10D911F811E811F2091B404249D51
:10677000E00D911D811E811F0091B504049D900DB7
:10678000811C811F3B9FE00D911D811E811F2B9F4E
:10679000900D811C811F0B9F800C811D4A9E012D35
:1067A000332722274F9E000D311D211FBA9F000D58
:1067B000311D211FBF9F300D211D432EB22F30915F
:1067C000AF04349DE119910B810A810B2091B00433
:1067D000249DE0199109810A810B0091B104049D67
:1067E00090198108810B3B9FE0199109810A810B67
:1067F0002B9F90198108810B0B9F8018810982C003
:106800003091B704349DE10D911F811E811F2091AD
:10681000B804249DE00D911D811E811F0091B904D3
:10682000049D900D811C811F3B9FE00D911D811ED9
:10683000811F2B9F900D811C811F0B9F800C811D40
:106840004A9E012D332722274F9E000D311D211F07
:10685000BA9F000D311D211FBF9F300D211D432EFA
:10686000B22F3091B304349DE119910B810A810B51
:106870002091B404249DE0199109810A810B0091B3
:10688000B504049D90198108810B3B9FE019910983
:10689000810A810B2B9F90198108810B0B9F801817
:1068A00081094A9E012D332722274F9E000D311D5D
:1068B000211FBA9F000D311D211FBF9F300D211DCB
:1068C000432EB22F3091AF04349DE10D911F811EF4
:1068D000811F2091B004249DE00D911D811E811F18
:1068E0000091B104049D900D811C811F3B9FE00D20
:1068F000911D811E811F2B9F900D811C811F0B9F5D
:10690000800C811D11244B820A83BC83AD83FE83DE
:10691000EF8338872987982C892EB12CA82E3ECE5C
:10692000AA89BB89D1968D909D90AD90BC90D4974B
:1069300035CED501C401B695A795979587958C7FDF
:106940008558954FFC01C590D490FC013296259155
:106950003491E82DE7708E2EE29FC001E39F900DE9
:10696000112433E0969587953A95E1F7C81AD90A2C
:10697000F12CE12C64CE40915C0450915D04609157
:106980005E0470915F04481759076A077B0708F097
:1069900030C28090570490905804A0905904B09051
:1069A0005A0480915B04EA89FB8981117CC0EF5B0A
:1069B000FF4FE080F18002811381EA89FB89E25B6D
:1069C000FF4F2081318142815381AA89BB89D196B1
:1069D0006D917D918D919C91D4970E94C019B1E0E9
:1069E000B0935B04EA89FB8941A952A963A974A900
:1069F0008BE792E1A1E0FC0105911591259134917D
:106A0000041715072607370758F4769567955795A5
:106A10004795AA0F0496E7E9F2E1E817F90759F755
:106A2000A0936004403251056105710520F440E2F5
:106A300050E060E070E04052510961097109411570
:106A4000F8E05F076105710508F4B3C124E0529FC7
:106A5000C00111248558914FFC0132962591349143
:106A6000AA27439FF001429FE10DFA1F0694EA1FF7
:106A7000FA1F1124AF0170E060E0FC01C590D490D2
:106A8000F12CE12CC41AD50AE60AF70A8C0C9D1CDD
:106A9000AE1CBF1C8092570490925804A0925904D7
:106AA000B0925A041BCD81AD92ADA3ADB4AD8816A2
:106AB0009906AA06BB0608F072C181149104A104CC
:106AC000B10449F440918F03509190036091910378
:106AD000709192038DCFA0E0BA85982D492D8A2D13
:106AE000FB85EC857D856E855F8538892989509188
:106AF0008B03599F712D662730918C03399F700D40
:106B0000611D10908D03199E600D549F700D611DC5
:106B1000349F600D589F600DF72FE62FF79F512D82
:106B200033272227F69F500D311D2A1FE79F500D56
:106B3000311D2A1FE69F300D211DF32FE22FF79FF5
:106B4000B12D33272227F69FB00D311D2A1FE79F55
:106B5000B00D311D2A1FE69F300D211DF32FE22FAE
:106B6000552790918F03409190038091910300905D
:106B7000BB040A2A09F483C03091B7043F9F51191E
:106B80009A0B4A0B8A0B2091B8042F9F5019910938
:106B90004A0B8A0BB091B904BF9F901941098A0B27
:106BA0003E9F501991094A0B8A0B2E9F901941095B
:106BB0008A0BBE9F40198109F79FB12D33272227E9
:106BC000F69FB00D311D2A1FE79FB00D311D2A1F02
:106BD000E69F300D211DF32FE22F3091B3043F9F2C
:106BE000510D9A1F4A1F8A1F2091B4042F9F500DE8
:106BF000911D4A1F8A1FB091B504BF9F900D411D82
:106C00008A1F3E9F500D911D4A1F8A1F2E9F900D77
:106C1000411D8A1FBE9F400D811DF79FB12D332757
:106C20002227F69FB00D311D2A1FE79FB00D311DA1
:106C30002A1FE69F300D211DF32FE22F3091AF0464
:106C40003F9F51199A0B4A0B8A0B2091B0042F9F3A
:106C5000501991094A0B8A0BB091B104BF9F90194A
:106C600041098A0B3E9F501991094A0B8A0B2E9FAE
:106C7000901941098A0BBE9F4019810982C0309149
:106C8000B7043F9F510D9A1F4A1F8A1F2091B804D5
:106C90002F9F500D911D4A1F8A1FB091B904BF9FAD
:106CA000900D411D8A1F3E9F500D911D4A1F8A1F46
:106CB0002E9F900D411D8A1FBE9F400D811DF79F85
:106CC000B12D33272227F69FB00D311D2A1FE79FD4
:106CD000B00D311D2A1FE69F300D211DF32FE22F2D
:106CE0003091B3043F9F51199A0B4A0B8A0B2091A4
:106CF000B4042F9F501991094A0B8A0BB091B50427
:106D0000BF9F901941098A0B3E9F501991094A0B68
:106D10008A0B2E9F901941098A0BBE9F4019810949
:106D2000F79FB12D33272227F69FB00D311D2A1F63
:106D3000E79FB00D311D2A1FE69F300D211DF32F57
:106D4000E22F3091AF043F9F510D9A1F4A1F8A1FB7
:106D50002091B0042F9F500D911D4A1F8A1FB091A2
:106D6000B104BF9F900D411D8A1F3E9F500D911D84
:106D70004A1F8A1F2E9F900D411D8A1FBE9F400DE6
:106D8000811D1124BA87FB87EC877D876E875F871B
:106D9000388B298B542F492F70E0682F29CE2A89F0
:106DA0003B89225B3F4FD9014D915D916D917C9163
:106DB0001FCEDB01CA01B695A795979587958C7F65
:106DC0008558954FFC01C590D490FC0132962591D1
:106DD00034914770429FC001439F900D1124A3E05E
:106DE00096958795AA95E1F7C81AD90AF12CE12C56
:106DF0004DCE8091300190913101A0913201B0913E
:106E00003301B7FF61C0EA89FB89EA5BFF4FC080AD
:106E1000D180E280F3808BE792E121E0FC01459193
:106E20005591659174914C155D056E057F0558F47B
:106E3000F694E794D794C794220F049647E952E159
:106E40004817590759F72093600450E2C516D1043A
:106E5000E104F10428F470E2C72ED12CE12CF12CCE
:106E600060E2C61AD108E108F108C11478E0D7063B
:106E7000E104F10408F431C0A4E0DA9EC001112459
:106E80008558914FFC01329625913491BC2D66278F
:106E9000B39FA001B29F410D561F0694461F561F77
:106EA000112470E060E0FC0185919491B0E0A0E0D5
:106EB000841B950BA60BB70B809330019093310187
:106EC000A0933201B0933301C0903001D0903101D2
:106ED000E0903201F090330101CBD701C601B695A5
:106EE000A795979587958C7F8558954FFC0125919F
:106EF0003491FC01329645915491EC2DE770E49F5A
:106F0000C001E59F900D112463E0969587956A95E1
:106F1000E1F7281B390BC901B0E0A0E0CDCFEA8929
:106F2000FB8985889688A788B08C81E081149104BC
:106F3000A104B10409F480E0AA89BB895996CD90D7
:106F4000DD90ED90FC905C97C114D104E104F10454
:106F500009F08260EA89FB89458D568D678D70A1A5
:106F6000411551056105710509F08460809369043C
:106F700010925704109258041092590410925A0417
:106F800010926104109262041092630410926404DF
:106F9000EA89FB8985A196A1A7A1B0A580936A047F
:106FA00090936B04A0936C04B0936D044424552417
:106FB0003201481A590A6A0A7B0A409247045092E1
:106FC00048046092490470924A0440924B045092E3
:106FD0004C0460924D0470924E0440924F045092C3
:106FE0005004609251047092520441A052A063A0D8
:106FF00074A0440C551C661C771C880C991CAA1C98
:10700000BB1C8092370490923804A0923904B0924D
:107010003A04CC0CDD1CEE1CFF1CC0923B04D09249
:107020003C04E0923D04F0923E04440F551F661F5D
:10703000771F40933F045093400460934104709342
:10704000420440924304509244046092450470927A
:107050004604880F991FAA1FBB1F80933304909387
:107060003404A0933504B093360410926E04109249
:107070006F04109270041092710481A592A5A3A5CB
:10708000B4A58093650490936604A0936704B093BD
:10709000680485A596A5A7A5B0A980935C049093E4
:1070A0005D04A0935E04B0935F04EB5BFF4F8081AF
:1070B0009091E106891721F08093E1060E94842BCC
:1070C0000E94852F44244A94542C3201409230016E
:1070D000509231016092320170923301EA89FB894A
:1070E000FD96E080F18002811381AA89BB89D19647
:1070F0002D913D914D915C91D4976D01BAE4CB0EE9
:10710000D11CF60160817181828193810E94C01936
:1071100010925B04D6014D915D916D917C918BE74E
:1071200092E1A1E0FC01059115912591349104179C
:1071300015072607370758F47695679557954795AD
:10714000AA0F0496E7E9F2E1E817F90759F7A093C7
:107150006004403251056105710520F440E250E0C1
:1071600060E070E040525109610971094115F8E091
:107170005F076105710508F462C024E0529FC001F9
:1071800011248558914FFC01329625913491AA27FC
:10719000439FF001429FE10DFA1F0694EA1FFA1F78
:1071A0001124AF0170E060E0FC01C590D490F12C97
:1071B000E12CC41AD50AE60AF70AC0927204D092EA
:1071C0007304E0927404F0927504809172049091BB
:1071D0007304A0917404B0917504AC01BD010097D3
:1071E00031E0A307B10520F04FEF5FEF60E070E002
:1071F000841B950BA60BB70B8093720490937304BA
:10720000A0937404B0937504F894809184009091D5
:1072100085004096A981A150A983AA2381F1240E5B
:10722000351E2816390610F40C9458303092890017
:107230002092880078946396E2E10C9425F0DB01BB
:10724000CA01B695A795979587958C7F8558954FD8
:10725000FC01C590D490FC01329625913491477081
:10726000429FC001439F900D112433E0969587956E
:107270003A95E1F7C81AD90AF12CE12C9ECF1C01EE
:10728000D5CF80EDC82E87E0D82EE12CF12C2DC96A
:10729000CF93DF9380915F1390916013891B80954A
:1072A0008F7019F40E943C8EF5CF80915F138F5F31
:1072B0008F70A0915F139BE5A99FD0011124FD0160
:1072C000E854F84FEF0119929A95E9F798E0908306
:1072D000A353B84F90E1E1E6F3E101900D929A9546
:1072E000E1F720915F1390916013291303C094E696
:1072F00090935C1380935F130E94632FDF91CF9173
:107300000895FC0120813181428153816091890D72
:1073100070918A0D80918B0D90918C0D0E9488E95F
:107320000E94A9F160936D1370936E1380936F1395
:107330009093701390915F1380916013981709F0E8
:10734000A7CF0E94822C0E94562F40916D1350911E
:107350006E1360916F13709170134093910450936A
:107360009204609393047093940481110C94632F9E
:1073700008954F925F926F927F928F929F92AF92F9
:10738000BF92CF92DF92EF92FF92CF93DF93EC0107
:107390002091890D30918A0D40918B0D50918C0D6B
:1073A0006C857D858E859F850E9488E90E94A9F164
:1073B0006B017C012091850D3091860D4091870DE8
:1073C0005091880D688579858A859B850E9488E91A
:1073D0000E94A9F14B015C012091810D3091820D39
:1073E0004091830D5091840D6C817D818E819F81B0
:1073F0000E9488E90E94A9F12B013C0120917D0D9A
:1074000030917E0D40917F0D5091800D6881798182
:107410008A819B810E9488E90E94A9F1609361138F
:107420007093621380936313909364134092651377
:10743000509266136092671370926813809269137A
:1074400090926A13A0926B13B0926C13C0926D135A
:10745000D0926E13E0926F13F092701390915F13BD
:1074600080916013981781F013DFDF91CF91FF9027
:10747000EF90DF90CF90BF90AF909F908F907F90D4
:107480006F905F904F9008950E94822C0E94562F1B
:10749000C82F81E693E10E94B719CC2331F30E94F3
:1074A000632FE3CFCF92DF92EF92FF92CF93DF93E0
:1074B000C82F0E94562F94E0C99FE0011124FE01BD
:1074C000EB57FB4FC080D180E280F38081110E9496
:1074D000632FC855D84FC701B6010E9429E92881FA
:1074E00039814A815B810E9488E9DF91CF91FF90C9
:1074F000EF90DF90CF9008958F929F92AF92BF92BE
:10750000CF92DF92EF92FF921F93CF93DF93CDB78D
:10751000DEB760970FB6F894DEBF0FBECDBF182F51
:1075200080E0C0DF4B015C0180920B0490920C0460
:10753000A0920D04B0920E0481E0B4DF6B017C01D7
:10754000C0920F04D0921004E0921104F092120441
:1075500082E0A8DF609313047093140480931504F1
:10756000909316041D861E861F86188A89829A8229
:10757000AB82BC82CD82DE82EF82F88669877A8711
:107580008B879C8783E08EDF6D877E878F87988BC4
:10759000CE0101960E94A42C1E3FD9F480E1FE0189
:1075A0003196A5E7B1E001900D928A95E1F76096DA
:1075B0000FB6F894DEBF0FBECDBFDF91CF911F9104
:1075C000FF90EF90DF90CF90BF90AF909F908F9003
:1075D000089584E0189FF0011124DF01AB58BE4FDD
:1075E00081E090E08C0F9D1FE80FF91F40815181D1
:1075F000628173814D935D936D937C931397D7CF85
:10760000CF92DF92EF92FF92CF93DF93C82F0E9429
:10761000562F94E0C99FE0011124FE01E758FB4F6B
:10762000C080D180E280F38081110E94632FC85511
:10763000D84FC701B6010E9429E9288139814A81C2
:107640005B810E9488E9DF91CF91FF90EF90DF90FE
:10765000CF900895A1E0B0E0E0E3FBE30C9419F0D3
:10766000898360E0CE0101960E94121B61E0CE0189
:1076700001960E94121B62E0CE0101960E94121B2D
:1076800089812196E2E00C9435F0A2E1B0E0EBE4D0
:10769000FBE30C9415F0DEDF8823C1F1EDB6FEB6F6
:1076A00041E952E082FF02C048E852E021E932E0BD
:1076B00081FF02C02AE832E080FD25C081E992E026
:1076C0005F934F933F932F939F938F938CE097E01B
:1076D0009F938F938E010F5F1F4F1F930F930E94F5
:1076E000BCE80E94AE89C8010E942F83C8010E9495
:1076F0003CC40FB6F894DEBF0FBECDBF81E06296EA
:10770000E6E00C9431F08CE892E0DACF80E0F7CF3D
:10771000A0E2B0E0EEE8FBE30C9409F080911401E4
:10772000882309F4BEC080911D04082F10E080FF5B
:107730003CC0C0901601D0901701E0901801F09065
:1077400019012091A0023091A1024091A202509112
:10775000A302C701B6010E94A4F1181644F4C09216
:10776000A002D092A102E092A202F092A302C090E5
:107770002201D0902301E0902401F0902501209176
:10778000A0023091A1024091A2025091A302C70130
:10779000B6010E9423E987FF08C0C092A002D092E0
:1077A000A102E092A202F092A30201FF3CC0C090AD
:1077B0001A01D0901B01E0901C01F0901D01209156
:1077C000A4023091A5024091A6025091A702C701E0
:1077D000B6010E94A4F1181644F4C092A402D092FB
:1077E000A502E092A602F092A702C0902601D090D6
:1077F0002701E0902801F09029012091A402309106
:10780000A5024091A6025091A702C701B6010E94AD
:1078100023E987FF08C0C092A402D092A502E0929B
:10782000A602F092A70202FF3CC0C0901E01D090B9
:107830001F01E0902001F09021012091A8023091D9
:10784000A9024091AA025091AB02C701B6010E9461
:10785000A4F1181644F4C092A802D092A902E092B2
:10786000AA02F092AB02C0902A01D0902B01E090C6
:107870002C01F0902D012091A8023091A902409195
:10788000AA025091AB02C701B6010E9423E987FF0B
:1078900008C0C092A802D092A902E092AA02F09277
:1078A000AB028091680D83FD61C020918101309110
:1078B000820140918301509184016091AC027091EA
:1078C000AD028091AE029091AF020E9423E988231D
:1078D00009F44CC00E948FB5182F882331F00E9404
:1078E000AE8981EF96E00E943E8320918101309124
:1078F000820140918301509184016091AC027091AA
:10790000AD028091AE029091AF020E9440F09F774D
:1079100020916F013091700140917101509172017D
:107920000E9488E920E030E046E154E40E94A4F19E
:107930001816D4F40E94AE8982ED96E00E943E8330
:107940008091AC029091AD02A091AE02B091AF02D5
:107950008093810190938201A0938301B09384016D
:107960008CEA92E0CEDC02C01111EACF2AE037EDBA
:1079700043E25CE360910E0170910F018091100170
:10798000909111010E9488E96B017C0160911201C4
:1079900070911301072E000C880B990B0E9429E9A6
:1079A0009B01AC01C701B6010E9488E9698B7A8B03
:1079B0008B8B9C8B8091B002882309F18090B1025F
:1079C0009090B202A090B302B090B402C090A8020E
:1079D000D090A902E090AA02F090AB0220E030E043
:1079E000A901C501B4010E9423E98823F9F0A70188
:1079F0009601C501B4010E94A4F11816BCF020E064
:107A000030E0A901BE016F5E7F4F80EA92E00E94E4
:107A1000B0C580E1E0EAF2E0A5E7B1E001900D92A7
:107A20008A95E1F7A096E2E10C9425F0209175018A
:107A30003091760140917701509178016091A002D8
:107A40007091A1028091A2029091A3020E9440F045
:107A50004B015C012091790130917A0140917B01C9
:107A600050917C016091A4027091A5028091A602C0
:107A70009091A7020E9440F06D8B7E8B8F8B988F28
:107A800020917D0130917E0140917F0150918001D4
:107A9000C701B6010E9440F06D8F7E8F8F8F98A333
:107AA00020918101309182014091830150918401A4
:107AB0006091AC027091AD028091AE029091AF02E4
:107AC0000E9440F0698F7A8F8B8F9C8F20E030E08E
:107AD000A901C501B4010E9423E981110CC020E075
:107AE00030E0A9016D897E898F89988D0E9423E9F4
:107AF000882309F484CFA5019401C501B4010E9433
:107B000088E96B017C012D893E894F89588DCA0116
:107B1000B9010E9488E99B01AC01C701B6010E942E
:107B200041F06B017C012D8D3E8D4F8D58A1CA0116
:107B3000B9010E9488E99B01AC01C701B6010E940E
:107B400041F06B017C01298D3A8D4B8D5C8DCA0112
:107B5000B9010E9488E99B01AC01C701B6010E94EE
:107B600041F06B017C010E94DDF12B013C012CEC0A
:107B70003CEB4CE85BE2C701B6010E9423E987FFBA
:107B800006C0498C5A8C6B8C7C8CE89477F82DEB72
:107B900037E346E855E3C301B2010E9423E987FDBC
:107BA00038CF2DEC3CEC4CE45EE3C301B2010E9403
:107BB00088E90E9425F11B01672B19F422242394E4
:107BC000312CB10190E080E00E9427E99B01AC01DB
:107BD00060E070E080E89FE30E94B8F06B017C01F8
:107BE000AC019B01C301B2010E9488E92B013C0159
:107BF000A7019601C501B4010E9488E94B015C010F
:107C0000A70196016D897E898F89988D0E9488E9E8
:107C10006D8B7E8B8F8B988FA70196016D8D7E8DDE
:107C20008F8D98A10E9488E96D8F7E8F8F8F98A38A
:107C3000A7019601698D7A8D8B8D9C8D0E9488E9B4
:107C4000698F7A8F8B8F9C8F80E1E5E7F1E08E0161
:107C50000F5F1F4FD80101900D928A95E1F70E94A6
:107C6000D9CF6B017C0128ECC20ED11CE11CF11CA8
:107C700081E0281A310809F454C00E94D9CF9B0131
:107C8000AC012C193D094E095F0957FD4DC06B0130
:107C90007C0128ECC20ED11CE11CF11C80E00E948A
:107CA0003C8EA501940169817A818B819C810E941F
:107CB00041F069837A838B839C832D893E894F8928
:107CC000588D6D817E818F8198850E9441F06D83F2
:107CD0007E838F8398872D8D3E8D4F8D58A169852A
:107CE0007A858B859C850E9441F069877A878B878E
:107CF0009C87298D3A8D4B8D5C8D6D857E858F851A
:107D000098890E9441F06D877E878F87988BA301A9
:107D10009201BE016F5E7F4FC8010E94B0C5811104
:107D2000A7CFA30192016ECE0E94C429BACF809141
:107D3000190490911A04A0911B04B0911C04809323
:107D40000E0190930F01A0931001B0931101809147
:107D500017049091180490931301809312010895D1
:107D600080910E0190910F01A0911001B09111012D
:107D70008093190490931A04A0931B04B0931C04DD
:107D8000809112019091130190931804809317042D
:107D900084E690E090931301809312010895ACE083
:107DA000B0E0E5EDFEE30C940BF02B013C012987DC
:107DB0003A874B875C8747015801D601CD90DD900B
:107DC000ED90FC9020E030E0A901C701B6010E94CF
:107DD00023E9811171C080916B0190916C01A09198
:107DE0006D01B0916E0189839A83AB83BC8320E0DF
:107DF00030E0A901C701B6010E9423E9811106C044
:107E0000C12CD12C80E8E82E80E4F82ECD82DE82D1
:107E1000EF82F886A501940160917D0170917E0149
:107E200080917F01909180010E9423E987FF0CC01F
:107E300080927D0190927E01A0927F01B09280019C
:107E4000CE0105960E948E224092750150927601D5
:107E5000609277017092780189859A85AB85BC859F
:107E60008093790190937A01A0937B01B0937C0178
:107E7000CE0101960E948E22A501940160917D01A0
:107E800070917E0180917F01909180010E94A4F108
:107E9000181664F480927D0190927E01A0927F0179
:107EA000B0928001CE0105960E948E220E94822C03
:107EB0002C96E0E10C9427F0D701C60194CFCF9225
:107EC000DF92EF92FF920F931F936B01FC01E08012
:107ED000F18002811381E5E7F1E02481358146815B
:107EE0005781608171818281938159DF1F910F9148
:107EF000FF90EF90DF90CF9008950C94D3C50F932F
:107F00001F93CF93DF93EC018B010E94068D882392
:107F100031F081E0DF91CF911F910F910895B80169
:107F2000CE01CDDF80912607C82FC47082FD0AC024
:107F30001092260782E0E0DAE0DF81E0CC2351F303
:107F400080E0E8CF0E94C58C882391F3E2CFCF93E5
:107F50000E94562FC82F8091601380935F138093E7
:107F60005E1380935D1384E680935C130E94E72F79
:107F700080ED93E09093B20D8093B10DC1110E94FA
:107F8000632F81E0809378040E94822C8EEFB4DA14
:107F9000B4DFCF910895ACE0B0E0E1EDFFE30C94E5
:107FA00019F00E944EB50E94562F9CE0E5E8F4E0DF
:107FB000DE01119601900D929A95E1F781110E94D0
:107FC000632FCE0101960E94FC2A2C96E2E00C94CD
:107FD00035F0B0E0A0E0EFEEFFE30C940BF0409042
:107FE00075015090760160907701709078018090D3
:107FF000790190907A01A0907B01B0907C01C090B3
:108000007D01D0907E01E0907F01F09080010E9480
:10801000162C60912E0170912F01072E000C880BF9
:10802000990B0E9429E92AE037ED43E25CE30E94C4
:1080300088E960936F017093700180937101909350
:10804000720106E111E0D0E0C0E0CE01815D954F04
:108050000E946176F80161937193819391938F01EE
:10806000CE018D5D954F0E946176F8016087718722
:10807000828793872496CC30D10539F760E08BE274
:1080800094E00E9442790E940F7A0E945A2CA30128
:1080900092016091750170917601809177019091C4
:1080A00078010E9423E981111BC0A5019401609110
:1080B000790170917A0180917B0190917C010E94FD
:1080C00023E981110DC020917D0130917E01409105
:1080D0007F0150918001C701B6010E9423E98111FF
:1080E0005ADFCDB7DEB7E0E10C9427F0A4E0B0E0B2
:1080F000ECE7F0E40C9419F084EF91E0A0E0B0E03C
:1081000089839A83AB83BC83BE016F5F7F4F8CE30F
:108110000E94E58188EB96E00E943E8386B162EB87
:1081200076E082FB882780F90E94E82186B16CEA1C
:1081300076E083FB882780F90E94E82186B166EA11
:1081400076E0829581700E94E821349907C00E94F0
:1081500019822496E2E00C9435F006C00E94028257
:108160002496E2E00C9435F08091E006811103C082
:108170008091E20681110C94852F0895ACE0B0E067
:10818000E4ECF0E40C9419F0A9E6BDE090E080E0A6
:10819000FC01E559F54F45915591659174914D93C9
:1081A0005D936D937D93FC01E55AF54F4591559193
:1081B0006591749150964D935D936D937C93539715
:1081C000FC01E55BF54F4591559165917491909651
:1081D0004D935D936D937C939397049680319105B5
:1081E000B9F680E29EE4A0E0B0E08093790D909330
:1081F0007A0DA0937B0DB0937C0D80E090E0AAEF08
:10820000B3E480939D0D90939E0DA0939F0DB0932A
:10821000A00D8093A10D9093A20DA093A30DB093F8
:10822000A40D8093A50D9093A60DA093A70DB093D8
:10823000A80D1092A90D1092AA0D1092AB0D1092DC
:10824000AC0D1092AD0D1092AE0D1092AF0D1092BC
:10825000B00D8AE097EDA3EABDE380938B0790937E
:108260008C07A0938D07B0938E0780E090E0A0E28A
:10827000B1E480932B0490932C04A0932D04B0932D
:108280002E040E94F8788CE0E5E8F1E0DE0111961A
:1082900001900D928A95E1F789819A81AB81BC8129
:1082A00080934E1390934F13A0935013B093511398
:1082B0008D819E81AF81B885809352139093531323
:1082C000A0935413B093551389859A85AB85BC85CB
:1082D0008093561390935713A0935813B093591348
:1082E0008EEB90E090934407809343078CE390E0FB
:1082F00090934607809345071092480710924707CE
:1083000086EE90E090934A078093490786E490E0D8
:1083100090934C0780934B0710924E0710924D0795
:108320008FE892ECADE8B1E48093B5129093B61269
:10833000A093B712B093B8128CE998EFA5E4BEE30E
:108340008093B9129093BA12A093BB12B093BC124F
:1083500081E49CEBABECB3E48093BD129093BE122E
:10836000A093BF12B093C01280E090E0AFEAB3E4F4
:108370008093370790933807A0933907B0933A0753
:1083800085E996E2A5E2B1E480933B0790933C0730
:10839000A0933D07B0933E0780EA9CE6ACE2B5E4CB
:1083A00080933F0790934007A0934107B093420703
:1083B0001092E0061092DF06D7DE0BDE2C96E2E08C
:1083C0000C9435F0DBCEA4E0B0E0E9EEF1E40C94DF
:1083D0000AF09091E206981709F455C0382E80E013
:1083E00090E0A0E2B1E489839A83AB83BC83C09020
:1083F0005613D0905713E0905813F090591320E083
:1084000030E0A901C701B6010E9423E987FF0CC033
:10841000A701960160E070E080E291E40E9440F0E4
:1084200069837A838B839C83CE0101960E9464C604
:1084300040907501509076016090770170907801BE
:108440008090790190907A01A0907B01B0907C019E
:108450003320F1F00E94068D19821A821B821C8241
:10846000E0907D01F0907E0100917F0110918001EC
:10847000CE0101966C01A5019401C301B2018FDC0C
:108480003092E20671DE80E02496E1E10C9426F061
:108490000E94C58CE1CFB0E0A0E0E1E5F2E40C94ED
:1084A0000BF0C82FE82EF12CF701EC57F24DD491C8
:1084B000823071F481E087DF811105C00E94068D52
:1084C000882309F4E2C0CDB7DEB7E0E10C9427F0D1
:1084D0006D2FDD0F770B880B990B0E9429E92B017B
:1084E0003C01C701880F991F880F991F855A984F23
:1084F0000E9461764B015C01A3019201C501B401A8
:108500000E9488E94B015C016701CC0CDD1CCC0C9E
:10851000DD1CC601815B984F0E946176A301920128
:108520000E9488E920E030E040EC5FE30E9488E9A7
:10853000AB01BC0100E010E098018C2F0E949AC9A9
:10854000C23009F0CCC00E94C58C20E030E0A90107
:10855000C501B4010E9423E9882329F100E010E05D
:1085600020E830E4B501A40170588C2F0E949AC90C
:10857000C23009F467C0A5019401C501B4010E948D
:1085800041F04B015C01C23009F062C000E010E034
:1085900020E030E4B501A4018C2F0E949AC9C230BA
:1085A00011F40E94C58C81E090E00C2E01C0880F70
:1085B0000A94EAF790917707982B90937707909118
:1085C0001D04892B80931D04C6018D5B984F0E946A
:1085D0006176F601EB58FE4F60837183828393834B
:1085E000C230D1F420915613309157134091581353
:1085F0005091591360917D0170917E0180917F01AE
:10860000909180010E9440F060937D0170937E0103
:1086100080937F019093800170DCF601E056FD4F5E
:10862000D601AB58BE4F8D919D910D90BC91A02D60
:1086300080839183A283B383C23009F044CF80E06A
:10864000C2DE41CF0E94068D882309F494CF3BCF30
:10865000F701E05CF84F6491611107C00E94AE8998
:108660008EE197E00E943E836AE070E090E080E057
:108670000E9427E99B01AC0161E070E088E492E48C
:108680000E94B8F08B019C0185CF83E697E00E94A1
:10869000617620E030E0A9010E9423E9882309F4F3
:1086A00017CF6D2FDD0F770B880B990B0E9429E9EF
:1086B0002B013C0183E697E00E9461764B015C014F
:1086C00020E030E040EA50E40E94A4F187FF14CF9C
:1086D000812C912C90EAA92E90E4B92E0DCF20E0A8
:1086E00030E0A901C501B4010E9423E9882309F4FF
:1086F0005ACF00E010E0980135CF809126078823FB
:1087000019F010922607089540E070E060E086E8D6
:1087100096E00E944D8D1F920F920FB60F9211247A
:108720000BB60F922F933F934F935F936F937F936B
:108730008F939F93AF93BF93EF93FF930E94852FE7
:10874000FF91EF91BF91AF919F918F917F916F9129
:108750005F914F913F912F910F900BBE0F900FBEE5
:108760000F901F9018950F931F938091870781306A
:1087700019F50E94D9CF00910204109103042091B1
:10878000040430910504601B710B820B930B28EEDF
:1087900033E040E050E00E9451EF6091FE037091A1
:1087A000FF038091000490910104620F731F841FE6
:1087B000951F1F910F910895609106047091070411
:1087C0008091080490910904D6CF109287071092E7
:1087D00002041092030410920404109205041092F3
:1087E00006041092070410920804109209041092D3
:1087F000FE031092FF0310920004109201040895EA
:10880000809187078130E1F08230C1F4ACDF609362
:10881000FE037093FF03809300049093010481E0B2
:10882000809387070E94D9CF60930204709303045A
:10883000809304049093050481E00895C6DFEFCF90
:1088400080E008950E94B2C60E94A97A882351F060
:108850008091C91482FD06C087EE91E09093E506F1
:108860008093E406CDCF80918707813079F482E050
:10887000809387070E94D9CF609306047093070402
:10888000809308049093090481E0089580E008959E
:10889000809187078150823070F4109287070E9480
:1088A000D9CF6093060470930704809308049093D3
:1088B000090481E0089580E008952091B21230917A
:1088C000B312263531053CF4209134073091350739
:1088D000263031051CF0882331F092CF662319F041
:1088E000D7DF0C94B2C608959C0197FF26C0EE27EF
:1088F000FF27E81BF90B2D398FEF38070CF05DC00F
:108900008DE280939B02CF0164E670E00E94DBEF72
:10891000CB012AE030E0B9010E94DBEF805D80935B
:108920009C02CF01B9010E94DBEFCB01B9010E948B
:10893000DBEF805D80939D022AC0283E83E03807EC
:10894000B4F1C90168EE73E00E94DBEFCB01EAE00D
:10895000F0E0BF010E94DBEF805D80939B02C901C4
:1089600064E670E00E94DBEFCB01BF010E94DBEF09
:10897000805D80939C02C901BF010E94DBEFCB01A7
:10898000BF010E94DBEF805D80939D02F901CF0162
:108990006AE070E00E94DBEF805D80939E028BE9CD
:1089A00092E008958DE237FDC5CF80E2C3CFF90193
:1089B00080E2243631050CF0A4CF80E280939B0244
:1089C00080939C02EA30F1056CF38DE237FF80E280
:1089D00080939C02CF016AE070E00E94DBEF605D53
:1089E00060939D02D4CF9C0197FD2DC080E2243678
:1089F00031055CF0C90164E670E00E94DBEFCB0159
:108A00006AE070E00E94DBEF805D80939C0280E270
:108A10002A3031055CF0EAE0F0E0C901BF010E94B4
:108A2000DBEFCB01BF010E94DBEF805D80939D02F5
:108A3000C9016AE070E00E94DBEF805D80939E02D6
:108A40008CE992E008953195219531098DE2DDCFD1
:108A5000CF92DF92EF92FF92FC01C080D180E28042
:108A6000F38020E030E0A901C701B6010E9423E9AC
:108A700087FD26C06DEB77E386E095E3A7019601BD
:108A80000E9441F06B017C0120E030E0A9010E94CE
:108A900023E920E030E040E05FE387FF04C020E00E
:108AA00030E040E05FEBC701B6010E9441F00E9458
:108AB00020F1CB0198DFFF90EF90DF90CF900895E9
:108AC0006DEB77E386E095EBD9CFA4E0B0E0EBE681
:108AD000F5E40C9419F00E9429E969837A838B8369
:108AE0009C83CE010196B4DF2496E2E00C9435F02D
:108AF000FC0160817181828193810E9420F1CB0110
:108B000072CFA4E0B0E0E7E8F5E40C9419F00E941D
:108B100029E969837A838B839C83CE010196E8DF00
:108B20002496E2E00C9435F08F929F92AF92BF9220
:108B3000EF92FF920F931F93CF93DF93EC018B0182
:108B4000E42EF22E80917113909172138C179D0771
:108B5000C9F122E6C137D20709F03FC0875B9A47C7
:108B600071F40E94D9CF6E517B4F8F4F9F4F60930E
:108B7000EC037093ED038093EE039093EF03D09397
:108B80007213C093711330E020E000936A071093D2
:108B90006B0720936C0730936D07E0926507F092A6
:108BA0006607C75BDA4721F41092FD031092EB03CE
:108BB00082E080936A0181E0809367071092FA0354
:108BC0001092F703DF91CF911F910F91FF90EF90DB
:108BD000BF90AF909F908F9008952AE7C73BD20730
:108BE00071F681579246D9F40E94D9CF8090EC0358
:108BF0009090ED03A090EE03B090EF03681979090F
:108C00008A099B0997FF0BC080917707877087308F
:108C100031F40E946523C3E4D7E58111B0CFC7EBDF
:108C2000DAE7ADCF20E040E070E060E084E593E279
:108C30007BCF0E948FB5882339F020E040E070E0C0
:108C400060E085E696E570CFEDCF21E02093FD034F
:108C5000FC0180819181A281B38180930A0190936C
:108C60000B01A0930C01B0930D0120E040E070E0F7
:108C700060E0809154079091550756CFA4E0B0E092
:108C8000E4E4F6E40C9419F08DEC9CECACECBCE361
:108C900089839A83AB83BC83CE010196D6DF249669
:108CA000E2E00C9435F0A4E0B0E0E9E5F6E40C94E1
:108CB00019F08DEC9CECACECBDE389839A83AB831B
:108CC000BC83CE010196C1DF2496E2E00C9435F01E
:108CD000A4E0B0E0EEE6F6E40C9419F080E090E059
:108CE000A0E8BFE389839A83AB83BC83CE0101965E
:108CF000ACDF2496E2E00C9435F0A4E0B0E0E3E8C9
:108D0000F6E40C9419F080E090E0A0E2B1E48983ED
:108D10009A83AB83BC83CE01019697DF2496E2E071
:108D20000C9435F081E08093FD0380917707877084
:108D3000873051F01092770710921D0480EF95E074
:108D40009093E5068093E4068091B0028093F90346
:108D500080E00E94B67820E040E070E060E082EBC6
:108D600096E4E2CE80916A01882331F041E062EA24
:108D700073E082E00E9447CA80911D0487708730AB
:108D800071F41092F80320E040E070E060E085EEBE
:108D900096E5CADE81E08093F7030C94962208954D
:108DA00020E040E070E060E087EB9AE7BDCE1092F3
:108DB000A7070E94E427F4CFB0E0A0E0E2EEF6E4DB
:108DC0000C9413F0CDB6DEB6EAE7F7E0DF010D90C4
:108DD0000020E9F7CD01825797402DB73EB7281BF9
:108DE000390B0FB6F8943EBF0FBE2DBF0DB71EB79F
:108DF0000F5F1F4FFF93EF9383E595E09F938F9352
:108E00001F930F930E94BCE8780134E0E30EF11C3D
:108E10000F900F900F900F900F900F90D7018D91A2
:108E20007D01882349F0082E000C990B0E9422F244
:108E3000F70131978083F2CF6EE475E0C8010E949C
:108E400055E84FE350E0B80186EE96E00E947AF2D2
:108E50000FB6F894DEBE0FBECDBEA2DF0E94B2C632
:108E6000E8E00C942FF08093280720E040E070E0C9
:108E700060E083E097E558CEA2E8B0E0E2E4F7E4F2
:108E80000C9409F0ADB6BEB684E690E090939E12C5
:108E900080939D121092C2121092C11241E064E0C0
:108EA00070E0CE0187589F4F0E9496B443E050E097
:108EB000BE0167587F4F86E392E00E946CF2892BD7
:108EC000F9F0ED968FADED97882339F08FE3EA96B0
:108ED0008FAFEA97EB961FAEEB9782E0C4DF81E09D
:108EE00080932A0490912A0481E089270FB6F89490
:108EF000BEBE0FBEADBECE57DF4FE2E10C9425F0F3
:108F000041E062E070E0CE0183589F4F0E9496B42A
:108F1000E9961CAE1DAE1EAE1FAEE9971092C212AE
:108F20001092C112CE018F579F4F0E946422EDB65E
:108F3000FEB6CF57DF4FC880C158D040D12C23E0B8
:108F4000C20ED11CCC0CDD1CCC0CDD1C8DB79EB729
:108F50008C199D090FB6F8949EBF0FBE8DBFEDB75B
:108F6000FEB731963F018C199D090FB6F8949EBF4C
:108F70000FBE8DBFEDB7FEB731964F018C199D091D
:108F80000FB6F8949EBF0FBE8DBF0DB71EB70F5F13
:108F90001F4FB601C3010E9469224091890381E0FD
:108FA000482764E070E089E79DE00E9496B4B6012E
:108FB000C4010E946922B601C8010E9469229091F1
:108FC0008903CE57DF4F9883C258D04091114BC0D0
:108FD000CF57DF4F8881C158D04090E00296A9E674
:108FE000BDE050E040E030E020E067E77AE0E7E60F
:108FF000CE2EEAE0DE2E821793070CF495C0F30123
:10900000E40FF51F20803180428053802D923D92E5
:109010004D925D92821793070CF48CC0F401E40F1B
:10902000F51F208031804280538050962D923D92D2
:109030004D925C925397821793070CF481C0F8010C
:10904000E40FF51F208031804280538090962D924E
:109050003D924D925C9293972F5F3F4F4C5F5F4FD5
:109060002430310541F68DE99DE00E943C2281EAE1
:109070009DE00E943C2285EA9DE00E943C2289EA14
:109080009DE00E943C228DEA9DE00E943C22CE01A0
:109090008B589F4F0E943C22CE018B589F4F0E94BD
:1090A0003C22CE018B589F4F0E943C22CE018B5810
:1090B0009F4F0E943C228BE897E00E943C220FB613
:1090C000F894FEBE0FBEEDBE8E010F5F1F4FC801AC
:1090D0000E945C22CE0183599F4F0E944422C80106
:1090E0000E943C228BE294E00E943C22CE018B58ED
:1090F0009F4F0E943C22CE0183599F4F0E946422C1
:10910000C8010E946422AE96CFACAE978981C89EFA
:1091100060011124E1E0CE1AD108C8F0CE018B58CD
:109120009F4F0E943C22F6CFFB0125903590459041
:1091300054906CCFF601259035904590549075CFA2
:10914000E7E5FAE025903590459054907FCF8EE486
:1091500093E10E945C228AE0D82EDA94CE01DD20D1
:1091600029F08B589F4F0E943C22F7CF80589F4F89
:109170000E946422CE0181589F4F0E946422C058F1
:10918000DF4F8881C058D040873009F05EC1C15898
:10919000DF4F8881CF57D040873009F056C1CE5776
:1091A000DF4F2881C258D040211103C080E00E94C7
:1091B000B67881E893E00E94542289E793E00E9408
:1091C00054224091890381E0482764EC70E085EBEC
:1091D00092E00E9496B4C8010E944C22CE018359AD
:1091E0009F4F0E94442240918903FF24F3944F250E
:1091F00064E070E0C8010E9496B483EE96E00E949D
:109200004C22409189034F256CE070E083E497E0A5
:109210000E9496B4409189034F2564E170E0C80133
:109220000E9496B4F0908903F11030C089819A8130
:10923000AB81BC818093B5129093B612A093B71204
:10924000B093B8122CEA35EC47E25EE36D817E8183
:109250008F8198850E9488E96093B9127093BA1241
:109260008093BB129093BC1220E030E543EC50E4B5
:1092700069857A858B859C850E9488E96093BD12FB
:109280007093BE128093BF129093C01241E04F259D
:1092900062E070E0C8010E9496B4C8010E943422C6
:1092A000D0908903D11030C089819A81AB81BC8173
:1092B0008093370790933807A0933907B0933A0704
:1092C0002CEA35EC47E25EE36D817E818F819885E3
:1092D0000E9488E960933B0770933C0780933D07A9
:1092E00090933E0720E030E543EC50E469857A85B1
:1092F0008B859C850E9488E960933F0770934007A7
:109300008093410790934207C8010E943422C8010C
:109310000E944422C8010E944422C8010E944422A3
:1093200085E0F80111928A95E9F7FF24F3944D2D19
:109330004F2565E070E0C8010E9496B4C8010E9404
:109340004C22409189034F2560E270E0C8010E94E1
:1093500096B4CE0183599F4F0E944C2240918903BD
:109360004F2569E070E0C8010E9496B440918903DE
:109370004F2562E170E0C8010E9496B440918903D4
:109380004F2564E270E0C8010E9496B440918903C1
:109390004F2560E170E0C8010E9496B440918903B6
:1093A0004F2569E070E0C8010E9496B4C8010E9490
:1093B0003C22409189034F256CE070E0C8010E9477
:1093C00096B4409189034F256CE670E0C8010E9475
:1093D00096B419821A821B821C821D821E821F82F1
:1093E000188619861A861B861C86C8010E9434229C
:1093F000409189034F2568E070E0C8010E9496B44F
:10940000C8010E945C22CE0181589F4F0E944422D5
:10941000CE0183599F4F0E943C2280919D129091D2
:109420009E128037934089F510922A042091C11230
:109430003091C212EF968EAD9FADEF972817390786
:1094400041F1F0922A0480E023C0CE0183599F4F5E
:109450000E945422C8010E945422C058DF4FC88085
:10946000C058D040C158DF4F8881CF57D040C89EE8
:109470006001112481E0C81AD10808F4ACCECE01F5
:109480008B589F4F0E943C22F5CFF0922A0481E036
:10949000EADC80918903811125CD80912A04811114
:1094A00021CD0E94E93F1ECD81E080938903E4DC59
:1094B00010928903882309F0DFCC0E94BE4080E02F
:1094C0000895F2CFCF93DF93C091EB03CC23B1F09B
:1094D000C150C093EB0389E0C89FE0011124CB5435
:1094E000DC4F6A817B812F814E81888199811CDBD1
:1094F00088858093FD03DF91CF91089551DCFBCFE8
:10950000A4E0B0E0E6E8FAE40C940CF00E945BCB37
:10951000F09065076F2C85E0782E7F0C86E0E82EB2
:10952000EF1885E0D82EDF18AA24AA94B12C84E085
:10953000C82ECF1882E0982E9F1881E0882E8F18B1
:109540005F2C5194F1105AC080916807882309F468
:1095500044C080916A01882359F081E090916807A6
:10956000911180E024E041E856E0652D0E94A7CAF1
:109570008091A7078093280724E0F212F7C0109289
:10958000740780916807843009F4DDC080916A0116
:109590008823E1F011E080916807843009F010E041
:1095A0008091280724E6829FC001112481589F4F93
:1095B000B5010E94DBEF862F0E94E51C00E09C01B4
:1095C00046E656E06C2D812F0E945F74F394F710ED
:1095D000B9CF87E0809366070DC080914F07109246
:1095E0004F07882309F4B5CF6DDF80916707882383
:1095F00009F4AFCF2496EFE00C9428F021E0F212AA
:1096000043C080916807813041F180916A018823CD
:10961000F9F011E080916807813009F010E0609165
:10962000120170911301072E000C880B990B0E94F8
:1096300029E969837A838B839C83CE01019658DA6A
:1096400000E09C014BE756E0682D812F0E945F747B
:109650008091A70780932807B9CF80914F07109278
:109660004F07882391F210E000E027EE33E04AE054
:1096700050E062E171E08BE796E00E9420CC80919F
:109680006707882311F2B6CF82E0F812D7C0809125
:109690006807823021F180916A018823C9F211E0C4
:1096A00080916807823009F010E06091B2127091E9
:1096B000B312072E000C880B990B0E9429E96983CD
:1096C0007A838B839C83CE01019612DA00E09C01A1
:1096D00044E756E0692D812F0E945F7449CF809145
:1096E0004F0710924F078823B1F20E944FCB02E33D
:1096F00012E225EF30E050E040E062EB72E184E7F7
:1097000096E00E9420CC80916707882321F272CFD7
:1097100080914F0710924F07882309F497C00E9449
:109720004FCB0DEE1BE623E730E050E040E064E372
:1097300077E080E796E00E9420CC8091670788233D
:1097400009F484C057CF80914F0710924F078823A8
:1097500009F41CCF0E944FCB86E696E00E9495CE7E
:1097600080916707882309F411CF44CF85E0F81270
:109770003DC080916807853011F180916A0188238E
:1097800009F424CF11E080916807853009F010E0DA
:1097900060912E0170912F01072E000C880B990B00
:1097A0000E9429E969837A838B839C83CE01019689
:1097B0009FD900E09C0141E656E06D2D04CF8091D9
:1097C0004F0710924F078823C1F206E01DE127EEF4
:1097D00033E04AE050E06EE271E081E696E00E94FC
:1097E00020CC80916707882341F204CF26E0F21253
:1097F000EDCE80916807863091F080916A018823D0
:1098000009F4E4CE81E090916807963009F080E099
:1098100023E042E556E06E2D0E94A7CAD7CE809184
:109820004F0710924F07882341F383E497E50E9486
:10983000B1CB80916707882301F3DCCE83E0F81277
:1098400097CE80916807833009F462CF80916A01D6
:10985000882309F4FDCE11E080916807833009F078
:1098600010E06091340770913507072E000C880BCB
:10987000990B0E9429E969837A838B839C83CE01AB
:10988000019636D963E0661900E09C0140E756E096
:1098900022CFA4E0B0E0EFE4FCE40C940AF0EE2464
:1098A000E3948091B2129091B312892B09F4E12CC8
:1098B0000E945BCBF09065074F2C95E0592E5F0C12
:1098C00088248A94912C83E0B82EBF1882E0A82EB9
:1098D000AF1881E0782E7F183F2C319486E0682EF7
:1098E0006F18F11015C080916807882309F4D7C05C
:1098F00080916A01882309F475C181E0909168071D
:10990000911180E024E04DE456E0632D0E94A7CA47
:109910008091B2129091B3129093290780932807F7
:1099200021E0F212E8C080916807813009F4C8C0D4
:1099300080916A01882309F44DC011E08091680785
:10994000813009F010E06091280770912907072EF7
:10995000000C880B990B0E9429E969837A838B8319
:109960009C83CE010196C4D800E09C0146E456E0F9
:10997000672D812F0E945F748091A707809328072D
:1099800093E0F91227C01092740780916807833022
:1099900009F4F4C080916A018823E1F011E080911C
:1099A0006807833009F010E08091280724E6829F41
:1099B000C001112481589F4FB4010E94DBEF862F14
:1099C0000E94E51C00E09C0148E356E06B2D812FCE
:1099D0000E945F74D12CC12C14E00F2D0419C09289
:1099E0002807F1121FC0F601EE0FFF1FEF5DF94FC0
:1099F000859194919093760780937507809168077D
:109A00008F1509F4CEC080916A01882359F081E056
:109A100090916807911380E023E04EE256E0602FBA
:109A20000E94A7CA812F9FEFC91AD90A15E0853075
:109A3000B1F68091340790913507892B19F4EE2007
:109A400009F4CEC026E0F21221C08091680786306A
:109A500009F4B8C080916A018823C1F087ED96E4CB
:109A60009F938F9385E296E09F938F936F9281E00F
:109A700090916807963009F080E08F930E94202330
:109A80000F900F900F900F900F900F9087E0EE24A3
:109A9000E394F394F51025CF809366070DC0809171
:109AA0004F0710924F07882309F422CF0BDD8091D6
:109AB0006707882309F41CCF2496E1E10C9426F073
:109AC00080914F0710924F07882309F431CF0E94ED
:109AD0004FCB00E313E225EF30E050E040E068E2D6
:109AE00077E086E496E00E9420CC80916707882387
:109AF00009F41ECFE1CF82E0F8123ECF80916807D3
:109B0000823019F180916A01882309F463CF11E052
:109B100080916807823009F010E0609134077091FD
:109B20003507072E000C880B990B0E9429E96983E1
:109B30007A838B839C83CE0101960E94784500E056
:109B40009C0142E456E06A2D14CF80914F07109299
:109B50004F078823B9F20E944FCB0DEE1BE623E797
:109B600030E050E040E064E377E082E496E00E9479
:109B700020CC80916707882329F29ECF80914F07E0
:109B800010924F07882309F405CF0E944FCB88E33A
:109B900096E00E9495CE80916707882309F4FACE5B
:109BA0008BCF80914F0710924F07882309F42BCF5A
:109BB0008BEF9DE40E94B1CB80916707882309F465
:109BC00022CF7ACF80914F0710924F07882309F454
:109BD00041CFEDD880916707882309F43BCF6CCF44
:109BE00086E057CF8091B2129091B31290932907DB
:109BF00080932807C1CEB0E0A0E0E1E0FEE40C9441
:109C00000BF0009128070E945BCBC091650710E024
:109C1000000F111F0F5D194F95E0592E5C0E29EFB3
:109C2000E22E25E0F22ED3E0DC1B30E4C32E33E23B
:109C3000D32E47E0A42E46E0B42E82E0782E7C1A84
:109C40005EE2852E56E0952E81E0682E6C1A4C2E31
:109C50004194C1112AC0809168078823B1F0809196
:109C60006A01882359F081E090916807911180E0A2
:109C700024E045E156E0642D0E94A7CACF5FC511DC
:109C8000E8CF84E0809366070BC080914F07109265
:109C90004F07882321F316DC809167078823F9F2A8
:109CA000CDB7DEB7E0E10C9427F0C13059F5F801EB
:109CB00085919491909376078093750780916807BA
:109CC000813081F080916A018823C1F21F929F92B6
:109CD0008F926F9281E090916807913009F474C07F
:109CE00080E072C080914F0710924F07882351F394
:109CF00080912807682F0E9424D0809167078823CD
:109D000009F3CECFC23009F042C0F8018591949199
:109D10009093760780937507809168078230D1F021
:109D200080916A01882309F4A9CFDF92CF92BF9274
:109D3000AF927F9281E090916807923009F080E0C5
:109D40008F930E9420230F900F900F900F900F90F1
:109D50000F9094CF80914F0710924F07882301F303
:109D60000E944023809167078823D1F299CF809188
:109D70004F0710924F078823C1F0609128078FEF9B
:109D80000E9424D080916707882379F089CFC3305F
:109D900009F074CFF80185919491909376078093A0
:109DA000750780916807833011F380916A018823D9
:109DB00009F464CF1F92FF92EF92DF9381E09091BC
:109DC0006807933009F08CCF8F930E9420230F9067
:109DD0000F900F900F900F9051CFB0E0A0E0E3EF05
:109DE000FEE40C9410F00E945BCBC091650785E007
:109DF000E82EEC0E95EDC92E95E0D92ED4E0DC1BB3
:109E000013E01C1B20EFA22E25E0B22E02E00C1B5B
:109E100081E0F82EFC1A9C2E9194C1112AC08091E9
:109E200068078823B1F080916A01882359F081E0A6
:109E300090916807911180E024E044EF55E0692D8E
:109E40000E94A7CACF5FEC12E8CF85E08093660737
:109E50000BC080914F0710924F07882321F332DB0C
:109E6000809167078823F9F2CDB7DEB7EBE00C9459
:109E70002CF0C13011F580916807813079F0809124
:109E80006A018823F9F281E090916807913009F026
:109E900080E023E046E45DE26F2DD2CF80914F0752
:109EA00010924F07882359F38AEC9FE40E94B1CBAC
:109EB00080916707882319F3D7CFC23009F053C0C8
:109EC00090916807923071F080916A01882309F4BB
:109ED000B9CF81E0923009F080E020E246EE55E013
:109EE000602FAECF80914F0710924F07882361F308
:109EF000B092E506A092E40680916707882321F3DB
:109F0000B3CF80916807833081F080916A01882304
:109F100009F498CF81E090916807933009F080E0D0
:109F200023E049ED55E0612F8BCF80914F071092D0
:109F30004F07882351F38DEC9FE50E94B1CB8091B0
:109F40006707882311F390CF80914F0710924F0736
:109F5000882391F0D092E506C092E40680916707CD
:109F6000882351F081CFC33061F2C43009F06ACF49
:109F700090916807943041F380916A01882309F435
:109F800061CF81E0943009F080E020E244EC55E0BC
:109F90006D2F56CFB0E0A0E0E0EDFFE40C9414F09C
:109FA0000E945BCBC091650785E0E82EEC0ED4E003
:109FB000DC1B13E01C1B02E00C1B81E0F82EFC1ADA
:109FC000DC2ED194C1112AC0809168078823B1F09A
:109FD00080916A01882359F081E09091680791117E
:109FE00080E024E04DEB55E06D2D0E94A7CACF5FC5
:109FF000EC12E8CF85E0809366070BC080914F0795
:10A0000010924F07882321F35DDA80916707882338
:10A01000F9F2CDB7DEB7E7E00C9430F0C13011F5BE
:10A0200080916807813079F080916A018823F9F284
:10A0300081E090916807913009F080E023E04CE6E0
:10A040005DE26F2DD2CF80914F0710924F0788238A
:10A0500059F38FE493E20E94B1CB80916707882384
:10A0600019F3D7CFC23009F055C08091680782300C
:10A0700081F080916A01882309F4B9CF81E0909141
:10A080006807923009F080E023E045E65DE2602F4A
:10A09000ACCF80914F0710924F07882351F38AE489
:10A0A00093E20E94B1CB80916707882311F3B1CF6F
:10A0B00080916807833081F080916A01882309F4D8
:10A0C00096CF81E090916807933009F080E023E01B
:10A0D0004EE55DE2612F89CF80914F0710924F07C7
:10A0E000882351F385E493E20E94B1CB8091670706
:10A0F000882311F38ECF80914F0710924F0788234A
:10A1000091F089E196E40E94B1CB809167078823A2
:10A1100051F07FCFC33061F2C43009F068CF809135
:10A120006807843041F380916A01882309F45FCF86
:10A1300081E090916807943009F080E023E040E5E9
:10A140005DE26D2F52CFACE0B0E0E9EAF0E50C94AF
:10A150000AF09C878B87362E80914F0710924F070D
:10A16000882339F01092FD03ADD92C96E1E10C94CF
:10A1700026F060916A0770916B0780916C0790914F
:10A180006D07611571058105910509F45CC0209189
:10A190001401222309F4AEC0209115012111AAC097
:10A1A00021E0321609F484C0E2E03E1609F491C0C1
:10A1B000C0901601D0901701E0901801F09019019D
:10A1C000409022015090230160902401709025015D
:10A1D0000E9429E920910A0130910B0140910C0164
:10A1E00050910D010E9488E96F83788789879A874B
:10A1F000F4E03F9E80011124C8018B589E4F9E833E
:10A200008D83FC0120813181428153816F8178856A
:10A2100089859A850E9441F04B015C01A30192015E
:10A22000C701B6010E9423E9811173C0F801EB5800
:10A23000FE4F80829182A282B382832D0E94E61E0D
:10A2400081E080936A0110926A0710926B07109266
:10A250006C0710926D0780916A01882309F485CFFD
:10A2600024E0329EF0011124EB58FE4FC080D180D3
:10A27000E280F380C982DA82EB82FC822DEC3CEC36
:10A280004CEC5DE360910A0170910B0180910C012F
:10A2900090910D010E94A4F187FD65C0CE01019649
:10A2A0000E94331BBC018B859C850E94F8735DCF97
:10A2B000C0901A01D0901B01E0901C01F0901D018C
:10A2C000409026015090270160902801709029014C
:10A2D0007FCFC0901E01D0901F01E0902001F09030
:10A2E000210140902A0150902B0160902C01709028
:10A2F0002D016ECF412C20E5522E23EC622E27E457
:10A30000722EC12C30E5D32E33ECE32E37ECF32E36
:10A310005FCF20E030E0A9016F81788589859A853B
:10A320000E9423E987FF0FC0A7019601C501B40170
:10A330000E9423E987FF7ACFED81FE81C082D1821E
:10A34000E282F3827ACFA3019201C501B4010E9497
:10A35000A4F118160CF06ACFED81FE814082518283
:10A36000628273826ACF20E030E44CE156E4C70198
:10A37000B6010E9488E94B015C0120E030E0A901B0
:10A38000C701B6010E9423E920E030E040EA50E432
:10A3900087FF04C020E030E040EA50ECC501B40182
:10A3A0000E9441F02DEC3CEC4CEC5DE30E9488E90E
:10A3B0000E9420F16B017C01F7FC64C020EA36E8C2
:10A3C00041E050E00E9473EFCA01B9012AE030E099
:10A3D00040E050E00E9473EF605D60939802C70117
:10A3E000B60120E137E240E050E00E9473EF8AE0DE
:10A3F000882E912CA12CB12CCA01B901A501940180
:10A400000E9473EF605D60939902C701B60128EE68
:10A4100033E040E050E00E9473EFCA01B901A501AA
:10A4200094010E9473EF605D60939A028EE28093C4
:10A430009B02C701B60124E630E040E050E00E94F4
:10A4400073EFCA01B901A50194010E9473EF605D29
:10A4500060939C02C701B601A50194010E9473EFAD
:10A460006B017C01CA01B901A50194010E9473EF3F
:10A47000605D60939D0280E3C80EC0929E0288E9F1
:10A4800092E010CFF094E094D094C094C11CD11C01
:10A49000E11CF11C6DE2A1CF62E08EE59DE253CE9E
:10A4A00061E085E69DE24FCE60E08CE69DE24BCE1A
:10A4B000A4E0B0E0EEE5F2E50C9419F080914F07CE
:10A4C00010924F07882341F01092FD030E94624AC8
:10A4D0002496E2E00C9435F060916A0770916B0766
:10A4E00080916C0790916D0761157105810591054B
:10A4F00061F10E9429E920910A0130910B014091FC
:10A500000C0150910D010E9488E920918101309148
:10A51000820140918301509184010E9441F0609337
:10A52000810170938201809383019093840183E081
:10A530000E94E61E81E080936A0110926A071092E1
:10A540006B0710926C0710926D0780916A01882347
:10A5500009F4BECF20915007309151074091520726
:10A560005091530760918101709182018091830124
:10A57000909184010E9440F069837A838B839C834D
:10A58000CE0101960E94331BBC0180E59DE20E9432
:10A59000F8739ECFB0E0A0E0E0EDF2E50C9414F08B
:10A5A0000E946523082F0E945BCBC0916507FC2E9B
:10A5B00085E0E82EEC0E11E01C1BDC2ED194C111BD
:10A5C00014C0809168078823F9F080916A0188237C
:10A5D00009F474C081E090916807911180E024E053
:10A5E0004CE753E06D2D0E94A7CA01113AC0D2E09A
:10A5F000C130C1F5809168078130B9F080916A015E
:10A60000811122C0D2E044C080914F0710924F07C1
:10A610008823D9F20E94624A809167078823A9F2B1
:10A62000CDB7DEB7E7E00C9430F080914F07109281
:10A630004F07882319F389EA94E50E94B1CB8091F2
:10A6400067078823D9F2ECCF81E0909168079130B9
:10A6500009F080E023E043E753E0612F0E94A7CA9E
:10A66000D1CFD1E0DC1314C0809168078D17B9F009
:10A6700080916A01882361F06C2F6F1981E09091BD
:10A6800068079C1380E023E047E653E00E94A7CAD6
:10A69000CF5FCE1194CFDF5FD0936607C1CF80919B
:10A6A0004F0710924F07882319F38CEC99E50E940D
:10A6B000B1CB809167078823D9F2B2CFD1E00023D4
:10A6C00009F4A0CFE5CFB0E0A0E0E9E6F3E50C9413
:10A6D0000DF00E945BCBC09165076C2E85E0782E53
:10A6E0007C0E00E312E89AE2A92E94E0B92ED5E0A0
:10A6F000DC1B22E0E22E22E8F22E84E0D82EDC1AC7
:10A7000083E0C82ECC1A82E0982E9C1A81E0882E15
:10A710008C1AC1112CC0809168078823B9F08091F0
:10A720006A01882361F0662D619581E09091680748
:10A73000911180E024E04EE454E00E94A7CACF5F6C
:10A74000C711E7CF86E0809366070CC080914F0762
:10A7500010924F07882319F30E94624A809167077D
:10A760008823E9F2CDB7DEB7EEE00C9429F0C130D2
:10A7700049F5809168078130A1F080916A018823B2
:10A78000F1F287E492E89F938F9388E494E09F939B
:10A790008F938F9281E090916807913069F180E00A
:10A7A0002BC080914F0710924F07882331F387E425
:10A7B00092E8892B11F00E944782809167078823D5
:10A7C000E1F2D0CFC23009F08FC0809168078230AB
:10A7D000E9F080916A01882309F4B1CF88E093E21F
:10A7E0009F938F938EE394E09F938F939F9281E04A
:10A7F00090916807923099F68F930E9420230F90D2
:10A800000F900F900F900F900F9099CF80914F075E
:10A8100010924F078823E9F20E940823809167076E
:10A820008823B9F29FCF809168078330A9F0809187
:10A830006A01882309F483CF89E192E89F938F937B
:10A8400087E394E09F938F93CF9281E09091680784
:10A85000933009F0A4CFD0CF80914F0710924F07CB
:10A86000882329F389E192E8892B11F00E9419824B
:10A87000809167078823D9F275CF8091680784306B
:10A8800099F080916A01882309F459CFFF92EF92E1
:10A8900082E394E09F938F93DF9281E09091680729
:10A8A000943009F07CCFA8CF80914F0710924F07CA
:10A8B000882339F3E114F10411F00E94028280919F
:10A8C00067078823F1F24ECF80914F0710924F0710
:10A8D0008823B1F00115110511F00E94308280919A
:10A8E0006707882369F03ECFC33009F49CCFC4309A
:10A8F00021F2C53009F023CF80916807853021F31C
:10A9000080916A01882309F41ACF1F930F93BF9295
:10A91000AF92DF9381E090916807953009F03FCFC7
:10A920006BCF80E090E0A0E8B0E480937D0190934D
:10A930007E01A0937F01B09380018AE292E00E94A1
:10A940008E228091F9030E94B6781092FD030C9438
:10A95000624AB0E0A0E0EFEAF4E50C9412F00E9445
:10A960005BCBC091650785E0C82ECC0ED4E0DC1B24
:10A9700013E01C1B82E0F82EFC1A81E0E82EEC1A92
:10A98000BC2EB194C1112BC0809168078823B1F00F
:10A9900080916A01882359F081E0909168079111B4
:10A9A00080E024E045E553E06B2D0E94A7CACF5F0D
:10A9B000CC12E8CF85E0809366070CC080914F07EA
:10A9C00010924F07882321F30E94624A8091670703
:10A9D0008823F1F2CDB7DEB7E9E00C942EF0C13058
:10A9E00089F5809168078130C1F080916A018823E0
:10A9F000F1F2DD24D39480916807813009F0D12CE5
:10AA00008DE79DE00E94191E00E09C014AE453E09E
:10AA10006E2D8D2D0E945F74CACF80914F071092CA
:10AA20004F07882311F30E944FCB41E85CE26DE7AA
:10AA30007DE08AE493E00E94C0CB80916707882381
:10AA4000A1F2C8CFC23009F073C08091680782308C
:10AA5000B1F080916A01882309F4A9CFDD24D39451
:10AA600080916807823009F0D12C81E89DE00E9436
:10AA7000191E00E09C014FE353E06F2DCACF809177
:10AA80004F0710924F07882321F30E944FCB40E8D5
:10AA90005CE261E87DE08FE393E00E94C0CB8091AF
:10AAA00067078823B1F296CF809168078330B1F0B1
:10AAB00080916A01882309F47ACFDD24D3948091B0
:10AAC0006807833009F0D12C85E89DE00E94191EAB
:10AAD00000E09C0144E353E0612F9BCF80914F073E
:10AAE00010924F07882321F30E944FCB4FE75CE27F
:10AAF00065E87DE084E393E00E94C0CB8091670726
:10AB00008823B1F267CF80914F0710924F078823B7
:10AB1000C9F00E944FCB4EE75CE269E87DE089E234
:10AB200093E00E94C0CB80916707882359F052CFF1
:10AB3000C33009F4B9CFC43009F039CF8091680728
:10AB4000843009F380916A01882309F430CFDD2431
:10AB5000D39480916807843009F0D12C89E89DE076
:10AB60000E94191E00E09C0149E253E06D2F51CF75
:10AB7000A3E0B0E0EEEBF5E50C9409F04C013B01ED
:10AB80005A011901280181E08093FD0340916A0771
:10AB900050916B0760916C0770916D0741155105DD
:10ABA0006105710571F0141615060CF080E08093B4
:10ABB000F70310926A0710926B0710926C071092BD
:10ABC0006D071091F70380914F078B8310924F0709
:10ABD000811105C080916A01882309F46FC0C20108
:10ABE0000E944A70082F80E0C114D10419F0C601F8
:10ABF0000E944A701A821982E114F104B1F4402FC4
:10AC000050E0282F30E0CA01820F931F46976CF462
:10AC100085E190E0841B950B821B930B97FD0196B9
:10AC2000959587958A8381E0898301E020E83AE65B
:10AC3000A201BE016F5F7F4FCE0102960E94A271FA
:10AC4000E114F10491F08A81882321F01A8289812C
:10AC50008F5F898300E023E83AE6A701BE016F5FBA
:10AC60007F4FCE0102960E94A271C114D10459F007
:10AC700000E020E83AE6A601BE016F5F7F4FCE01FB
:10AC800002960E94A27141E04127B30181E00E9437
:10AC90005ED2C4010E944A70412FB40194E1981B16
:10ACA000892F0E945ED2EB81EE2341F0111101C089
:10ACB0005101A114B10431F0F50109952396E2E1A7
:10ACC0000C9425F00E94624AF9CFCF92DF92EF9266
:10ACD000FF920F931F938EE9C82E85E0D82EF12C9A
:10ACE000E12C00EA15E030E020E042E156E460EBC0
:10ACF00075E085EB95E03CDF1F910F91FF90EF90A1
:10AD0000DF90CF900895B0E0A0E0E9E8F6E50C947C
:10AD100011F0ADB6BEB6809123106AE777E08823C4
:10AD200011F063E270E1FB0101900020E9F7CF012F
:10AD3000861B970B01962DB73EB7281B390B0FB614
:10AD4000F8943EBF0FBE2DBF8DB79EB701967C0114
:10AD500080E2EDB7FEB78183C70101960E9465F2DC
:10AD60008AE5C82E85E0D82E0CE515E030E020E01D
:10AD70004CED56E468E675E08FE695E0F9DE0FB637
:10AD8000F894BEBE0FBEADBEEAE00C942DF0CF929B
:10AD9000DF92EF92FF920F931F9388EBC82E84E00F
:10ADA000D82EF12CE12C0BE215E030E020E04DEB49
:10ADB00054E66AEB74E08FEB94E0DADE1F910F91BA
:10ADC000FF90EF90DF90CF900895CF92DF92EF92B7
:10ADD000FF920F931F938AE8C82E83E0D82EF12CA0
:10ADE000E12C0CE813E021E934E546E952E268E998
:10ADF00073E08DE993E0BCDE1F910F91FF90EF901F
:10AE0000DF90CF900895B0E0A0E0E9E0F7E50C9482
:10AE100011F0ADB6BEB683E392E00E944A7090E0B6
:10AE200001962DB73EB7281B390B0FB6F8943EBFDD
:10AE30000FBE2DBF8DB79EB701967C0163E372E014
:10AE40000E946BE88091280700E012E0813031F029
:10AE50000BEE11E0823011F003E112E084E2C82E23
:10AE600082E0D82E20ED36E44FE352E666E272E04F
:10AE70008DE292E07DDE0FB6F894BEBE0FBEADBE91
:10AE8000EAE00C942DF08F929F92AF92BF92CF92F6
:10AE9000DF92EF92FF920F9380914F0710924F072E
:10AEA000882371F01092FD030E94624A0F91FF9077
:10AEB000EF90DF90CF90BF90AF909F908F900895CC
:10AEC00081E08093FD0380916A0790916B07A091C8
:10AED0006C07B0916D070097A105B10509F44AC050
:10AEE0005C01AA0CBB1CAA0CBB1C10926A07109236
:10AEF0006B0710926C0710926D07B5010B2C000CBC
:10AF0000880B990B0E9429E92091B0073091B10775
:10AF10004091B2075091B3070E9488E920915613DF
:10AF20003091571340915813509159130E9441F09A
:10AF30006B017C0120E030E040EA51EC0E94A4F17A
:10AF400087FD18C020E030E040EA51E4C701B601B7
:10AF50000E9423E9181674F0C5010E94D5C6C0925C
:10AF60005613D0925713E0925813F092591382E07F
:10AF700080936A0180916A01882309F497CFC09079
:10AF80005613D0905713E0905813F090591320E0C7
:10AF900030E44CE156E4C701B6010E9488E94B0158
:10AFA0005C0120E030E0A901C701B6010E9423E95D
:10AFB00020E030E040EA50E487FF04C020E030E0C9
:10AFC00040EA50ECC501B4010E9441F02DEC3CEC8C
:10AFD0004CEC5DE30E9488E90E9420F16B017C014A
:10AFE0008BE2F7FE09C0F094E094D094C094C11CA9
:10AFF000D11CE11CF11C8DE280939802C701B601BF
:10B0000020E137E240E050E00E9473EF6AE0862ED4
:10B01000912CA12CB12CCA01B901A50194010E9467
:10B0200073EF605D60939902C701B60128EE33E0CB
:10B0300040E050E00E9473EFCA01B901A5019401FC
:10B040000E9473EF605D60939A028EE280939B0290
:10B05000C701B60124E630E040E050E00E9473EF03
:10B06000CA01B901A50194010E9473EF605D60936C
:10B070009C02C701B601A50194010E9473EF6B0108
:10B08000CA01B901A50194010E9473EF605D60934C
:10B090009D0260E36C0D60939E0268E972E084EFAC
:10B0A00092E00E94F873C0905613D0905713E0902E
:10B0B0005813F09059138090F3039090F403A090EC
:10B0C000F503B090F603A5019401C701B6010E94F3
:10B0D00023E98823E9F020E030E0A901C701B601A7
:10B0E0000E9423E9882309F479C0A5019401C701CE
:10B0F000B6010E9423E987FD73C081E08093F203CB
:10B10000C092F303D092F403E092F503F092F603B9
:10B11000D090F2038091AB13813188F48091AD130C
:10B12000833068F044E04D195CEDE52E52E0F52ED9
:10B130000CE022E062E487E793E10E949AD38091D9
:10B14000AB13853180F48091AD13843160F049ED0B
:10B15000E42E42E0F42E01E023E044E16CE387E7D3
:10B1600093E10E949AD38091AB138F3308F09ECE67
:10B170008091AD138F3208F499CE40E34D198FEBD7
:10B18000E82E82E0F82E0DE022E06AE587E793E101
:10B190000E949AD341E34D1995EAE92E92E0F92EE7
:10B1A00022E065E087E793E10E949AD325E7E22E4B
:10B1B00022E0F22E00E123E04FE262E187E793E133
:10B1C0000E949AD335E4E32E32E0F32E23E04FE2DF
:10B1D00067E687E793E10E949AD368CE80E08ECF3E
:10B1E0008FEF8CCF0F931F93CF93DF93FC01EB0175
:10B1F00080916A0790916B07A0916C07B0916D07E1
:10B20000B7FF08C010926A0710926B0710926C0784
:10B2100010926D078091590790915A07A0915B0792
:10B22000B0915C0740916A0750916B0760916C0781
:10B2300070916D0784179507A607B70744F48093AC
:10B240006A0790936B07A0936C07B0936D0780918A
:10B250006A018823E1F060916A0770916B07809121
:10B260006C0790916D0700915D0710915E0720912A
:10B270005F0730916007600F711F821F931F099550
:10B28000BC0180916307909164070E94F8738091DC
:10B290004F07811108C0809156078823A9F180913A
:10B2A0006A01882389F18091610790916207009774
:10B2B000B1F040916A0750916B0760916C077091F3
:10B2C0006D0700915D0710915E0720915F07309137
:10B2D0006007400F511F621F731FFE010995E09127
:10B2E0005707F0915807309741F080915607811128
:10B2F00003C080914F078111099580914F071092EB
:10B300004F0781110E94624ADF91CF911F910F91E7
:10B3100008956FE17DE188E39DE164CF6CE97DE113
:10B3200085E695E45FCF6AEA7DE18DEC9EE15ACF38
:10B330006EEB7DE182ED9DE155CF6BE07EE181E832
:10B3400095E450CFE091EB03E63028F581E08E0FD5
:10B350008093EB0340916A0750916B0760916C07F3
:10B3600070916D0720916507909166078091FD03AC
:10B3700039E0E39FF0011124EB54FC4FA0917113CD
:10B38000B0917213B183A083428353836483758326
:10B390002683978380870895A7E0B0E0E2EDF9E582
:10B3A0000C9409F00E945BCBF09065072F2C85E090
:10B3B0008F0D8D833324339483E0E82E98EE892E0D
:10B3C00093E0992EA12CB12C84E08F198E839E2DB1
:10B3D0009F199F8382E0D82EDF18C32CCF18F1105D
:10B3E0002CC0809168078823C1F080916A0188236E
:10B3F00061F0622D619581E090916807911180E084
:10B4000024E045E553E00E94A7CAF3949D81F91218
:10B41000E6CF85E0809366070CC080914F071092BD
:10B420004F07882311F30E94624A8091670788239F
:10B43000E1F22796E2E10C9425F081E0F8122DC0AC
:10B44000909168079130B9F080916A018823E9F200
:10B4500081E0913009F080E0909199032DE133E093
:10B46000911102C029E133E001E040E253E06C2D8C
:10B470000E945F74CACF80914F0710924F078823B4
:10B4800019F3809199038F2580939903E0926A01C3
:10B49000809167078823C1F2CCCF92E0F912D1C026
:10B4A00080916807823021F180916A01882309F434
:10B4B000ACCF11E080916807823009F010E0609114
:10B4C000080170910901072E000C880B990B0E944E
:10B4D00029E969837A838B839C83CE0101960E943C
:10B4E000784500E09C0142E153E06D2D812FC0CFF3
:10B4F00080914F0710924F078823B1F210E000E0CF
:10B5000025EF30E050E040E068E071E082E193E058
:10B510000E9420CC80916707882331F28ACF8091E6
:10B520006807833019F180916A01882309F46DCF8F
:10B5300011E080916807833009F010E06091060106
:10B5400070910701072E000C880B990B0E9429E9C6
:10B5500069837A838B839C83CE0101960E94784510
:10B5600000E09C014BE053E06F81C0CF80914F071A
:10B5700010924F078823B9F210E000E025EF30E089
:10B5800050E040E066E071E08BE093E00E9420CC68
:10B5900080916707882339F24CCF80914F07109232
:10B5A0004F07882309F459C020E030E048EC52E40A
:10B5B0006091020170910301809104019091050155
:10B5C0000E9488E90E9425F12B0130926707BADEBC
:10B5D000E0926A0183E093E09093640780936307AD
:10B5E00082E091E0909362078093610710925D077B
:10B5F00010925E0710925F071092600780925907C1
:10B6000090925A07A0925B07B0925C07712C612C54
:10B6100040926A0750926B0760926C0770926D07B8
:10B6200088E999E5909372138093711310925807EB
:10B63000109257071092560780916707882369F088
:10B64000F8CE83E0F81609F46ACF94E0F912DDCE63
:10B6500080916807843009F4A0CF80916A01882323
:10B6600009F4D3CE11E080916807843009F010E02E
:10B670004090020150900301609004017090050118
:10B6800020E030E0A901C301B2010E9423E92DEBC3
:10B6900037E346E055EB87FD04C02DEB37E346E08A
:10B6A00055E3C301B2010E9441F069837A838B8321
:10B6B0009C83CE0101960E94A91B00E09C0143E0FF
:10B6C00053E06E8113CFB0E0A0E0E9E6FBE50C9417
:10B6D00019F08D8190919410891778F080939410CF
:10B6E0009E01285F3F4F4E815F8164E570E08FE3EC
:10B6F00090E10E94EBE810923E10E2E00C9435F0ED
:10B700000F931F93CF93DF936F3F11F41092941018
:10B710002091941021111EC08C010E9472E8800FAC
:10B72000911FEC01C01BD10BC535D1053CF0019731
:10B73000FC012491207C2038D1F3F3CFDD27AE012A
:10B74000B8018FE390E10E9493E8C15CDF4E18825C
:10B7500010923E10DF91CF911F910F910895A6E8AE
:10B76000B0E0E5EBFBE50C9414F0C358DF4F188212
:10B7700019821A821B82CD57D04080918E029091FF
:10B780008F02A0919002B0919102CF57DF4F888332
:10B790009983AA83BB83C158D04084E690E09093FC
:10B7A0009E1280939D121092C2121092C11210929A
:10B7B0002A0464E070E0CE018F579F4F0E9483CF30
:10B7C00080919D1290919E12029690939E1280936A
:10B7D0009D121092C2121092C11281E0CA57DF4F1F
:10B7E0008883C658D040CE018A579F4F0E94772247
:10B7F00068E470E089E69DE00E9483CF80E1E1E9A2
:10B80000F1E08E010F5F1F4FD80101900D928A95D4
:10B81000E1F760E170E0C8010E9483CF8BE897E018
:10B820000E947F228CE0F80111928A95E9F7C80105
:10B830000E947B227E01FDE6EF0EF11C8FEFF701E7
:10B840008083C7010E94772219821A821B821C8280
:10B85000C8010E947F228091B1029091B202A09112
:10B86000B302B091B40289839A83AB83BC83C801CD
:10B870000E947F22C358DF4F188219821A821B82CE
:10B88000CD57D04083E0F70180838983CE01835870
:10B890009F4F0E947F22C7010E947722C8010E9409
:10B8A00077222AE0D22EDA94DD2031F0CE018358BF
:10B8B0009F4F0E947F22F7CF8EE493E10E947B226C
:10B8C000C358DF4F188219821A821B82CD57D0408D
:10B8D0009AE0D92EDA94DD2031F0CE0183589F4FC3
:10B8E0000E947F22F7CF87E08983F7018083C80118
:10B8F0000E947722C7010E94772268E070E081E809
:10B9000093E00E9483CF68E070E089E793E00E94B3
:10B9100083CF64EC70E085EB92E00E9483CF1982C4
:10B92000DD24DA94F701D082C8010E947322C70196
:10B930000E94772264E070E082E392E00E9483CF6D
:10B940008091E3068983C8010E9473226CE070E055
:10B9500083E497E00E9483CF198A1A8A1B8A1C8A83
:10B9600080E090E0A0E8BFE38D879E87AF87B88B2B
:10B970008091B5129091B612A091B712B091B81201
:10B9800089839A83AB83BC8320E030E543EC50E4A9
:10B990006091B9127091BA128091BB129091BC1251
:10B9A0000E9488E96D837E838F8398872CEA35EC2B
:10B9B00047E25EE36091BD127091BE128091BF12AA
:10B9C0009091C0120E9488E969877A878B879C874B
:10B9D00064E170E0C8010E9483CF84E190E09A8323
:10B9E000898362E070E0C8010E9483CF80913707AD
:10B9F00090913807A0913907B0913A0789839A83CB
:10BA0000AB83BC8320E030E543EC50E460913B071E
:10BA100070913C0780913D0790913E070E9488E914
:10BA20006D837E838F8398872CEA35EC47E25EE353
:10BA300060913F07709140078091410790914207C4
:10BA40000E9488E969877A878B879C87C8010E9452
:10BA50006F228CE0E1EAF1E0D80101900D928A9525
:10BA6000E1F7C8010E946F221982C8010E94772263
:10BA70008FE78983C8010E947722D982C8010E947A
:10BA8000772285E0EDEAF1E0D80101900D928A95E8
:10BA9000E1F765E070E0C8010E9483CF1982C80118
:10BAA0000E94732280E2E2EBF1E0D80101900D9256
:10BAB0008A95E1F760E270E0C8010E9483CFF70148
:10BAC0001082C7010E9473221982C8010E9473224A
:10BAD00080E090E0A0EEBFE3C358DF4F88839983F6
:10BAE000AA83BB83CD57D040CE0183589F4F0E947D
:10BAF0007F22C358DF4F188219821A821B82CD57CA
:10BB0000D040CE0183589F4F0E947F2282E1F801EE
:10BB100011928A95E9F762E170E0C8010E9483CF33
:10BB200084E2E2EDF1E0D80101900D928A95E1F70F
:10BB300064E270E0C8010E9483CF80E1F8011192B5
:10BB40008A95E9F760E170E0C8010E9483CF89E03F
:10BB5000F80111928A95E9F769E070E0C8010E9446
:10BB600083CFC358DF4F188219821A821B82CD57A8
:10BB7000D040CE0183589F4F0E947F228CE0D82E68
:10BB8000F8018D2D11928A95E9F76CE070E0C801FB
:10BB90000E9483CF8CE6F80111928A95E9F76CE652
:10BBA00070E0C8010E9483CF8EE194E00E946F2272
:10BBB000F70110821182128213821482158216827A
:10BBC000178268E070E0C7010E9483CFF7011192ED
:10BBD000DA94E9F7CB57DF4F1882C558D04080E0A0
:10BBE00090E0A0E4B0E4ED968CAF9DAFAEAFBFAFF8
:10BBF000ED97C7010E947B22CE018B579F4F0E9479
:10BC00007722CE0187589F4F0E947F2280912A047D
:10BC1000811127C000919D1210919E128091C11236
:10BC20009091C212F7019183808384E690E0909313
:10BC30009E1280939D1264E070E086E392E00E9481
:10BC400083CF62E070E0C7010E9483CF91E00037AC
:10BC5000F3E01F0709F490E080912A04892B809378
:10BC60002A0480912A04811104C060E08BE39AE0E9
:10BC700047DD90912A0481E08927CA57DF4FE7E02A
:10BC80000C9430F06CCDA3E0B0E0E9E4FEE50C9458
:10BC900009F00E946523582E0E945BCB2091650716
:10BCA0002A83422E2B5F2B8383E0782E74180CE5B9
:10BCB00014E021E6E22E2AE4F22E3DE6C32E34E023
:10BCC000D32E42E4A42E4EE5B42E5BE7852E54E03D
:10BCD000952E82E08419898381E0382E3418242C33
:10BCE00021948A8181118EC080916807882309F48C
:10BCF00077C080916A01882359F081E090916807AC
:10BD0000911180E024E043EB54E0622D0E94A7CA29
:10BD100051103DC18A81833009F029C180916807A3
:10BD2000833009F4C3C080916A018111D0C084E0DE
:10BD3000682E81E0860D51104AC09A8189131FC078
:10BD400080916807891709F4F4C080916A018823FB
:10BD5000B1F0FF92EF92DF92CF928A8184198F9394
:10BD600081E0909168072A81921380E08F930E946E
:10BD700020230F900F900F900F900F900F9082E064
:10BD8000860D9A81891321C080916807891709F46B
:10BD9000DFC080916A018823C1F082EE91E49F9315
:10BDA0008F931F930F938A8184198F9381E09091D1
:10BDB00068072A81921380E08F930E9420230F90BE
:10BDC0000F900F900F900F900F9083E0860D9A8147
:10BDD0009F5F9A832B81291384CF809366070EC0BF
:10BDE00080914F0710924F07882309F482CF0E9459
:10BDF000624A80916707882309F47BCF2396E2E1AA
:10BE00000C9425F09A81913051F58091680781302A
:10BE1000B9F080916A01882309F47ACF81E090918A
:10BE20006807913009F080E023E041EA54E0632D97
:10BE30000E94A7CA5110ABC085E094E0692E7DCF67
:10BE400080914F0710924F07882319F38AEC92E5EF
:10BE50000E94B1CB809167078823D9F2CFCF2A8186
:10BE6000223009F055CF80916807823081F08091AF
:10BE70006A01882309F44CCF81E0909168079230E1
:10BE800009F080E023E042E954E06981D1CF80915C
:10BE90004F0710924F07882351F383E497E50E94E0
:10BEA000B1CB80916707882311F3A8CF80914F070A
:10BEB00010924F07882309F436CF83E693E50E945A
:10BEC000B1CB80916707882309F42DCF97CF81E00C
:10BED00090916807933009F080E023E04AE854E04D
:10BEE000672D0E94A7CA23CF80914F0710924F075A
:10BEF000882309F446C033DC80916707882309F45E
:10BF000040C07CCFBF92AF929F928F928A8184195A
:10BF10008F9381E0909168072A81921380E08F933C
:10BF20000E9420230F900F900F900F900F900F9072
:10BF30002CC080914F0710924F07882309F405CF3A
:10BF40000E94544A80916707882309F4FECE56CF99
:10BF500080914F0710924F07882309F41ACF0E944F
:10BF6000BE4080916707882309F413CF47CF8A81A9
:10BF7000843009F061CF809168079A81891709F4AC
:10BF8000B3CF80916A018111BDCF8A81D1CE9A81D0
:10BF900084E0933009F01BCFEECFA7E0B0E0E3EDF3
:10BFA000FFE50C9409F08091770787708983809072
:10BFB000810390908203A0908303B09084030E9439
:10BFC0005BCB209165072E833981373009F075C02E
:10BFD00085E194E09B838A831E81312F3B5F3C8304
:10BFE00033243394812F81958D83232C211A84E669
:10BFF000482E512C612C712C2E81222309F462C011
:10C000003981373009F434C22E81213009F029C238
:10C0100090916807913009F445C180916A018111BE
:10C0200054C182E0F82E81E08F0D8F839981973083
:10C0300009F063C020E030E0A901C501B4010E940D
:10C0400023E9882309F459C03F818E81381331C018
:10C050009091B0029F83809168072E81821311C056
:10C0600080914F0710924F07882359F093259F83A3
:10C0700083E080936A010E94832280916707811187
:10C080000DC180916A018823A1F06E81611B81E05E
:10C09000909168073E81931380E09F8126EF33E003
:10C0A000911102C022EF33E001E049EF53E00E941A
:10C0B0005F74F394F394FF8220C020E134E03B836B
:10C0C0002A838ACF80916807882309F4D9C0809198
:10C0D0006A01882309F494CF81E090916807911157
:10C0E00080E024E043E254E06D810E94A7CA898188
:10C0F000873009F41DC193E09F838091B102909134
:10C10000B202A091B302B091B40280932807909339
:10C110002907A0932A07B0932B072F813E81231371
:10C120001EC080916807821709F407C180916A01D7
:10C130008823A9F0EE80E11AFF24F3948091680728
:10C140003E818313F12C88E297E00E94284500E0AD
:10C150009C0146EE53E06E2D8F2D0E945F748F81FF
:10C160008F5F9E81891316C080916807891709F433
:10C1700039C180916A01882369F06E81611B81E079
:10C18000909168072E81921380E023E047ED53E001
:10C190000E94A7CA8F818E5F3E81831316C0809153
:10C1A0006807831709F42FC180916A01882369F019
:10C1B0006E81611B81E0909168072E81921380E06F
:10C1C00023E04AEC53E00E94A7CA8F818D5F3E8135
:10C1D000831323C080916807831709F425C18091D8
:10C1E0006A018823D1F081E69AE49F938F938CEBC8
:10C1F00093E09F938F938E81811B8F9381E0909129
:10C2000068073E81931380E08F930E9420230F9054
:10C210000F900F900F900F900F908F818C5F9E81E9
:10C22000891323C080916807891709F40CC1809194
:10C230006A018823D1F082E49EE59F938F938DEA73
:10C2400093E09F938F938E81811B8F9381E09091D8
:10C2500068072E81921380E08F930E9420230F9015
:10C260000F900F900F900F900F903E813F5F3E8395
:10C270008C818313C1CE9F819B5F909366070EC014
:10C2800080914F0710924F07882309F420CF0E9416
:10C29000624A80916707882309F419CF2796E2E163
:10C2A0000C9425F080914F0710924F07882309F4D2
:10C2B000B4CE20EF35E03093E5062093E40680917C
:10C2C0006707882309F4A9CEE9CF81E0913009F00E
:10C2D00080E020E249E154E0622D0E94A7CAA1CE8D
:10C2E000909168073E81931731F080916A01811126
:10C2F00013C08E8197CE80914F0710924F078823ED
:10C30000A1F32A813B813093E5062093E4068091D6
:10C310006707882351F3C2CF6E81611B81E03E81A4
:10C32000931380E020E246E054E00E94A7CAE1CFE8
:10C3300022E02F83FF24F3947DCE80914F0710924B
:10C340004F07882309F4F2CE0E944FCB6091280753
:10C350007091290780912A0790912B070E9425F15F
:10C360006B01309267070E94A25983E080936A01B3
:10C3700086EE93E0909364078093630728E237E0AA
:10C38000309362072093610710925D0710925E0759
:10C3900010925F07109260074092590750925A0717
:10C3A00060925B0770925C07F12CE12CC0926A07E7
:10C3B000D0926B07E0926C07F0926D078EE899E5DA
:10C3C000909372138093711329E832E230935807E7
:10C3D000209357071092560780916707882309F426
:10C3E000A5CE5CCF80914F0710924F07882309F4A8
:10C3F000C0CE83E497E50E94B1CB80916707882384
:10C4000009F4B7CE4BCF80914F0710924F07882386
:10C4100009F4CACE82E996E40E94B1CB8091670705
:10C42000882309F4C1CE3ACF80914F0710924F076D
:10C43000882309F4D4CE0E94544A80916707882348
:10C4400009F4CDCE2BCF80914F0710924F07882350
:10C4500009F4EDCE84D980916707882309F4E7CEEB
:10C460001DCF2E81223009F43BCF33E03F8345CEF0
:10C470008E81813009F434CF92E09F835BCF0E949C
:10C48000BE406DD90C94D046CF938091AD038111FD
:10C4900009C08CED91E09093F1038093F00381E06B
:10C4A0008093AD030E94A25920E040E070E060E07C
:10C4B00080E793E20E949445C1E0C093FD030E948F
:10C4C000822C0E94624AC093FD0360E08AEB9DE2E9
:10C4D00017D988ED91E09093E5068093E406CF911B
:10C4E0000895A6E0B0E0E7E7F2E60C9409F00E94B8
:10C4F000967A382E8091C91484FB662460F8412C0A
:10C5000084FF03C00E94A97A482E0E945BCB209131
:10C5100065072D83522E2B5F298380E009E115E00A
:10C5200091E0792E7518952D91959A8394E4E92ED2
:10C5300092E6F92E26E3C22E25E0D22E92E095193E
:10C540009B8393E095199C8335ED832E34E0932EE5
:10C550004AEEA42E44E0B42E9D812981921709F45D
:10C5600009C2992349F131106AC00E94EC808823E6
:10C5700009F47AC19D81913009F444C122E02E83EF
:10C580002D818E8128135FC180916807281709F4D7
:10C590006EC180916A01882309F455C16D816519C6
:10C5A00081E0909168072D81921380E023E042E1C1
:10C5B00055E00E94A7CA47C180916807882379F196
:10C5C00080916A01882379F281E090916807911146
:10C5D00080E024E042E455E06A810E94A7CA33204B
:10C5E00021F224E02E839D812E8192134AC08091F6
:10C5F0006807981709F44CC180916A01882309F4EF
:10C6000040C06D81651981E0909168072D8192137A
:10C6100080E023E046E055E00E94A7CA32C0809146
:10C620004F0710924F07882359F20E94624A809167
:10C630006707882329F22696E2E10C9425F08D8184
:10C64000813009F47FC0823009F4A6C09D81933007
:10C6500041F680916807833009F4C3C080916A0174
:10C66000882309F4BECF81E090916807933009F0E8
:10C6700080E023E046E255E06C810E94A7CA84E096
:10C680008E838E818F5F9D81981316C0809168077D
:10C69000981709F40EC180916A01882369F06D81B1
:10C6A000651981E0909168072D81921380E023E065
:10C6B00048EF54E00E94A7CA8E818E5F662009F47D
:10C6C00030C141103BC09D8198131BC0209068076A
:10C6D000921509F4FFC080916A01882391F01F929E
:10C6E000BF92AF928D8185198F9381E02D812211A8
:10C6F00080E08F930E9420230F900F900F900F9057
:10C700000F908E818D5F9D81981316C08091680770
:10C71000981709F4F5C080916A01882369F06D814A
:10C72000651981E0909168072D81921380E023E0E4
:10C7300049ED54E00E94A7CA8E818C5F9D819F5F66
:10C740009D830ACF809168078130D1F080916A0182
:10C75000882309F446CFFF92EF92DF92CF927F9227
:10C7600081E090916807913009F080E08F930E94FA
:10C7700020230F900F900F900F900F900F9031CFBC
:10C7800080914F0710924F07882301F37DDE80913F
:10C7900067078823D9F24FCF80916807823091F0E4
:10C7A00080916A01882309F41CCF81E09091680789
:10C7B000923009F080E023E04BE255E06B810E946B
:10C7C000A7CA0FCF80914F0710924F07882341F3DC
:10C7D00087EC96E50E94B1CB80916707882301F32F
:10C7E0002ACF80914F0710924F07882309F436CF44
:10C7F00080E89AE40E94B1CB80916707882309F40E
:10C800002DCF19CF80916807813009F180916A019D
:10C81000882309F4B3CE82E294E49F938F931F930D
:10C820000F937F9281E090916807913009F080E04A
:10C830008F930E9420230F900F900F900F900F90D6
:10C840000F9082E08E838E818F5F8E83CCCE80911D
:10C850004F0710924F078823C9F20E94224480910B
:10C860006707882399F2E7CE91E09E8389CE809175
:10C870004F0710924F07882309F48BCE8DEE9EE46C
:10C880000E94B1CB80916707882309F482CED3CE72
:10C8900080914F0710924F07882309F4ADCE89E4A9
:10C8A0009CE40E94B1CB80916707882309F4A4CE51
:10C8B000C2CE80914F0710924F07882309F4EBCE28
:10C8C00083E49EE50E94B1CB80916707882309F439
:10C8D000E2CEB1CE80914F0710924F07882309F422
:10C8E000FACE4FE350E064EC74E086EE96E00E94EE
:10C8F0007AF280916707882309F4EDCE8D811ECFEF
:10C9000080914F0710924F07882309F404CF81EBE1
:10C9100098E60E94B1CB80916707882309F4FBCE8B
:10C92000EDCF9D81981314C0909168072D81291730
:10C9300091F080916A01882359F06D81651981E039
:10C940002D81291380E020E248EC54E00E94A7CA20
:10C950008E818D5FF3CE80914F0710924F07882311
:10C9600041F39092E5068092E40680916707882360
:10C9700001F3C4CF809366075ECE109297021092A7
:10C9800069010E94A97A9091C91480FB97F990934C
:10C99000C91460E08AEC91E00E94805B0C94D04660
:10C9A0000F931F930E94D9CF0091A9031091AA035E
:10C9B0002091AB033091AC03601B710B820B930B86
:10C9C00097FD0CC089B183FB882780F991E0892706
:10C9D0004A9B8260309B84608093A8038091A80367
:10C9E00081709091A80391FD82609091A7039817A0
:10C9F00049F0813009F148F0823079F0833091F0CC
:10CA00008093A7031F910F910895913079F0923090
:10CA1000B9F79091960291500CC0992339F0933058
:10CA2000C1F3EECF9130A9F3923051F79091960275
:10CA30009F5F90939602E4CF992359F3933001F7C7
:10CA4000F5CF1F93CF93DF93809137018F3708F491
:10CA500075C08F579091B4129093AE04992309F446
:10CA60006BC05D9A909136079093AD04992309F4B9
:10CA70006FC05C9A8F5F809337018091AC0491E026
:10CA800089278093AC0481118BDF8091360191E07E
:10CA9000980F85300CF090E0823009F4A8C00CF0BB
:10CAA00059C0882309F46EC0813009F495C0909371
:10CAB0003601C0917807D0917907209709F42DC0ED
:10CAC000F89413B1147082E00E94012C00C000C0E1
:10CAD0001C161D060CF0B9C02A9A00C000C02B9A83
:10CAE00000C0000082E090E00197F0F72B9800C0B2
:10CAF00000C0112309F4ABC02A9A00C000C078948A
:10CB000080917807909179071C161D060CF0A1C042
:10CB1000019790937907809378078091B10D909158
:10CB2000B20D009729F001979093B20D8093B10D4B
:10CB3000DF91CF911F9108955D9894CF9091AE04AD
:10CB4000891708F05D989091AD04891708F492CF89
:10CB50005C9890CF843009F461C00CF45BC08530E0
:10CB600009F0A5CF2091AB04211102C08093AB0442
:10CB70008091AB0481508093AB04882309F497CF54
:10CB800095E095CF809135018F5F80311CF48093C3
:10CB900035018DCF1092350180919A03811113C018
:10CBA0002091AA123091AB123093AD122093AC12A7
:10CBB00020912C0730912D0730932F0720932E07BB
:10CBC00081E080939A031092AB121092AA121092F5
:10CBD0002D0710922C076BCF10927B0087E4809377
:10CBE0007C0080917A00806480937A0060CF80918D
:10CBF0007A0086FD26C040917800509179002091FE
:10CC0000AA123091AB12240F351F3093AB12209330
:10CC1000AA124DCF10927B0086E4E1CF80917A007A
:10CC200086FD11C0409178005091790020912C0729
:10CC300030912D07240F351F30932D0720932C079B
:10CC400036CF92E034CF94E032CF2A9846CF2A985C
:10CC500054CF01965ECF4F925F926F927F928F92E8
:10CC60009F92AF92BF92CF92DF92EF92FF92CF93BB
:10CC7000DF9300D000D0CDB7DEB70E94D9CF6B01D3
:10CC80007C01809100018F3FC1F10E94D9CF80903B
:10CC90009B0390909C03A0909D03B0909E03681905
:10CCA00079098A099B0997FD28C080915F139091AB
:10CCB00060138F5F8F70891701F1E0910001E530FB
:10CCC00008F0DBC024E0E29FF0011124E650FE4FA3
:10CCD00080819181A281B38189839A83AB83BC8354
:10CCE00020E030E0A901BE016F5F7F4F85E791E052
:10CCF0000E94B0C58FEF8093000152DE8091A8039F
:10CD000082FFC4C08091A60381111DC091E0909361
:10CD1000A60380919702892780934F07109297026C
:10CD200083E080936A011092A8030E94D9CF6C50CF
:10CD30007E4F8F4F9F4F6093A9037093AA038093F8
:10CD4000AB039093AC038091920290919302A091D7
:10CD50009402B0919502A7019601281B390B4A0B4A
:10CD60005B0BDA01C901B7FF05C08091FA03882384
:10CD700009F4C7C1D701C6018C599F4FAF4FBF4FB0
:10CD80008093920290939302A0939402B0939502A1
:10CD900060919602062E000C770B77FF03C0719509
:10CDA00061957109909196028091A503981371C0C5
:10CDB000633008F06EC010929602809196028093C4
:10CDC000A503643008F075C080914F078111F3C04E
:10CDD0008091711390917213875B9A4741F480910F
:10CDE0000101882309F4F9C08150809301010E9458
:10CDF000562F8090A3079090A407A090A507B0900D
:10CE0000A60781110E94632FD501C4013AE0B695AF
:10CE1000A795979587953A95D1F7009741E0A40794
:10CE2000B10520F08FEF9FEFA0E0B0E096958795D9
:10CE300020916A012111E3C03091FA0331118DC1B3
:10CE40008091711390917213875B9A4709F46CC1BA
:10CE50008091FD03811168C18091A1039091A2038B
:10CE6000A091A303B091A403C81AD90AEA0AFB0A45
:10CE7000F7FC68C10E94D04665C180916B0190911A
:10CE80006C01A0916D01B0916E0126CF1092A603A6
:10CE90005ACF633009F091CF8091960287FD07C089
:10CEA00081E0880F880F8093960264E086CF8FEF31
:10CEB000F8CF8091720721E030E040E050E0882315
:10CEC00009F456C080906E0790906F07A09070078D
:10CED000B090710781149104A104B104E9F170E0EC
:10CEE00090E080E00E9427E920E030E040E85EE347
:10CEF0000E9488E92B013C01C701B6016819790934
:10CF00008A099B090E9427E99B01AC01C301B20178
:10CF10000E94B8F020E030E04AE754E40E9488E93B
:10CF20004B015C0120E030E040EA52E40E94A4F1B1
:10CF300024E630E040E050E087FF12C020E030E01F
:10CF400040EF51E4C501B4010E94A4F12AE030E0B1
:10CF500040E050E087FF04C021E030E040E050E0D6
:10CF6000C0926E07D0926F07E0927007F09271073F
:10CF7000A09196020A2E000CBB0B0E9499EF24E0B0
:10CF800030E040E050E00E9473EF80916A0790919A
:10CF90006B07A0916C07B0916D07820F931FA41FC0
:10CFA000B51F80936A0790936B07A0936C07B093AB
:10CFB0006D0710929602D701C6018856954CAF4F67
:10CFC000BF4F8093A1039093A203A093A303B093B8
:10CFD000A40381E080936A01FBCE8CE08093010181
:10CFE00080919F039091A003009729F0019790935F
:10CFF000A00380939F0381E080936A01F8CE00979D
:10D0000041F040919F035091A0034817590708F041
:10D0100017CF8091FA03811112C0223038F02430EA
:10D0200008F441C0243011F410926A0183E793E1BF
:10D030000E946D7281E0809369078093FA0383E018
:10D040000E94367181E080939713E0917113F09103
:10D0500072130995109269078091FA03811127C014
:10D0600010924F078091711390917213875B9A47CA
:10D0700009F0EECE0E94D9CFDC01CB018C199D09BD
:10D08000AE09BF0980909F039090A003B12CA12C02
:10D0900088169906AA06BB0608F0D2CE9093A00384
:10D0A00080939F03CDCE81E080936A01BFCF87E755
:10D0B00093E10E9494D291E0811101C090E090939D
:10D0C000FA03882369F28091711390917213875B40
:10D0D0009A47B9F40E94D9CFDC01CB018C199D0984
:10D0E000AE09BF09C0909F03D090A003F12CE12CA2
:10D0F000C816D906EA06FB0620F49093A003809395
:10D100009F030F900F900F900F90DF91CF91FF90A2
:10D11000EF90DF90CF90BF90AF909F908F907F90D7
:10D120006F905F904F90089548E9C40E4AE3D41E73
:10D13000E11CF11CC092A103D092A203E092A303D0
:10D14000F092A4038091FA038111DBCF80916A01F0
:10D150008130B9F610926A01D4CF009709F46FCFED
:10D1600050CFACE3B0E0E7EBF8E60C9409F0809127
:10D170006907882369F18091C91410E000E084FFF9
:10D1800023C08EED92E10E94AC248BE1EEEDF2E142
:10D19000DE01919601900D928A95E1F710E000E092
:10D1A000BE016F5F7F4FCE0181960E9485D9181610
:10D1B0003CF4CE0101960E94F8D3080F111DF0CF68
:10D1C000CE0181960E947C261093FC030093FB0302
:10D1D0000E945BCB10916507312E85E0810F8CAFEB
:10D1E000212E21948DE5A82E8DE1B82E9BE8892E65
:10D1F00095E0992E01E0011B20E9622E25E0722EB8
:10D20000111113C080916807882391F180916A0100
:10D21000882359F081E090916807911180E024E023
:10D2200049E955E0622D0E94A7CA8091C91486FF82
:10D230003EC01130D9F480916807813049F1809166
:10D240006A01882309F43EC11F927F926F920F9367
:10D2500081E090916807913009F080E08F930E94FF
:10D2600020230F900F900F900F900F9082E04FC0EF
:10D2700080914F0710924F07882341F20E94624A23
:10D2800080916707882311F2EC96E2E10C9425F077
:10D2900080914F0710924F07882389F210926507FB
:10D2A0000E94DEDC80916707882349F2EDCF84FF7E
:10D2B0002DC01130D9F6809168078130D1F080916E
:10D2C0006A01882309F4FEC0BF92AF929F928F92A9
:10D2D0000F9381E090916807913009F080E08F937F
:10D2E0000E9420230F900F900F900F900F900F909F
:10D2F000BDCF80914F0710924F07882301F30E9402
:10D300005D1D809167078823D1F2BECF81E09091A7
:10D310006A01992309F4D7C0582ED12CC12C412E73
:10D320004318852DE090FB03F090FC03CE14DF043E
:10D3300008F0C9C05112A5C091E0E91AF108EC1833
:10D34000FD088EED92E10E94AC248BE1EEEDF2E15E
:10D35000DE01919601900D928A95E1F7F12CBE01C4
:10D360006F5F7F4FCE0181960E9485D918167CF49D
:10D37000CE0101960E94F8D3882389F3EF106BC089
:10D38000BE016F5F7F4F8AE797E00E9413D4CE0102
:10D3900081960E947C268091C9149091680785FF30
:10D3A00075C0911363C080914F0710924F07882377
:10D3B00009F45CC019821C828091E11269EF72E16C
:10D3C000882311F06EED72E121E04AE757E0CE01CB
:10D3D00001960E948126882309F43FC08BE1FE015B
:10D3E0003196AEEDB2E101900D928A95E1F7809110
:10D3F000C9148F7B8093C914A091BF14AA3080F404
:10D4000081E08A0F8093BF148BE18A9FD0011124A1
:10D41000AF54BC4EEEEDF2E101900D928A95E1F72A
:10D42000CE0101960E947C261092650782E090E072
:10D43000A0E0B0E080936A0790936B07A0936C071D
:10D44000B0936D0781E0809367071092FA0383E041
:10D4500080936A0119CFF39482CF0E94AE896AE764
:10D4600077E085E795E00E94D3D3DACF80916A0117
:10D47000882339F081E0911380E041E0642D0E941F
:10D48000E5CA8FEFC81AD80A53944BCF911759F0B9
:10D4900080916A018823A9F381E090916807911334
:10D4A00080E040E0EBCF80914F0710924F07882338
:10D4B00079F383E896E50E94B1CB809167078823D2
:10D4C00039F3E2CE82E01F5F9CAD911399CE809339
:10D4D0006607DACEFC01A081B1811C92A281B381E2
:10D4E0008C918F5F8C930280F381E02D90818CE092
:10D4F000989F800D1124E3E7F3E113AE84AF089504
:10D50000FC0184910895FC0180810895009751F0F9
:10D51000FC0180E09191992331F0907C9038D1F317
:10D520008F5FF8CF80E00895119800C087FD43C059
:10D53000419800C0119A00C000C0119800C086FD3B
:10D5400046C0419800C0119A00C000C0119800C0A8
:10D5500085FD3BC0419800C0119A00C000C01198E1
:10D5600000C084FD30C0419800C0119A00C000C0C6
:10D57000119800C083FD25C0419800C0119A00C0D9
:10D5800000C0119800C082FD1AC0419800C0119AD5
:10D5900000C000C0119800C081FD0FC0419800C0BC
:10D5A000119A00C000C0119800C0419800C0119AA3
:10D5B00000C000C00895419ABCCF419AF0CF419A73
:10D5C000E5CF419ADACF419ACFCF419AC4CF419A61
:10D5D000B9CF90E080E00895CF93DF93DB01F901AC
:10D5E0009C919130C1F0943080F094509C9388309D
:10D5F000D1F480819181009771F0019791838083AC
:10D60000480F591FEA01188206C08C3539F49C5F17
:10D610009C93943041F4DF91CF9108958B3339F787
:10D6200081E08C93F8CF20813181B9016F5F7F4F0A
:10D6300071836083420F531FEA0188838081918147
:10D640008F3591056CF7E7CF0F931F9381E0009121
:10D65000C5141091C6142091C7143091C81440917C
:10D66000C1145091C2146091C3147091C414041772
:10D6700015072607370708F480E01F910F910895DA
:10D6800090E080E0089520911206833021F425FD7A
:10D690000CC024FD0CC030E0A90102C0559547958F
:10D6A0008A95E2F7CA018170089581E0089580E0CB
:10D6B000089580912E0684FD0BC08091300687FD71
:10D6C00007C090913106937081E019F480E00895CD
:10D6D00081E008952FEB280F2A3108F047C0E22F90
:10D6E000F0E080912E0690912F06A0913006B09127
:10D6F000310604C0B695A795979587952A95D2F7D8
:10D7000080FD02C081700895EC5EF94FE081EE2348
:10D7100041F18091890790918A07E80FF92FF11D57
:10D72000808190ED980F9A3030F08E3251F48181E3
:10D7300080538A3098F4F0930306E093020681E068
:10D7400008958D3211F08B3249F4818190ED980F5C
:10D750009A3088F38E3211F48281EACFF0E0E0E073
:10D76000EACF1092030610920206E9CF80E00895F6
:10D77000CF93DF9385E4AEDF882309F188E0409101
:10D780002E0650912F066091300670913106972F2A
:10D790009170C92F90E0D92FCC0FDD1F71FB22278C
:10D7A00020F930E0220F331F220F331FC22B67FBFB
:10D7B000442740F9C42B8C2BDF91CF91089580E052
:10D7C000DECF88DF882341F081E02091020630918E
:10D7D0000306232B09F480E00895CF93DF93C091D3
:10D7E0003407D0913507209729F160913007709167
:10D7F000310780913207909133070E9420F16E5FCC
:10D800007F4F24976C177D07ACF47093940360935B
:10D8100093030E94D9CF605A75418F4F9F4F6093F9
:10D820009503709396038093970390939803DF91E9
:10D83000CF9108951092950310929603109297033A
:10D8400010929803F4CFB0E0A0E0E9E2FCE60C947B
:10D8500012F06B01E9014A3009F4D5C0453109F0F5
:10D8600081C0DB011296ED91FC91F2809681878157
:10D87000139A00C00000E6E2F0E03197F0F7092FBC
:10D88000182FEF2CE29420EFE22230E1B32EBF0CF0
:10D89000E80188EF49DE00C0000086E290E00197D1
:10D8A000F0F7BFE1BF1508F49BC08F2D807780682B
:10D8B0003BDE8E2D39DE00C0000086E290E001974D
:10D8C000F0F780E831DE80E02FDE00C0000086E265
:10D8D00090E00197F0F78AEF27DE00C0000086E2B3
:10D8E00090E00197F0F7005F1F4F8881807F1CDE7A
:10D8F00089918295807F18DEC017D107B1F700C0EB
:10D90000000086E290E00197F0F7F394E0E1EE0E7C
:10D91000FB10BECF1398D6011296ED91FC91808139
:10D920009281980F92832181921708F09FC1948170
:10D930009F5F94839381890F821710F08FEF820F7E
:10D940008383458150E0440F551F70E060E086817D
:10D9500097810E9440F281E0CDB7DEB7E9E00C94F8
:10D960002EF0DEC1FB0102811381423309F485C12F
:10D9700008F48DC1463409F475C1473409F482C1F5
:10D980004B3349F789812B81D80112967C911297EC
:10D9900013963C91213009F4BFC1233009F0A0C196
:10D9A00048EF480F582F91E0341708F490E031E029
:10D9B000541708F030E0492F432B61E0571708F463
:10D9C00060E0462311F4932331F2FA8030E0F9014C
:10D9D000E25BFD4FD080265B3D4FF901E08099C1AD
:10D9E00080EE8F0D8068807F9FDD8F2D8295807FF8
:10D9F0009BDD00C0000086E290E00197F0F780E830
:10DA000093DD80E861CF0B9A1398399A4198099A6F
:10DA1000119A139A00C0000086E290E00197F0F797
:10DA200088E790E0CEE9DFE0FE013197F1F701975A
:10DA3000D9F788EF79DD00C0000086E290E0019719
:10DA4000F0F780E271DD80E06FDD00C0000086E26B
:10DA500090E00197F0F780E067DD80E865DD00C0C9
:10DA6000000086E290E00197F0F780E05DDD80E164
:10DA70005BDD00C0000086E290E00197F0F7CE0188
:10DA80000197F1F7CE010197F1F7CE010197F1F778
:10DA9000CE010197F1F7CE010197F1F7CE01019781
:10DAA000F1F7CE010197F1F7CE010197F1F7CE0121
:10DAB0000197F1F7CE010197F1F7CE010197F1F748
:10DAC000CE010197F1F7CE010197F1F7CE01019751
:10DAD000F1F72197F1F780E227DD80E425DD00C032
:10DAE000000086E290E00197F0F780E21DDD80E61D
:10DAF0001BDD00C0000086E290E00197F0F7D0E067
:10DB0000C0E08C2F807780680FDD8D2F0DDD00C089
:10DB1000000086E290E00197F0F780E805DD80E004
:10DB200003DD00C0000086E290E00197F0F78AEF85
:10DB3000FBDC00C0000086E290E00197F0F780E295
:10DB4000119800C0419800C0119A00C000C01198FF
:10DB500000C0419800C0119A00C000C0119800C0D8
:10DB6000419800C0119A00C000C0119800C04198AF
:10DB700000C0119A00C000C0119800C0419800C0B8
:10DB8000119A00C000C0119800C0419800C0119ABD
:10DB900000C000C0119800C0419800C0119A00C098
:10DBA00000C0119800C0419800C0119A00C000C088
:10DBB000119800C0419800C0119A00C000C011988F
:10DBC00000C0419800C0119A00C000C0119800C068
:10DBD000419800C0119A00C000C0119800C041983F
:10DBE00000C0119A00C000C0119800C0419800C048
:10DBF000119A00C000C0119800C0419800C0119A4D
:10DC000000C000C0119800C0419800C0119A00C027
:10DC100000C0119800C0419800C0119A00C000C017
:10DC200000C00000E6E2F0E03197F0F7815009F023
:10DC300087CF88EF79DC00C0000086E290E0019792
:10DC4000F0F7CF5FD05FC03209F05BCF80E06CDCD3
:10DC500080EC6ADC00C0000086E290E00197F0F7FB
:10DC6000139879CEF8018581888375CE80E0CDB791
:10DC7000DEB7E9E00C942EF053C0B901C8010E9450
:10DC8000D7D069CED80111968C91888364CE443167
:10DC900091F0473109F05FCE1882D80112968C912D
:10DCA0001297898315968C91159781508A831396C4
:10DCB0008C918B8350CED80115964C91159750E0DE
:10DCC000440F551F70E060E016968D919C910E9464
:10DCD00040F2F801128280818150838314823BCE0E
:10DCE000381708F438CE871708F435CEFA80E12CBF
:10DCF000D12C243070F46ACEBE01C8010E94D7D066
:10DD0000898198819D0D98838E0D8983FF0C09F47C
:10DD100022CEF7FEF6CFF0CF58E0580F482F43CE73
:10DD2000EF92FF920F931F93CF93DF93EC018B0140
:10DD30007A018A859B858617970731F088819981BA
:10DD40000E94C4D21B870A87B701888199810E94EB
:10DD50001DCB2E813F81820F932F911D9F838E8338
:10DD600090E080E0CDB7DEB7E6E00C9431F0B0E0B3
:10DD7000A0E0EDEBFEE60C9411F0EC017B018A01D2
:10DD80008A859B858617970731F0888199810E9443
:10DD9000C4D2FB86EA8688859985019609F5CC80F0
:10DDA000DA808E81D80EA880B980D5015596ED9184
:10DDB000FC91C5010995C80E780110E0F701219189
:10DDC0007F0121111FC08E819F81810F911D9F8333
:10DDD0008E8390E080E0CDB7DEB7EAE00C942DF0C2
:10DDE000EE80FF80B801888199810E941DCB8E0D45
:10DDF0009F2D911D288539852817390780F681E0E8
:10DE000090E0E9CF4C2D6D2DC5010E941CD3D80E9A
:10DE1000180FD4CFB0E0A0E0E0E1FFE60C9414F0DE
:10DE2000EC01D62E1CAD0BAD7C0184E0E80EF11C9C
:10DE3000E98DFA8DC7010995412F480F2D2D602FCF
:10DE4000C7010E941CD39BAD890F8BAF81E090E08E
:10DE5000CDB7DEB7E7E00C9430F0682F70E090E0CB
:10DE600080E00C943AB280910206909103060097EC
:10DE700031F04AE050E070E060E00C9444E760E08C
:10DE800070E0CB01089580910206909103060097FF
:10DE900031F04AE050E070E060E00C9417E660E09A
:10DEA00070E0CB010895EFDF97FD0AC0ECDF6F3F14
:10DEB00071058105910509F02CF4E5DF862F0895A1
:10DEC00080E008958FEF0895CF93C62F7ADC8823E2
:10DED00011F0E9DFC82F8C2FCF91089580910206B1
:10DEE00090910306892B39F0DEDF91E0811101C0AA
:10DEF00090E0892F089591E0FCCFCF93DF93C82F56
:10DF0000D62F5FDC882321F0E9DFDF91CF910895E0
:10DF10008C2FE0DB8111F9CF8D2FF7CFB4DFCB0150
:10DF20000895CF93DF93EB014CDC882311F0F6DFEB
:10DF3000EC01CE01DF91CF9108950F931F93CF9302
:10DF400080910206909103060097D9F0FC018F01A1
:10DF5000C1912C2F2F7D81F0C53411F0C536B9F752
:10DF6000F801108270E060E00E94C1E4F801C08313
:10DF7000CF911F910F91089570E060E00E94C1E47D
:10DF8000F7CF60E070E0CB01F3CFCF92DF92EF925A
:10DF9000FF926A017B0115DC882319F0CEDF6B014B
:10DFA0007C01C701B601FF90EF90DF90CF900895FC
:10DFB000CF9380913E06811154C01092AE131092FF
:10DFC000AF131092B01310927C1310927B13109227
:10DFD0007E1310927D131092801381E080937F1343
:10DFE00082E2809381131092861310928513EAE9DE
:10DFF000F3E128EA33E18FEF81932E173F07E1F732
:10E00000C1E0C09397132EE630EB30938D1320932D
:10E010008C13C0938E1310928F131092901390E470
:10E0200090939113109292132DE630EB3093A91335
:10E030002093A81327E531E030937A1320937913C6
:10E040009EE190939E1391E190939F139CE1909396
:10E050009C1380939B1380939A130E9416D1C093B4
:10E060003E0681E080933D0685E492E29093A11202
:10E070008093A0121092A3121092A21253985B9A4E
:10E0800052985A9A3898409A0E94D06410929602F8
:10E09000CF910895FC0180E0309749F09491992345
:10E0A00031F0907C903809F08F5F3196F7CF08956A
:10E0B000B0E0A0E0EEE5F0E70C9411F0EC015B01BC
:10E0C0008A01FB01099587FD10C0C82ED12CF12CC7
:10E0D000E12C2196F801C082D182E282F382CE0146
:10E0E000CDB7DEB7EAE00C942DF0982F907E903CEF
:10E0F000A9F48F7190E0B0E0A0E06C017D0156E0E2
:10E10000CC0CDD1CEE1CFF1C5A95D1F7CE010196FC
:10E11000F50109958F73C82A2296DCCF982F907F3E
:10E12000903E11F58F7090E0B0E0A0E06C017D01B1
:10E1300036E0CC0CDD1CEE1CFF1C3A95D1F7CE016D
:10E140000196F50109958F73C82A46E0CC0CDD1CB9
:10E15000EE1CFF1C4A95D1F7CE010296F5010995F8
:10E160008F73C82A2396B6CF982F987F903F79F562
:10E17000877090E0B0E0A0E06C017D0186E0CC0CFF
:10E18000DD1CEE1CFF1C8A95D1F7CE010196F5012E
:10E1900009958F73C82A96E0CC0CDD1CEE1CFF1C81
:10E1A0009A95D1F7CE010296F50109958F73C82A89
:10E1B00026E0CC0CDD1CEE1CFF1C2A95D1F7CE010D
:10E1C0000396F50109958F73C82A249683CF982F5B
:10E1D000907C903841F4807C803869F42196CE019F
:10E1E000F5010995F8CF8E7F8D3F28F02196CE015D
:10E1F000F5010995F8CFC12CD12C76016BCF9CE0AD
:10E20000899F802D112491E0980F90933C062CE07B
:10E21000280F2093730730E02E5F3F4F4091AB13E0
:10E220004217130619F014F080E008952091AD1301
:10E230009217D0F7662341F08E5F0E94FBD1809148
:10E2400073078E5F0E94FBD1809173079091AB138F
:10E25000891750F32091AD1390913C06291720F3B4
:10E260001092AE138093AF1381E0089520913B0686
:10E27000022E000C330B8217130641F080933B06ED
:10E2800060EB73E287E793E10C94C4D20895ACE0AD
:10E29000B0E0EDE4F1E70C9413F06F3F71058105F8
:10E2A000910509F070F483E793E1B4DDE0917B130D
:10E2B000F0917C133196849190E02C96E8E00C94D8
:10E2C0002FF0F090AE13E090AF1320913D06211196
:10E2D0000FC047E152E26E2D8F2D0E9475D390E062
:10E2E00080E0F80EF092AE13E092AF139927E5CFDD
:10E2F000C0907B13D0907C1327E733E13A832983C6
:10E300002F2D30E03C832B832E2D30E03E832D8358
:10E3100018861F822FEF3FEF3A8729871C861B86BE
:10E3200007EB1EE69E012F5F3F4FAB01BC01C6010C
:10E330000E947CB1B60187E793E10E94C4D28F812D
:10E340009885CFCF4F925F926F927F928F929F92DC
:10E35000BF92CF92DF92EF92FF920F931F93CF93D2
:10E36000DF93CDB7DEB728970FB6F894DEBF0FBEA8
:10E37000CDBF7C016A014901FB0190818CE0989F2F
:10E38000800D1124982FF7012081822F880F820F92
:10E39000880F8093AE139093AF134115510559F137
:10E3A000FA82E9827C836B8301111EC0AE014B5F50
:10E3B0005F4FB401C6017CDE6C016D817E818F816F
:10E3C00098856115710581059105A9F060DFF70158
:10E3D00080818F5F8083853148F3CE0101967AD8A2
:10E3E000E5CFB12C860129C08A01B12C26C0452871
:10E3F00046284728B1F728960FB6F894DEBF0FBE1F
:10E40000CDBFDF91CF911F910F91FF90EF90DF90E3
:10E41000CF90BF909F908F907F906F905F904F9024
:10E420000895B39407C0B1102DC001151105C9F2AC
:10E430000F5F1F4F01151105A9F2AE014B5F5F4F32
:10E44000B401C60135DE6C014D805E806F8078843A
:10E450004114510461047104A9F0F0E24F16510413
:10E460006104710401F3D301C2018D97A109B109BF
:10E470000297A105B10530F04BE244165104610446
:10E48000710479F6F7018081482F4B0D5527551FF0
:10E49000463151052CF0853018F0CE0101961AD87E
:10E4A00081E0411451046104710409F480E0B80E64
:10E4B000F70180818B0D8083BB2009F498CFBA943B
:10E4C000AE014B5F5F4FB401C801F2DD8C016D817D
:10E4D0007E818F819885DBDEEFCFCF93DF93FC01C8
:10E4E00025AD211104C021E025AF0E9416D1C091B5
:10E4F0007913D0917A13E091A813F091A91382E0D7
:10E500000995E091A813F091A91381E0099530E0F5
:10E5100020E044E1BE0187E793E10E9411D12AEA9D
:10E5200033E147E1BE0187E793E10E9411D1E09119
:10E53000A813F091A91380E00995DF91CF91089578
:10E54000ACE0B0E0E6EAF2E70C9413F0F090AE1322
:10E55000E090AF1320913D06211112C047EF51E228
:10E560006E2D8F2D0E9475D390E080E0F80EF09212
:10E57000AE13E092AF1399272C96E8E00C942FF09D
:10E58000C0907B13D0907C1327E733E13A83298333
:10E590002F2D30E03C832B832E2D30E03E832D83C6
:10E5A00018861F827A8769871C861B8607EB1EE602
:10E5B0009E012F5F3F4F40E85AE6BC01C6010E9412
:10E5C00011B2B60187E793E10E94C4D28F8198858A
:10E5D000CDCFA4E0B0E0EFEEF2E70C940FF07C01B9
:10E5E000062F5A01122F862F660F990B9C012A5B6A
:10E5F0003D4F690186E0882E912C11160CF03DC02C
:10E60000AE014F5F5F4F60E87AE6C70151DD7C01E4
:10E6100069817A818B819C816115710581059105E4
:10E6200061F16D3371058105910509F450C06E37B4
:10E6300071058105910509F44AC06A3271058105A9
:10E64000910501F507FF11C08BE392E20E3F11F037
:10E6500087E392E236E01302B001112471DF66E035
:10E6600070E00E94DBEF161B60C065E470E080E0A4
:10E6700090E00DDE115069F510E0812F2496ECE05A
:10E680000C942BF0643271058105910571F4A1148D
:10E69000B104D1F0E6E01E02B0011124C50150DF43
:10E6A000B4010E94DBEF161BA8CF60347105810511
:10E6B000910551F41150F6016081062E000C770B84
:10E6C000880B990BE4DD99CFE2DD115096CF07FD61
:10E6D000BBCF61E089819A81AB81BC81CD97A105D7
:10E6E000B10509F460E0600F6A30A4F01150862F84
:10E6F0006AE00E94BAEF092F682F880F770B605DE0
:10E700007F4F072E000C880B990BC1DD112309F4F4
:10E71000B3CF602F062E000C770B605D7F4F072E66
:10E72000000C880B990BB3DD1150112309F4A4CF11
:10E7300086E01802B0011124C70102DF66E070E034
:10E740000E94DBEF161B99CFE3E7F3E183AF64AFE1
:10E750006FEF7FEFCA01F4CEACE0B0E0E2EBF3E79D
:10E760000C9413F0F090AE13E090AF1320913D069F
:10E77000211112C047ED51E26E2D8F2D0E9475D3ED
:10E7800090E080E0F80EF092AE13E092AF1399277C
:10E790002C96E8E00C942FF0C0907B13D0907C1363
:10E7A00027E733E13A8329832F2D30E03C832B8305
:10E7B0002E2D30E03E832D8318861F827A8769874D
:10E7C0001C861B8607EB1EE69E012F5F3F4F43E82A
:10E7D0005AE6BC01C6010E9411B2B60187E793E177
:10E7E0000E94C4D28F819885CDCF6FEF7FEFB4CFD9
:10E7F000B0E0A0E0EEEFF3E70C9411F05C016B01E8
:10E8000049DCE82EC6010E94866AF12C03E110E083
:10E81000081B1109C5E20E151F050CF4CFE18C2F62
:10E8200090E09C012E5F3F4F4091AB1342171306BF
:10E8300009F08CF509972091AD13281719065CF1A2
:10E840004091750750917607609174071092AE134E
:10E85000C093AF1325E1C501BCDED1E0C114D104E2
:10E86000A9F06AE370E080E090E011DD0E151F056D
:10E87000A4F4C45F8091AB13C81740F02091AD138E
:10E880004C2F4950550B241715064CF4CDB7DEB765
:10E89000EAE00C942DF0D0E0E1CFDD23B9F3802F36
:10E8A000880F080F000F0093AE13C093AF1360E200
:10E8B00070E080E090E0EBDCC60197DFE7CFACE0F2
:10E8C000B0E0E5E6F4E70C940FF0982F862F6A018C
:10E8D0007901B02E692F93DC882309F487C0109149
:10E8E0003D06C701002371F1D5DBA82E80907B1374
:10E8F00090907C13111142C02FEF3FEF122F23E1B4
:10E900002A19409175075091760760917407C601E6
:10E9100060DEAA2009F46AC0B6E08B9F6001112472
:10E920006AE370E080E090E0B2DC57E0C516D10405
:10E9300008F442C060E270E080E090E0A8DCC81A11
:10E94000D90AF3CF0E94866AA82E80907B139090FC
:10E950007C13112389F2FE0133968AE0DF011D92B8
:10E960008A95E9F787E793E19A83898300E91EE6B0
:10E970009E012F5F3F4F43E85AE612C0FE013396D7
:10E980008AE0DF011D928A95E9F787E793E19A8390
:10E99000898300E91EE69E012F5F3F4F40E85AE65B
:10E9A000B701C4010E9411B2B40187E793E10E944C
:10E9B000C4D22F813885A2CF40917307212F30E038
:10E9C000A6E0AA9EC00111242E5F3F4F28173907E9
:10E9D0000CF49C0180E8821B8093AE134093AF132C
:10E9E000BB2041F06FEF7FEFC701AADD2C96ECE072
:10E9F0000C942BF0C701F9DEF9CFE3E7F3E183AF25
:10EA000064AFCA01F2CE0C9497B24F925F926F92AC
:10EA10007F928F929F92BF92CF92DF92EF92FF925E
:10EA20000F931F93CF93DF93109233061092320609
:10EA30002FE320933606109235061092340610927A
:10EA40002E0610922F0610923006109231069C016D
:10EA5000F90190812F5F3F4F9032D1F39E34C9F47A
:10EA6000818190ED980F9A3020F08D3211F08B3229
:10EA700081F432969F012F5F3F4F808180538A300F
:10EA800008F46DC09F012F5F3F4F8081803209F4F1
:10EA900068C0F0938A07E09389078F010F5F1F4FCB
:10EAA000C0816AE270E0C8010E945AF2009731F01A
:10EAB000FC01319780818032E1F31182CD3421F065
:10EAC000C43511F0C734D9F5F80180810F5F1F4FAD
:10EAD0008032D1F380538A3090F5C093360690E0AF
:10EAE00080E06AE0AF014F5F5F4F689F9001699FD0
:10EAF000300D1124C901C0972081820F911D27FD7F
:10EB00009A95FA01208120532A3060F390933506BC
:10EB100080933406DF0131962C912032D9F3CD3425
:10EB200061F58E31910539F0F0F48731910519F0D6
:10EB30008C31910511F5B0933306A0933206DF9125
:10EB4000CF911F910F91FF90EF90DF90CF90BF90EA
:10EB50009F908F907F906F905F904F900895F901F4
:10EB600089CFF9018FCF8537910538F08737910527
:10EB700010F3803A13E09107F1F2809089079090AA
:10EB80008A0740E050E0BA0130E020E0C12CD12CEF
:10EB90007601C394FD013196DC91DD2309F484C034
:10EBA000D132F1F4CD34E1F480329105C9F44093CF
:10EBB0002E0650932F066093300670933106F09323
:10EBC0003306E093320663E270E0CF010E945AF20E
:10EBD000009709F4B4CFFC011082B1CFDF01DACF86
:10EBE000D154DA3108F05BC0DF011D91103291F091
:10EBF000A0EDA10FAA30E8F01E3271F4A181A0535C
:10EC0000AA30B8F02115310519F49F0121503109BE
:10EC1000B12C13C0FD01E8CF1D3211F01B3291F76A
:10EC2000A181B0EDBA0FBA3020F0AE3259F7A2810F
:10EC3000E6CFBE2EB818309759F3AD2FB0E02601BD
:10EC4000370104C0440C551C661C771CDA95D2F7BA
:10EC50004429552966297729AC5EB94FBC92A08119
:10EC6000A154AA3108F4BACFDF01D191DD2309F410
:10EC700091CF00EDB02EBD0E19E01B15A8F713EDD6
:10EC8000B12EBD0E11E01B1578F7DB3269F3FD01E3
:10EC90003196DC91D03209F07DCFDF01F8CF21151C
:10ECA0003105E9F69D01DBCF309333062093320620
:10ECB00040932E0650932F066093300670933106D2
:10ECC0003ECFFC01659175918591949108958F9245
:10ECD0009F92AF92BF92CF92DF92EF92FF92CF932B
:10ECE000DF93EC018090B1029090B202A090B30249
:10ECF000B090B40220E030E0A901C501B4010E9447
:10ED000023E9882309F452C0C880D980EA80FB80B7
:10ED1000A7019601C501B4010E9423E918160CF061
:10ED20004AC02091FE053091FF05409100065091A8
:10ED30000106C701B6010E9423E9882321F1C09290
:10ED4000FE05D092FF05E0920006F09201062091A8
:10ED5000FA053091FB054091FC055091FD05C70176
:10ED6000B6010E9488E99B01AC0160E070E080E898
:10ED70009FE30E9440F060934C0170934D0180939B
:10ED80004E0190934F0160914C0170914D01809123
:10ED90004E0190914F01DF91CF91FF90EF90DF9066
:10EDA000CF90BF90AF909F908F90089560E070E0FB
:10EDB00080E89FE3F0CF60E070E0CB01ECCFB0E003
:10EDC000A0E0E5EEF6E70C940BF0EC01209179035E
:10EDD00030917A0340917B0350917C036881798163
:10EDE0008A819B810E9440F04B015C0120917D0350
:10EDF00030917E0340917F03509180036C817D812F
:10EE00008E819F810E9440F06B017C01A5019401DD
:10EE100060914401709145018091460190914701B4
:10EE20000E9423E9882309F454C0809244019092FF
:10EE30004501A0924601B09247012091F205309120
:10EE4000F3054091F4055091F505C501B4010E9408
:10EE500088E92B013C010E9451F14B015C0120E04B
:10EE600030E040EA50E40E9423E9181634F4812C83
:10EE7000912CC0EAAC2EC0E4BC2E20E030E0A90109
:10EE8000C501B4010E94A4F187FF03C0812C912C1D
:10EE90005401A5019401C301B2010E9440F06093A6
:10EEA000EA057093EB058093EC059093ED05C501A1
:10EEB000B4010E9420F16093E805062E000C770B48
:10EEC0006F5F7F4F6630710514F066E070E060930D
:10EED000E605D09142011091E805A70196016091E5
:10EEE00048017091490180914A0190914B010E9423
:10EEF00023E9811123C0D11375C02091CE05309133
:10EF0000CF054091D0055091D1056091EA057091EF
:10EF1000EB058091EC059091ED050E9488E9209128
:10EF2000D2053091D3054091D4055091D5050E946A
:10EF300041F0CDB7DEB7E0E10C9427F0C092480174
:10EF4000D0924901E0924A01F0924B012091F605DE
:10EF50003091F7054091F8055091F905C701B601C8
:10EF60000E9488E94B015C010E9451F16B017C0118
:10EF700020E030E040EA50E40E9423E9181634F41F
:10EF8000C12CD12CB0EAEB2EB0E4FB2E20E030E017
:10EF9000A901C701B6010E94A4F187FF03C0C12CDB
:10EFA000D12C7601A7019601C501B4010E9440F061
:10EFB0006093EE057093EF058093F0059093F10553
:10EFC000C701B6010E9420F16093E905062E000CEE
:10EFD000770B6F5F7F4F6630710514F066E070E06D
:10EFE0006093E705C091E905D11305C08091430105
:10EFF0008C1709F470C08091E8059091E905909311
:10F000004301809342010C2E000CDD0B27E012031C
:10F01000C0011124FC01EC0FFD1FEE0FFF1FEE0FCE
:10F02000FF1FEB54FD4F208131814281538120939A
:10F03000E2053093E3054093E4055093E505009124
:10F04000E705002E000C110BFC01E00FF11FEE0F85
:10F05000FF1FEE0FFF1FEB54FD4F60817181828116
:10F0600093810E9440F06093DE057093DF058093EA
:10F07000E0059093E1052091E60537E02303F001D8
:10F080001124CE0FDF1FCC0FDD1FCC0FDD1FCB54A3
:10F09000DD4F288139814A815B812093DA053093E5
:10F0A000DB054093DC055093DD05E00FF11FEE0F0B
:10F0B000FF1FEE0FFF1FEB54FD4F608171818281B6
:10F0C00093810E9440F06093D6057093D70580939A
:10F0D000D8059093D9058090EE059090EF05A0900B
:10F0E000F005B090F1052091DE053091DF054091EB
:10F0F000E0055091E105C501B4010E9488E9209125
:10F10000E2053091E3054091E4055091E5050E9448
:10F1100041F06B017C01C092D205D092D305E09200
:10F12000D405F092D5052091D6053091D7054091B0
:10F13000D8055091D905C501B4010E9488E92091F4
:10F14000DA053091DB054091DC055091DD050E9428
:10F1500041F0A70196010E9440F06093CE057093A4
:10F16000CF058093D0059093D105C7CEACE0B0E039
:10F17000ECEBF8E70C9418F0182F882379F020E0D6
:10F1800030E0A90160918103709182038091830333
:10F19000909184030E9423E98823F1F08091B002CA
:10F1A0008117D1F00E94822C8CE0EAE3F2E0DE01CC
:10F1B000119601900D928A95E1F7CE010196FFDD3F
:10F1C0008091B002882361F085E791E00E94D82CFD
:10F1D0001092B0020E947D3F2C96E3E00C9434F034
:10F1E00081E08093B00285E791E00E94A42CF2CFE9
:10F1F000CF92DF92EF92FF9280E0B8DF10927D0312
:10F2000010927E0310927F03109280031092790374
:10F2100010927A0310927B0310927C031092850364
:10F220001092860310928703109288031092810334
:10F2300010928203109283031092840345EB52E0F4
:10F2400027E0C12CD12C60ECE62E6FE7F62E90E083
:10F2500080E0FC01EE0FFF1FEE0FFF1FE40FF51F14
:10F26000C082D182E282F38201968730910589F7CC
:10F270002150445E5F4F2111EACFFF90EF90DF9065
:10F28000CF9008954F925F926F927F928F929F924C
:10F29000AF92BF92CF92DF92EF92FF921F93CF93E4
:10F2A000DF93EC01162F2091B1023091B202409110
:10F2B000B3025091B402688179818A819B810E9456
:10F2C00023E9882309F497C0B090B00280E04EDFB4
:10F2D000C880D980EA80FB8020E030E0A901C70126
:10F2E000B6010E94A4F187FF03C0C12CD12C760186
:10F2F000C092B102D092B202E092B302F092B40294
:10F300002DEB37E346E855EBC701B6010E9423E930
:10F3100087FD0BC02DEB37E346E855E3C701B60187
:10F320000E94A4F118160CF076C0A701960160E0C7
:10F3300070E080E89FE30E94B8F06093FA05709354
:10F34000FB058093FC059093FD0580EF9FEFA9E7F7
:10F35000B4EC8093FE059093FF05A0930006B09354
:10F360000106BB2009F447C040907501509076011A
:10F3700060907701709078018090790190907A0187
:10F38000A0907B01B0907C01C0907D01D0907E0167
:10F39000E0907F01F090800181E0E8DE112359F1D7
:10F3A000A3019201609175017091760180917701BE
:10F3B000909178010E9423E981111BC0A50194015D
:10F3C0006091790170917A0180917B0190917C012B
:10F3D0000E9423E981110DC020917D0130917E01B1
:10F3E00040917F0150918001C701B6010E9423E93D
:10F3F00081110E94CB3FDF91CF911F91FF90EF9041
:10F40000DF90CF90BF90AF909F908F907F906F9044
:10F410005F904F90089560E070E0CB018ECF8F92A7
:10F420009F92AF92BF92CF92DF92EF92FF92C090E5
:10F430008103D0908203E0908303F090840320E066
:10F4400030E0A901C701B6010E9423E98823E1F158
:10F45000A701960160E070E080E89FE30E94B8F0A9
:10F460006B017C018090850390908603A0908703B8
:10F47000B090880320E030E0A901C501B4010E94EA
:10F4800023E9882329F1A501940160E070E080E878
:10F490009FE30E94B8F0C092F205D092F305E0928B
:10F4A000F405F092F5056093F6057093F7058093E7
:10F4B000F8059093F905FF90EF90DF90CF90BF9003
:10F4C000AF909F908F900895C12CD12C7601CACF18
:10F4D00060E070E0CB01DFCFCF92DF92EF92FF923E
:10F4E0006B017C0183E3C816D104E104F10470F0E0
:10F4F00082E3C81AD108E108F10862E370E080E015
:10F5000090E00E9450CF0E94C429ECCFC701B60101
:10F510000E9450CF0E94C429FF90EF90DF90CF90BF
:10F520000895BC0190E080E00C943AB28091870786
:10F53000813069F09091C91492FB882780F992FF7D
:10F5400007C097FB882780F991E08927089581E01B
:10F5500008959091C91494FB882780F994FF06C000
:10F5600081E09091C612911101C080E00895A4E05D
:10F57000B0E0EDEBFAE70C940BF01092720780917B
:10F580004F0710924F07882361F020E040E070E0C1
:10F5900060E081E792E60E9494452496E0E10C94B5
:10F5A00027F0209112013091130140916A07509188
:10F5B0006B07CA01820F931F2436310509F01DC461
:10F5C0004730510544F006978A3091050CF024C469
:10F5D0008AE090E02BC406964A3F5F4FACF38091DF
:10F5E0006907882309F4C8C16091B2127091B312FF
:10F5F000072E000C880B990B0E9429E9B1E0B98312
:10F600002091AE123091AF124091B0125091B112D0
:10F610000E94A4F118160CF01982609134077091C1
:10F620003507072E000C880B990B0E9429E92091C1
:10F6300030073091310740913207509133070E94D3
:10F64000A4F118161CF4E981E260E983C980C09234
:10F650006E06C0907501D0907601E0907701F09031
:10F6600078018091790190917A01A0917B01B0910C
:10F670007C0189839A83AB83BC8380907D019090C9
:10F680007E01A0907F01B090800120E030E04AE749
:10F6900054E4C501B4010E9488E92B013C0120E03B
:10F6A00030E0A901C501B4010E9423E920E030E067
:10F6B00040EA50EC87FD04C020E030E040EA50E42E
:10F6C000C301B2010E9441F02DEC3CEC4CEC5DE337
:10F6D0000E9488E90E9420F14B015C0180E2B7FEA4
:10F6E00009C0B094A09490948094811C911CA11C9A
:10F6F000B11C8DE28093980260E290E1891697E256
:10F700009906A104B1048CF0C501B40120E137E2EF
:10F7100040E050E00E9473EFCA01B9012AE030E0F6
:10F7200040E050E00E9473EF605D6093990260E2F8
:10F73000A8EE8A16A3E09A06A104B1048CF0C501D4
:10F74000B40128EE33E040E050E00E9473EFCA01BC
:10F75000B9012AE030E040E050E00E9473EF605DC4
:10F7600060939A02C501B40124E630E040E050E025
:10F770000E9473EF6AE0462E512C612C712CCA0155
:10F78000B901A30192010E9473EF605D60939B0237
:10F79000C501B401A30192010E9473EF4B01CA019C
:10F7A000B901A30192010E9473EF882009F44EC3AE
:10F7B0002EE220939C02605D60939D02B0E38B0E6D
:10F7C00080929E0268E972E086E696E00E9465F209
:10F7D00020E030E0A901C701B6010E9423E920E042
:10F7E00030E040E05FEB87FD04C020E030E040E027
:10F7F0005FE3C701B6010E9441F00E9420F1CB01F6
:10F800000E947444BC0181E696E00E9465F220E00B
:10F8100030E0A90169817A818B819C810E9423E972
:10F8200020E030E040E05FEB87FD04C020E030E006
:10F8300040E05FE369817A818B819C810E9441F085
:10F840000E9420F1CB010E947444BC018CE596E03B
:10F850000E9465F28091C91483FD0AC37ADE882371
:10F8600009F409C38091C1149091C214A091C314EA
:10F87000B091C4140097A105B10509F4FCC2BC0104
:10F88000CD016D597F4F8F4F9F4F24E630E040E010
:10F8900050E00E9451EF6091C5147091C6148091A0
:10F8A000C7149091C8140E9451EF29830E94B3435A
:10F8B0004B015C01162F80915E01C9808C15C1F04F
:10F8C000C0925E0128E4C29EB001112490E080E065
:10F8D0000E9427E92AE037ED43E25CE30E9488E9D1
:10F8E0000E9425F160935B06C110C7C210925606B4
:10F8F00080915D01181709F43FC080925D01C50138
:10F90000B40120E13EE040E050E00E9451EF690187
:10F9100089019CE3492E512C612C712CC501B40145
:10F92000A30192010E9451EF4B015C01CA01B90190
:10F93000A30192010E9451EFC114D10409F0C4C285
:10F940009F928F927F936F938BE592E29F938F9319
:10F9500086E496E09F938F930E94BCE80FB6F894DC
:10F96000DEBF0FBECDBF85E0982F990F990F891B81
:10F97000880F8058809345060E94D9CF0091400699
:10F980001091410620914206309143066B017C01A3
:10F99000C01AD10AE20AF30A9701860137FD11C0A5
:10F9A00020913F06209520933F066A547C4F8F4F4D
:10F9B0009F4F609340067093410680934206909358
:10F9C0004306D0903F06D98281E00E943671809133
:10F9D000AB13873180F48091AD13843060F08EE3F7
:10F9E000E82E83E2F82E03E126E044E064E087E7B6
:10F9F00093E10E949AD380916E06982F927048E00E
:10FA00000CE081FD02C042E102E08091AB13843141
:10FA100080F48091AD13841760F0992309F473C2C8
:10FA20008AE193E27C0123E060E587E793E10E94AD
:10FA30009AD38091AB138431C0F48091AD1382309E
:10FA4000A0F0C980CC2009F461C28091A707882367
:10FA500009F45CC28EED92E27C0102E123E042E017
:10FA600068E687E793E10E949AD38091AB138C31CB
:10FA700008F09DC08090AE129090AF12A090B0128E
:10FA8000B090B112C090B212D090B312843198F4F9
:10FA90008091AD13883078F080916E0680FF39C276
:10FAA00080E992E27C010CE022E048E069E387E72C
:10FAB00093E10E949AD38091AB13883040F4D7FE33
:10FAC0002BC244E752E267E087E30E94A47380916F
:10FAD000AB138C31B0F48091AD13843190F020E001
:10FAE00030E040E05FE3C501B4010E9441F00E94B4
:10FAF00020F177FF34C244E752E26CE187E30E94D1
:10FB0000A473C0903007D0903107E0903207F09096
:10FB100033078091AB13883060F480913407909163
:10FB2000350797FF3FC244E752E267E081E50E9454
:10FB3000A4738091AB138C31B0F48091AD138431F8
:10FB400090F020E030E040E05FE3C701B6010E94A2
:10FB500041F00E9420F177FF47C244E752E26CE196
:10FB600081E50E94A4738091AB138C3100F58091E4
:10FB7000AD138431E0F08091A7078823C1F024E61B
:10FB8000829FC001112481589F4F6FEF70E00E9447
:10FB9000DBEFCB010E94F344AC016CE187E60E94ED
:10FBA000FD7465E270E080E090E00E944771D1DC76
:10FBB000882379F18091AB13843358F58091AD138C
:10FBC0008A3238F107E028E04AE26AE287E793E107
:10FBD0000E9441D205E022E04CE262E387E793E134
:10FBE0000E9441D224E04AE061E38AE20E9411D2FD
:10FBF0006091791370917A1382E3809393138BE26F
:10FC00008093941323E933E142E387E793E10E9471
:10FC100011D18091AB13853350F48091AD138133B2
:10FC200030F024E04AE461E386E30E9411D280913F
:10FC3000AB13843368F48091AD13823348F002E053
:10FC400020915B0642E367E387E793E10E9441D29C
:10FC50008091AB138033D8F48091AD138832B8F023
:10FC600080915606882361F046E556E060E387E31D
:10FC70000E94FD7465E270E080E090E00E944771B0
:10FC800046E456E060E3809145060E94FD74809151
:10FC9000AB13883208F060C08091AD138D3108F449
:10FCA0005BC02BE040E86DE180E00E9411D28091C2
:10FCB000AB13873208F050C08091AD138F3108F438
:10FCC0004BC083E08093AE1316E21093AF1368E548
:10FCD00070E080E090E00E9447718BE08093AE136B
:10FCE0001093AF13C980CC2009F4A1C181E696E03E
:10FCF0000E94F57388E28093AE1316E21093AF135F
:10FD000069E570E080E090E00E94477180E38093B5
:10FD1000AE131093AF13C980CC2009F4ABC18CE5AE
:10FD200096E00E94F5738DE48093AE1316E2109373
:10FD3000AF136AE570E080E090E00E94477185E5CE
:10FD40008093AE131093AF13C980CC2009F4B5C1D2
:10FD500086E696E00E94F5738091AB13833338F505
:10FD60008091AD138B3218F183E00E94367183E0ED
:10FD70008093AE1383E38093AF1366E070E080E07E
:10FD800090E00E94477181E00E94367180911201DB
:10FD9000909113010E94F344AC0163E38CE00E9454
:10FDA000FD7465E270E080E090E00E944771809110
:10FDB000AB13813408F0F1CB8091AD13863308F496
:10FDC000ECCB1092AE138EE38093AF138FE390E1F0
:10FDD0000E94866A182F863108F092C18FE390E165
:10FDE0000E94F573153109F4D8CB60E270E080E031
:10FDF00090E00E9447711F5FF5CF243631054CF427
:10FE00008536910504F58A30910534F48AE090E056
:10FE100009C084369105BCF0883EA3E09A0714F02F
:10FE200087EE93E02817390709F4D9CB9093130193
:10FE30008093120110926A0710926B0710926C0760
:10FE400010926D07CCCB84E690E0F0CF662351F0A2
:10FE50002EE220939C02605D60939D0280E280937D
:10FE60009E02B0CC80E280939D0280939C02F6CFEC
:10FE7000E4E6E9831BCD198219CD498180E244363D
:10FE800028F0842F64E60E94AEEF805D80939C0290
:10FE9000698190E26A3040F02AE0862F622F0E944A
:10FEA000AEEF0E94AEEF905D90939D0289816AE073
:10FEB0000E94AEEF905D90939E026CE972E086E541
:10FEC00096E00E9465F214CD0436110538F47F9354
:10FED0006F93DF92CF928FE492E238CD7F936F934E
:10FEE000DF92CF9285E492E29F938F9386E496E02F
:10FEF0009F938F930E94BCE80FB6F894DEBF0FBEAD
:10FF0000CDBF86E031CD84E193E28CCD88EA92E2E8
:10FF1000A3CD88E792E2C6CDC6010E94F344FC015E
:10FF2000808193E0803229F4818192E0803209F46B
:10FF300091E043E050E0491B51094E0F5F1F892FAC
:10FF4000880F880F981B892F67E0805C0E94FD74E2
:10FF500069E070E080E090E00E944771B8CDCB018D
:10FF60000E94F344FC01808193E0803229F4818176
:10FF700092E0803209F491E043E050E0491B5109DE
:10FF80004E0F5F1F892F880F880F981B892F6CE1F8
:10FF9000805C0E94FD7469E070E080E090E00E9467
:10FFA0004771AFCD0E94F344FC01808193E0803221
:10FFB00029F4818192E0803209F491E043E050E03D
:10FFC000491B51094E0F5F1F892F880F880F981BFF
:10FFD000892F67E0865A0E94FD7469E070E080E036
:10FFE00090E00E944771A5CDCB010E94F344FC0133
:10FFF000808193E0803229F4818192E0803209F49B
:020000021000EC
:1000000091E043E050E0491B51094E0F5F1F892FDB
:10001000880F880F981B892F6CE1865A0E94FD7407
:1000200069E070E080E090E00E9447719CCD87E03D
:100030000E942A3B80FF13C001E616E0D8016D91B3
:100040008D01662309F456CE6F320CF06FE3062E55
:10005000000C770B880B990B0E944771EFCF8091B2
:10006000770780FD43CE6FEF7FEF8FE692E20E942D
:10007000A07240CE87E00E942A3B81FF13C00CE5AE
:1000800016E0D8016D918D01662309F44CCE6F32D4
:100090000CF06FE3062E000C770B880B990B0E9477
:1000A0004771EFCF8091770781FD39CE6FEF7FEFFA
:1000B0008FE692E20E94A07236CE87E00E942A3B31
:1000C00082FF13C006E616E0D8016D918D0166230C
:1000D00009F442CE6F320CF06FE3062E000C770B62
:1000E000880B990B0E944771EFCF8091770782FDB3
:1000F0002FCE6FEF7FEF87E692E20E94A0722CCEA8
:1001000081E0C980C11001C080E090914406891748
:10011000C9F0D0903E10D982809344068FE390E1DD
:100120000E94866AD81608F054C029812F5F29835F
:10013000E22FF0E0E15CFF4E8081807C8038A9F303
:1001400020933E1000913E1010E0015C1F4EC8014C
:100150000E94866A898360E870E0C8010E94AC73DF
:100160004981453108F019CA60E270E080E090E012
:100170000E9447716981643109F40FCA60E270E03E
:1001800080E090E00E9447718981833109F405CABB
:1001900060E270E080E090E00E94477199819231C6
:1001A00009F4FBC9292F30E02E5F3F4F4AEF42038D
:1001B000B001439F700D112460587F4F8FE390E191
:1001C0000E94AC7360E270E080E090E00E944771B2
:1001D000E4C910923E10B6CF80918707823059F063
:1001E000B8D9882349F08091C91482FB882780F907
:1001F00091E08927089581E0089581E00895DC0168
:10020000EC918E2F90E0FC01EE0FFF1FE80FF91F1D
:10021000EA5DFC4E80818F7780830895892B79F485
:100220001092900082E080939100109295001092BD
:100230009400C19A8091710082608093710008954A
:10024000B0E0A0E0E6E2F1E80C940EF0EC017B01F6
:1002500088818C3008F0A4C090E0FC01EE0FFF1FF5
:10026000E80FF91FEA5DFC4E80818F770E94C2B4CF
:1002700019821A8288812CE0622F0E94AEEF829F41
:10028000B001112430E020E0AB01420F531FFA010E
:10029000EE0FFF1FE40FF51FEA5DFC4E908197FD06
:1002A00007C02F5F3F4F2C30310571F790E0B6DF6C
:1002B0007880072D10E06801CC0CDD1CF601E00F02
:1002C000F11FEA5DFC4E80818068808377FC68C006
:1002D00080E2E81682E0F8060CF03FC08A8128E54B
:1002E00032E0281B310987FD3395220F331F220F7F
:1002F000331F032E000C440B550B898178E8872EA1
:10030000912C881A910887FD9394880C991C880C6D
:10031000991C092C000CAA08BB0860E070E0CB0116
:10032000F7FC0AC0B701653B710514F064EB70E09F
:10033000072E000C880B990B281939094A095B090B
:100340000E9442EF24EB30E040E050E00E9473EF67
:10035000820E931EA41EB51E74018BE08715D8F083
:10036000298188E890E0821B910927FD9395880FE9
:10037000991F880F991FE816F906BCF402972FB74A
:10038000F894E601C00FD11FCA5DDC4E880F991F9B
:100390009A8389832FBF62E370E080E090E09CD86D
:1003A000CDB7DEB7EDE00C942AF02A8188E592E023
:1003B000821B910927FD9395880F991F880F991F1C
:1003C000E816F906DCF6C701D9CFCF93DF93EB012E
:1003D000682F70E08BE493E133DF688179818A8153
:1003E0009B81643F21E072078105910520F464EF51
:1003F00071E080E090E070D886B182958170DF91E5
:10040000CF910895A4E0B0E0E8E0F2E80C9419F090
:100410008EEE92E0A0E0B0E089839A83AB83BC8348
:10042000BE016F5F7F4F8AE5D0DF2496E2E00C9437
:1004300035F0A4E0B0E0EFE1F2E80C9419F08EEEB4
:1004400092E0A0E0B0E089839A83AB83BC83BE01D5
:100450006F5F7F4F8AE0B9DF2496E2E00C9435F0BD
:10046000A4E0B0E0E6E3F2E80C9419F084EF91E048
:10047000A0E0B0E089839A83AB83BC83BE016F5F49
:100480007F4F8CE3A2DF2496E2E00C9435F0A4E0E9
:10049000B0E0EDE4F2E80C9419F084EF91E0A0E014
:1004A000B0E089839A83AB83BC83BE016F5F7F4FCB
:1004B00080EA8BDF2496E2E00C9435F01F920F92D5
:1004C0000FB60F9211240BB60F922F933F934F93B9
:1004D0005F936F937F938F939F93AF93BF93EF93AC
:1004E000FF938091BF0587FF27C01092950010925F
:1004F00094008091BF058F5F8093BF058091BF05F9
:10050000082E000C990B20914A132817190629F080
:1005100024F08091BF058C30DCF1809194009091A3
:100520009500049680349C4908F47DC08091940025
:1005300090919500049679C08091BF05082E000C1B
:10054000990B20914A132817190699F294F2E09119
:10055000BF058E2FEE0F990BFC01EE0FFF1FE80F6A
:10056000F91FEA5DFC4E808187FFC3CFE091BF0594
:100570008E2FEE0F990BFC01EE0FFF1FE80FF91FF6
:10058000EA5DFC4E808160E08F770E94F4CEB1CFAF
:100590002091940030919500E091BF058E2FEE0FD1
:1005A000990BFC01EE0FFF1FE80FF91FEA5DFC4EEF
:1005B00081819281820F931F90939900809398007C
:1005C000E091BF058E2FEE0F990BFC01EE0FFF1F80
:1005D000E80FF91FEA5DFC4E808187FF11C0E091B2
:1005E000BF058E2FEE0F990BFC01EE0FFF1FE80FDA
:1005F000F91FEA5DFC4E808161E08F770E94F4CEA6
:10060000FF91EF91BF91AF919F918F917F916F91EA
:100610005F914F913F912F910F900BBE0F900FBEA6
:100620000F901F90189580E49CE990939900809317
:1006300098008FEF8093BF05E3CF9091C00095FFA6
:10064000FCCF8093C6000895CF93DF93EC0189918E
:10065000882311F0F2DFFBCFDF91CF910895CF9384
:10066000DF93EC018991882311F0E7DFFBCF8DE068
:10067000E4DF8AE0E2DFDF91CF910895CF93DF934B
:10068000EC01FE0184912196882311F0D6DFF9CF89
:10069000DF91CF9108950F931F93CF938C01C62FB5
:1006A00089EB9FE1EBDFC801E9DF8AE3C6DF80E386
:1006B0008C0FC3DF8AE0C1DFCF911F910F910895A6
:1006C000CF92DF92EF92FF926A017B01D7DF42E087
:1006D000C701B6010E94E1B4FF90EF90DF90CF9088
:1006E0000895CF93DF9360ED7FE10E942EC6C09105
:1006F0005A13D0915B13488159816A817B8187ECC1
:100700009FE1DEDF4C815D816E817F818DEC9DE21A
:10071000D7DF409156135091571360915813709141
:1007200059138AEC9DE2CCDF84EC9FE1A7DF8EEBCE
:100730009FE1A4DF8AE081DFDF91CF910895C0DFE0
:100740008AE07BCFADE5B0E0E8EAF3E80C9409F08D
:1007500070E060E085E40E94916F7C01182F8F3F6C
:10076000B1F1882341F083EB91E288DFC35ADF4F78
:10077000E2E10C9425F06EEB70E083E50E94916F4E
:100780005C0165E070E083E40E94916F6C0160E0C1
:1007900085E50E947D6F2C968FAF2C9760E086EAEE
:1007A00091E20E94805B0E94D9CF69877A878B870C
:1007B0009C871F3F09F067C434E7A316B1040CF40B
:1007C00089C18BE791E25ADF0E94B2C6CFCF6CE3BA
:1007D00070E0D3CF20E030E040E05EE32BAF3CAFF1
:1007E0004DAF5EAFABC12AE939E949E15FE323963A
:1007F0002CAF3DAF4EAF5FAF2397ADC14090AE126F
:100800005090AF126090B0127090B11251C22B96FE
:10081000EEADFFAD2B974083A4C24BEEC42ED12C7E
:10082000E12CF12C22C384E190E0A0E0B0E08D87C0
:100830009E87AF87B88B34E1C32ED12CE12CF12CED
:1008400024C3CD86DE86EF86F88A1FC32B96EEADD5
:10085000FFAD2B978083E9C3D501C4012EA53FA529
:1008600048A959A9821B930BA40BB50BB7FD47C030
:100870002D968FAD2D970E943B278AE0DEDED501B5
:10088000C4018053984FAF4FBF4F8EA79FA7A8AB0F
:10089000B9AB9AA991116FC02BA93CA94DA95EA92A
:1008A000C301B2010E94A4F118160CF050C020E060
:1008B00030E040E050E4C301B2010E9441F06BAB74
:1008C0007CAB8DAB9EAB2AA53BA54CA55DA5280DA9
:1008D000391D4A1D5B1D2FAB38AF49AF5AAF6D961E
:1008E0006CAD7DAD8EAD9FAD6D970E9429E9A301E2
:1008F00092010E9423E9881F8827881F8AAB898577
:100900009A85AB85BC85898F9A8FAB8FBC8F2989DF
:100910003A894B895C89281739074A075B0720F415
:10092000298F3A8F4B8F5C8F898D9A8DAB8DBC8DC3
:10093000881A990AAA0ABB0A91E889169FE49906BF
:1009400092E1A906B10460F18FE990E22DC2D501D0
:10095000C4012FA938AD49AD5AAD821B930BA40B2E
:10096000B50B4FEE52E16EEF72E1B7FDC8CF812FAC
:100970000E948228C4CF69966CAD7DAD8EAD9FADCF
:1009800069970E9429E99B01AC01C301B2010E9451
:1009900023E987FFB4CF4CE253E16CE373E1E7CF87
:1009A0002996AEADBFAD2997A215B3050CF08FC047
:1009B000B3E02B1631040CF48AC082E490E25EDED0
:1009C0001F3F09F066C0E2E3F0E2FE83ED8381E2BF
:1009D00090E254DE8D819E8151DE49815A816B8186
:1009E0007C818EE390E2ABDE81E290E247DE8D8196
:1009F0009E8144DE4D8D5E8D6F8D78A18AE390E2FD
:100A00009EDE81E290E23ADE8D819E8137DE49A151
:100A10005AA16BA17CA186E390E291DE2C963FADBA
:100A20002C97332309F4D0CE2CEA35EC47E25EE371
:100A30006D8D7E8D8F8D98A10E9488E96B017C0160
:100A400020E030E543EC50E469A17AA18BA19CA1A0
:100A50000E9488E929813A814B815C811F3FF1F432
:100A600020933707309338074093390750933A075C
:100A7000C0923B07D0923C07E0923D07F0923E07C0
:100A800060933F077093400780934107909342071C
:100A90009BCE2DE13DE23E832D8399CF2093B5126D
:100AA0003093B6124093B7125093B812C092B91255
:100AB000D092BA12E092BB12F092BC126093BD12B7
:100AC0007093BE128093BF129093C0127DCE0E948D
:100AD0002B66CEC087E691E2D1DD0E94E4278FE746
:100AE000809336072CE330E0C9A6A8EEB3E00E945D
:100AF0009FEF6AA77BA78CA79DA729853A854B8581
:100B00005C85260F371F481F591F2FAB38AF49AFE1
:100B10005AAF81E08093690160E083E591E20E9431
:100B2000805B02E00E0D023008F054CE8BEA9AEAA8
:100B3000AAEABEE38BAF9CAFADAFBEAF023008F008
:100B400052CE8DEC9CECACE4BEE323968CAF9DAF13
:100B5000AEAFBFAF2397023008F4E12C2D96EFAE75
:100B60002D9789859A85AB85BC85898B9A8BAB8BB4
:100B7000BC8B8EA79FA7A8ABB9AB19A21AA21BA2C8
:100B80001CA21D8E1E8E1F8E18A219821A821B8215
:100B90001C822FE730E040E050E02D873E874F87F2
:100BA000588B80E090E4ACE1B6E48D839E83AF8304
:100BB000B8871D8A1E8A1F8A188EFFE7CF2ED12C78
:100BC000E12CF12C1AAA1BAA1CAA1DAA1EAA1DA25E
:100BD0001EA21FA218A691E024969FAF2497312C45
:100BE000212C412C512C320195010B2C000C440B73
:100BF000550B61962CAF3DAF4EAF5FAF619749A5E6
:100C0000042E000C550B29965FAF4EAF299757E184
:100C10001502C0011124DC01AC54BD4E2B96BFAFB0
:100C2000AEAF2B97C5014E969C01092E000C440BCC
:100C3000550B65962CAF3DAF4EAF5FAF6597CC9728
:100C40009C01990F440B550B69962CAF3DAF4EAFED
:100C50005FAF699736E0A31AB108C5010B2C000CF1
:100C6000AA0BBB0B6D968CAF9DAFAEAFBFAF6D97B0
:100C700080916901882309F498C00E94D9CF4B0163
:100C80005C0190919A036E969FAF6E97992309F439
:100C90007BC00E945D2910929A031F3F09F0AECDE0
:100CA00040903007509031076090320770903307C2
:100CB000A30192016D897E898F89988D0E94A4F18C
:100CC00087FF04C04D8A5E8A6F8A788EA3019201E5
:100CD0006D817E818F8198850E9423E9181624F406
:100CE0004D825E826F82788661966CAD7DAD8EADF1
:100CF0009FAD61970E9429E9698F7A8F8B8F9C8FB6
:100D00002496AFAD2497AA2309F454C09B01AC01EB
:100D1000C301B2010E94A4F11816B4F5D501C401B3
:100D200029893A894B895C89821B930BA40BB50BEB
:100D3000AC01BD01485853416109710977FD24C0D8
:100D40004D855E856F8578894C195D096E097F092F
:100D500075956795579547951F3F09F058CD409376
:100D600036078DA39EA3AFA3B8A7298D3A8D4B8DCF
:100D70005C8D2D8B3E8B4F8B588F89869A86AB86E8
:100D8000BC8624961FAE249765966CAD7DAD8EAD66
:100D90009FAD65970E9429E9A30192010E9423E972
:100DA00087FF5ACD8DEB90E269DC109269010E94B9
:100DB000E4270ACD298D3A8D4B8D5C8DC301B2019C
:100DC0000E9423E987FFE0CFD501C40129853A8538
:100DD0004B855C85821B930BA40BB50BAC01BD014D
:100DE000485853416109710977FDCECF2114310470
:100DF00009F40AC12DA13EA14FA158A5280F391F02
:100E00004A1F5B1F298B3A8B4B8B5C8B2DA13EA11C
:100E10004FA158A5281B390B4A0B5B0BC701B60124
:100E20000E9442EF29893A894B895C890E9473EFBD
:100E3000CD84DE84EF84F888C20ED31EE41EF51E36
:100E400034E1C316D104E104F1040CF4ECCC4CEE13
:100E5000C416D104E104F1040CF0DFCC50E8C5164F
:100E6000D104E104F1040CF4ECCCCD86DE86EF86EF
:100E7000F88A8EEF90E0A0E0B0E09C01AD012C1963
:100E80003D094E095F0969017A018BE491E2F6DBC5
:100E90006D857E858F8598890E94037586E491E231
:100EA000EDDBC701B6010E9403754D815E816F8144
:100EB00078858FE391E204DC4D895E896F89788DB6
:100EC00088E391E2FDDB93E0291631040CF49CC029
:100ED000C701B6010E9429E920E030E040E850E473
:100EE0000E9488E969837A838B839C832D813E816C
:100EF0004F8158856D897E898F89988D0E9440F039
:100F00002BED3FE049EC5FE30E9488E99B01AC01D7
:100F100069817A818B819C810E94B8F027966CAFA1
:100F20007DAF8EAF9FAF279769897A898B899C891E
:100F30000E9429E92FE632E143E85AE30E9488E95A
:100F40006D837E838F83988723962CAD3DAD4EAD08
:100F50005FAD239727966CAD7DAD8EAD9FAD279786
:100F60000E9488E969837A838B839C839B01AC010F
:100F70000E9441F02D813E814F8158850E94B8F03A
:100F80006D8F7E8F8F8F98A32BAD3CAD4DAD5EAD39
:100F90006D817E818F8198850E9488E929813A81BF
:100FA0004B815C810E9488E969A37AA38BA39CA3EF
:100FB00027964CAD5DAD6EAD7FAD279782E391E294
:100FC0007FDB4D815E816F8178858CE291E2B7DBBA
:100FD0008DE191E2023010F08EE091E24FDB498129
:100FE0005A816B817C8188E091E26ADB4D8D5E8D58
:100FF0006F8D78A182E091E263DB49A15AA16BA1D8
:101000007CA18CEF90E29BDB8D859E85AF85B889B6
:101010008C0D9D1DAE1DBF1DB595A7959795879508
:101020001F3F09F013CC809336072996FFAD29970F
:10103000FF9329A52F933F922F9288EE90E29F93E2
:101040008F9383EF90E29F938F931F920E94635B35
:101050003FEF231A330A0FB6F894DEBF0FBECDBFA1
:10106000898D9A8DAB8DBC8D8D839E83AF83B88720
:10107000898A9A8AAB8ABC8A6E969FAD6E972496AF
:101080009FAF249781CE8E2C0E2C000C9908F40172
:1010900083E0EE0FFF1F8A95E1F7EF59FE4F86813F
:1010A00097810F978A159B050CF48BCB87E691E20D
:1010B000E5DA0E94E42787E1889DF001899DF00D23
:1010C0001124E655FD4E8FE7828724E130E00CCDF8
:1010D000CF93DF9362E179E10E942EC6CCE2D7E0A4
:1010E0004B855C856D857E8589E099E1E9DA20E0B4
:1010F00030E543EC50E46F85788989899A890E94AC
:1011000088E9AB01BC0186E099E1DADA2CEA35EC3A
:1011100047E25EE36B897C898D899E890E9488E91C
:10112000AB01BC0183E099E10ADBDF91CF91089527
:1011300064E978E10E942EC66091790D70917A0D74
:1011400080917B0D90917C0D0E9427E9AB01BC0141
:101150008BE898E1B5DA4091A90D5091AA0D609104
:10116000AB0D7091AC0D88E898E1AADA4091AD0D15
:101170005091AE0D6091AF0D7091B00D85E898E182
:101180009FDA40918B0750918C0760918D07709189
:101190008E0782E898E1D3CACF93DF9368E378E1C2
:1011A0000E942EC6C9E6DDE04CA95DA96EA97FA903
:1011B0008FE298E185DA48AD59AD6AAD7BAD8CE23E
:1011C00098E17EDA4CAD5DAD6EAD7FAD85E898E11E
:1011D000B6DADF91CF910895CF93DF9364E178E1A0
:1011E0000E942EC6C9E6DDE04CA15DA16EA17FA1E3
:1011F0008BE098E165DA48A559A56AA57BA58DEC39
:101200009DE25EDA4CA55DA56EA57FA58AEC9DE208
:1012100057DA48A959A96AA97BA987EC9DE28FDA18
:10122000DF91CF910895CF93DF936FEE77E10E9426
:101230002EC6C9E6DDE0688179818A819B810E94A2
:1012400027E9AB01BC0186EE97E13ADA6C817D813A
:101250008E819F810E9427E9AB01BC018DEC9DE24C
:101260002FDA688579858A859B850E9427E9AB01FD
:10127000BC018AEC9DE224DA6C857D858E859F8594
:101280000E9427E9AB01BC0187EC9DE258DADF91AF
:10129000CF9108958F929F92AF92BF92EF92FF925B
:1012A0000F931F93CF93DF938FE496E1E7D9C0E0CC
:1012B000D7E0D15019F080E2C0D9FBCF8C2F0E942B
:1012C0002D6FCF5FC730A1F78AE0B7D905EB12E0E9
:1012D000C0E080E2B2D98C2F0E942D6F7801D7E058
:1012E00080E2ABD9F70180809180A280B38020E0BA
:1012F00030E0A901C501B4010E94A4F187FD02C03C
:101300008BE29BD943E0C501B4010E94E1B4D15006
:10131000FCE1EF0EF11CD111E3CF8AE08ED9CF5F53
:101320000C5F1F4FC730A9F68AE087D9DF91CF91B4
:101330001F910F91FF90EF90BF90AF909F908F9073
:101340000895811105C088E496E198D98AE075C9AD
:101350008CE496E1FACF81E496E190C98BE396E1C3
:101360008DC9CF9384E50E94E16BC0E08823D9F05A
:101370000E94536FC82F1816B4F4F0DF8DE45DD9C6
:1013800080913406909135060E94917A8EED99E114
:1013900075D96C2FCC0F770B880B990B0E9497B2E5
:1013A0008AE04BD9CFEF8C2FCF910895CF93C82FE0
:1013B00068EF78E10E9417C6C11101C0CFDF4091EC
:1013C000B5125091B6126091B7127091B8128FEEAB
:1013D00098E176D920E030E543EC50E46091B91211
:1013E0007091BA128091BB129091BC120E9488E950
:1013F000AB01BC018CEE98E163D92CEA35EC47E2F5
:101400005EE36091BD127091BE128091BF12909107
:10141000C0120E9488E9AB01BC0189EE98E150D965
:101420008AE00BD9CF910895B0E0A0E0EAE1FAE8B4
:101430000C9413F061E083E50E947D6FC1E0C82742
:1014400061ED79E18C2F0E9417C6C11101C086DFC2
:1014500089EC99E113D98EEB9FE110D98AE0EDD8A0
:1014600067EB79E18C2F0E9417C6C11101C076DFAE
:101470008AE999E103D98C2F0E9437C68C2FACDE04
:101480008C2FD1DE8C2F88DE8C2F52DE6EE479E13A
:101490008C2F0E942EC6D091B00285E499E1EED83F
:1014A0006D2F70E090E080E00E9497B24091B10211
:1014B0005091B2026091B3027091B4028AEC9DE245
:1014C000FFD888E399E1DAD88091B0023ADF20E0D2
:1014D00030E0A901609181037091820380918303C0
:1014E000909184030E9423E9882379F185EBE82E0B
:1014F00082E0F82E10E0670100E0C11101C02EDF8C
:1015000080E999E1BBD8802F0E942D6F8DE899E189
:10151000B5D8812F0E942D6F8AEC9DE2AFD8F601DD
:10152000608171818281938145E00E94E1B48AE00B
:1015300084D80F5FFCE1CF0ED11C0730F1F61F5F9E
:1015400084E0E80EF11C1730B1F662E779E18C2FE8
:101550000E9417C603E417E0D0E0C11101C0FEDE0F
:1015600089E699E18BD88D2F0E942D6FF80160815B
:101570007181072E000C880B990B0E9429E9AB01A1
:10158000BC0186E699E19CD8F80162817381072E3F
:10159000000C880B990B0E9429E9AB01BC0183E682
:1015A00099E18ED8F801E480F58080E699E166D86B
:1015B000C7010E94917A8AE040D80A5F1F4FD1305C
:1015C00059F48C2FF3DE8C2F83DD8C2F8AD8CDB786
:1015D000DEB7E8E00C942FF0D1E0BFCFACE1B0E093
:1015E000E4EFFAE80C9409F083E50E946A6B182F87
:1015F000882309F41CC10E946E6F8D838091750150
:1016000090917601A0917701B0917801898F9A8F9E
:10161000AB8FBC8F2091790130917A0140917B0191
:1016200050917C012D8B3E8B4F8B588F80917D018B
:1016300090917E01A0917F01B09180018D879E875E
:10164000AF87B88B112331F09D81911103C080E0E9
:101650000E94B67880912E0690912F06A0913006B8
:10166000B091310635E1B695A795979587953A954E
:10167000D1F79C01AD0121703327442755272987D5
:101680003A874B875C8720E030E0A90160918103B5
:101690007091820380918303909184030E9423E9D7
:1016A000882309F4C8C083E40E946A6B882309F484
:1016B00093C00E949D6F698B7A8B8B8B9C8B45EBC3
:1016C00052E05F834E838A0157E05887412C512CAA
:1016D00098EC692E92EC792E812C912C28ECA22E7C
:1016E00022E4B22E312C212CF101EE0FFF1FEE0F60
:1016F000FF1FE00FF11FC080D180E280F380A701BF
:101700009601C501B4010E9423E9181614F446019C
:101710005701A7019601C301B2010E94A4F187FFFE
:1017200002C0260137018FEF281A380A97E02916E0
:101730003104D1F6A885A150A887045E1F4FA111DE
:10174000D1CFA3019201C501B4010E9441F020E074
:1017500030E040E05FE30E9488E929893A894B89BB
:101760005C890E9441F04B015C012DEB37E346E8B8
:1017700055EB0E9423E987FD0AC02DEB37E346E8CD
:1017800055E3C501B4010E94A4F118162CF580E0C0
:101790000E94B67817E0EE80FF8007E0F7016191C4
:1017A0007191819191917F016F01F4E0CF1AD1087D
:1017B000A50194010E9440F0D6016D937D938D9315
:1017C0009C931397015051F71150EE81FF817C9645
:1017D000FF83EE831111DFCF89859A85AB85BC85A8
:1017E000892B8A2B8B2B79F020E030E0A9016091C6
:1017F00081037091820380918303909184030E94FE
:1018000023E9811147DD8AE50E946A6B882359F03C
:101810000E949D6F69837A838B839C8360E0CE01F5
:1018200001960E9442798D810E94B67814C0209161
:10183000B0022D83E3CEFD81F11108C029853A85E0
:101840004B855C85232B242B252BE9F287DD81E258
:1018500097E10E943E839D81992349F08091B002D7
:10186000811105C078DD82E097E10E943E8376DD3C
:1018700084EF96E10E943E838091B00262DD6EDDCE
:1018800087EE96E10E943E83C090B102D090B202F2
:10189000E090B302F090B40220E030E0A901C7016B
:1018A000B6010E94A4F118160CF040C042E0C70136
:1018B000B6010E94E1B48DE00E941D838AE00E947F
:1018C0001D83298D3A8D4B8D5C8D609175017091D2
:1018D000760180917701909178010E9423E981112E
:1018E0001FC02D893E894F89588D60917901709173
:1018F0007A0180917B0190917C010E9423E9811102
:101900000FC020917D0130917E0140917F01509167
:1019100080016D857E858F8598890E9423E98111DC
:101920000E94CB3F6C96E2E10C9425F082EE96E1AA
:101930000E943E83C6CFCF93DF93EB010E943E838C
:10194000BE01DD0F880B990B0E9497B2DF91CF91FA
:1019500008950E94E4270E9448448091270781301F
:1019600099F0F9DC84EC95E10E943E8360E08AEB1B
:1019700095E10E94805B6EE571E080E090E00E945E
:101980006C7A81E0809327070895CF92DF92EF92DF
:10199000FF921F93CF93DF9300D000D0CDB7DEB777
:1019A0008EEEC82E82E0D82EE12CF12CC982DA828C
:1019B000EB82FC82BE016F5F7F4F8AE50E94E5816A
:1019C00081110EC010E0812F0F900F900F900F909B
:1019D000DF91CF911F91FF90EF90DF90CF9008950E
:1019E0000E944782C982DA82EB82FC82BE016F5F6D
:1019F0007F4F8AE50E94E581182F882319F3ABDC1D
:101A000085EA96E10E943E83A4DFDDCFCF92DF928C
:101A1000EF92FF921F93CF93DF9300D000D0CDB70A
:101A2000DEB78EEEC82E82E0D82EE12CF12CC982D2
:101A3000DA82EB82FC82BE016F5F7F4F8AE00E94F8
:101A4000E58181110EC010E0812F0F900F900F9053
:101A50000F90DF91CF911F91FF90EF90DF90CF908B
:101A600008950E9447820E9402820E9419820E9469
:101A70000282C982DA82EB82FC82BE016F5F7F4FF5
:101A80008AE00E94E581182F8823E9F264DC88E669
:101A900096E10E943E835DDFD7CFEC018B01F42EEF
:101AA0000E94E427209709F47AC058DCCE010E94F6
:101AB0003E838AE00E941D830115110511F40DE19A
:101AC0001DE20E94D86F1F930F93DF93CF938AE894
:101AD00095E19F938F9381E08F930E94635B0E94B7
:101AE000D046C0917813C695C69583E793E10E94CE
:101AF0006D72DC2FDD0F1D2F1C0F8DB79EB7079663
:101B00000FB6F8949EBF0FBE8DBF83E00E94367162
:101B10004FE350E16C2F80E00E94FD741092AE13F1
:101B2000D093AF136FEF7FEF8BE795E10E94A07228
:101B30001092AE131093AF136FEF7FEF8EE695E127
:101B40000E94A07287E793E10E9494D28111DDCFB9
:101B500002DC8AE995E10E943E8389EE93E00197D9
:101B600039F000C00000EEE5F9E03197F0F7F7CF6B
:101B7000F89489EE93E0019739F000C00000E6EE9A
:101B8000F3E03197F0F7F7CF0E94E427FF2021F030
:101B90000E94FA2BA895FECF0E94B52BFBCF011512
:101BA000110511F40DE11DE2C1E9D5E18ACF809163
:101BB000B30D9091B40D2FEF3FEF981751F0E92F2F
:101BC000F0E0ED54F24F228130E09F5F9F779093D9
:101BD000B40DC90108951F920F920FB60F921124F0
:101BE0000F900FBE0F901F9018951F920F920FB677
:101BF0000F9211240BB60F922F938F939F93EF9315
:101C0000FF939091C6002091B40DE091B30D81E057
